:100000000C9444250C9475250C9475250C94752539
:100010000C9475250C9475250C9475250C947525F8
:100020000C9475250C9475250C9475250C947525E8
:100030000C9475250D941D260C9475250C9475252E
:100040000C9475250D94D4030C9475250C9475258A
:100050000C9475250C9475250D949E760D94D325DE
:100060000C9475250C94388C0C942E8C0C9475255E
:100070000C9475250C9475250C9475250C94752598
:100080000C9475250C9475250C9475250C94752588
:100090000C9475250C9475250C9475250C94752578
:1000A0000C9475250C9475250C9475250C94752568
:1000B0000C9475250C9475250C9475250C94752558
:1000C0000C9475250C9475250C9475250C94752548
:1000D0000C9475250C9475250C9475250C94752538
:1000E0000C9475258F4896484949064A584B614BF0
:1000F000714B0E56F155F4551156F755FA55FD55FD
:10010000095600561C560356065604029A028402EB
:100110005A0220015E010802D802D60230020E0205
:100120005601EC0298025E012802A802A002E80132
:100130003202760186018A026A01A4015E02FC0194
:100140007802C6013402A80144016A01EE0162018D
:100150005C01084AD73B3BCE016E84BCBFFDC12F7A
:100160003D6C74319ABD56833DDA3D00C77F11BEA8
:10017000D9E4BB4C3E916BAAAABE000000803F05AB
:10018000A84CCDB2D44EB93836A9020C50B99186DC
:1001900088083CA6AAAA2ABE000000803F07634246
:1001A00036B79BD8A71A39685618AEBAAB558C1D0E
:1001B0003CB7CC5763BD6DEDFD753EF6177231BF90
:1001C000000000803F08000000BE922449123EABB0
:1001D000AAAA2ABECDCCCC4C3E00000080BEABAA61
:1001E000AAAA3E00000000BF000000803F000000FF
:1001F0000000084178D3BB4387D1133D190E3CC39F
:10020000BD4282AD2B3E68EC8276BED98FE1A93E1D
:100210004C80EFFFBE01C4FF7F3F000000000000E4
:100220000C94B5500C9404B80C9489C40D94A0633C
:100230000C9441A50C9496480C94B9500C9478C039
:100240000D949D8B0C9401C30D943E250C94614B31
:100250000C94A9500D94757F0C94A7C40C94F5BB15
:100260000C9406560C947BBE0C94C5C40C9473631A
:100270000C944AC60C94AF9D0D94C6260C94BD50A8
:100280000C940E560C9449490D94C48C0C941C5635
:100290000C94735C0C94B9C20C94ECB80D94556634
:1002A0000D9439270C94E3C40C94F1BF0D94C28BC8
:1002B0000C9441C60C94C16A0D94E28C0D94DD8BB4
:1002C0000C947FB60D94D88C0C9449790C944A56B2
:1002D0000C94A05A0D94EC8C0C94936A0C943CB83A
:1002E0000C949D500C94828D0D94A5630D945F8C9D
:1002F0000C94AA6A0C94F0770C944D5E0C94ABB6F7
:100300000C94DC6F0C94365A0D94D9260D94698C9C
:100310000C9492C40C9410C30C947C800D94C7264A
:100320000D9454840C944AC00D9489250C94064A6B
:100330000C94E6C20C9411560C94966F0C941FC644
:100340000C947A9C0C946B630D947D8C0D94B86620
:100350000D94BA8C0C94C8C20C9464A30C94985954
:100360000C94A7560C94DDC40C94C1500C944076A8
:100370000C94FA550D9445630C948ABD0C94315637
:100380000C9418C00C944F5A0C94F7550D94A18CF2
:100390000C94C7560D94AF630C94B9C40C94C55516
:1003A0000C94F4550D9404AB0D940FA80C94635A5F
:1003B0000C94045A0C9445C20D948F630C9465C040
:1003C0000D945C7F0D9478690D94C8830C94B3C42C
:1003D0000D94558C0C946F5A0C94E77E0D94CE8C32
:1003E0000C94439B0C9409560C94B9610D94D567F9
:1003F0000C94D1550D9468250D948D8C0C941D5A38
:100400000C94D86A0C9450C20D94A38B0C94D1C454
:100410000D94AA8B0C94879F0C94499C0D94BC8BD3
:100420000C94C7500C947C6A0C94CA500C94F081C4
:100430000C94CBC40C94BFC40C94B74D0C94A59DE4
:100440000D94AA630C943EBC0C94C4500C945F535E
:100450000D94D08B0C941FC30C94499F0C94584B53
:100460000D94B88B0D945A8C0D94AB8C0C945878D9
:100470000C94A2B60C944F4E0D94607F0C94E1B690
:100480000C94A5500C94CFB90C9431C00D94C16656
:100490000C9400560D9464660C945F670C94D7C45A
:1004A0000D94F4750D940B7F0C946F630C948F482E
:1004B0000D9495630D94998B0C949BBA0D94858C37
:1004C0000C947A600C94B7C00C941BC60C94F3BBCC
:1004D0000D94CE630C941E560D949B630D9489630A
:1004E0000D94A4250C945F4C0C94FF770C945D4CF8
:1004F0000D94978C0C941DC60C9471630D94D72F9A
:100500000C94AD500C94D2540D94958B0D94836340
:100510000C9403560D94738C0C947E4C0C941BBA63
:100520000C946D630C94F2C20C94A1500C94194D70
:100530000D94CA8B0D94A68B0C9419C60C94AA9D8D
:100540000D94D88B0C94DB9E0C94A65A0C9445BC4D
:100550000D94D48B0C94ADC40D945A660C94FD5537
:100560000C94FFBF0C94D0C00D944D630D945F6646
:100570000C949A5A0C94F1550C94B1500C94A1C45B
:100580000C94F1BB0C94E9C00C945B670D94717FE3
:100590000D9475250C94A4C00C94815A0C94FAC542
:1005A0000C94A7C60C9499500C9402C10D94B48B72
:1005B0000D94AE8B0C94714B0C94D7C20D940663C2
:1005C0000C94D5560C948BC00C9432C60C94DB6AF8
:1005D0000C94945A0D94AE830D94C68B4E414E49A3
:1005E0004E495459494E46CDCCCC3D0AD7233C17F1
:1005F000B7D13877CC2B329595E6241FB14F0A003E
:100600000020410000C84200401C4620BCBE4CCA2D
:100610001B0E5AAEC59D7400407A10F35A00A072AA
:100620004E18090010A5D4E80000E876481700002D
:10063000E40B54020000CA9A3B000000E1F50500FB
:100640000080969800000040420F000000A0860144
:10065000000000102700000000E803000000006414
:1006600000000000000A000000000001000000007F
:10067000002C76D888DC674F0823DFC1DFAE59E154
:10068000B1B796E5E3E453C63AE651997696E8E6C3
:10069000C28426EB898C9B62ED407C6FFCEFBC9C96
:1006A0009F40F2BAA56FA5F490055A2AF75C936BA8
:1006B0006CF9676DC11BFCE0E40D47FEF520E6B563
:1006C00000D0ED902E0300943577050080841E083D
:1006D0000000204E0A000000C80C333333330F985B
:1006E0006E12831141EF8D2114893BE65516CFFE22
:1006F000E6DB18D1844B381BF77C1D901DA4BBE4AE
:1007000024203284725E228100C9F124ECA1E53DEF
:1007100027434F4D4D554E49434154494F4E004498
:10072000525952554E004552524F525300494E466F
:100730004F004543484F0047322F473320626164E2
:1007400020706172616D65746572730A00536C6527
:1007500065702E2E2E00205A3A200020593A200093
:1007600042656420583A20004D65736820706F69B7
:100770006E74206F7574206F662072616E67650AF3
:1007800000436C69636B20746F20526573756D65EF
:100790002E2E2E004E6F204D6F76652E00456E6416
:1007A0002066696C65206C6973740A00426567692C
:1007B0006E2066696C65206C6973740A004E6F2048
:1007C0006D656469610A00286E6F2066696C652931
:1007D0000043757272656E742066696C653A20001C
:1007E0005344207072696E74696E67206279746513
:1007F00020004E6F74205344207072696E74696ECD
:10080000670A0044656C6574696F6E206661696C87
:1008100065642C2046696C653A200046696C652049
:1008200064656C657465643A00256979202569649E
:10083000202569682025696D20256973005072693B
:100840006E742074696D653A200045202553006F51
:1008500066660044454255473A004D3131322053D7
:10086000687574646F776E004D31313320530042E8
:10087000656420436F6F6C696E672E2E2E00426593
:10088000642048656174696E672E2E2E00416E7972
:100890006375626963204B6F7373656C204F4646C6
:1008A0002E004348414D4245525F54454D504552FC
:1008B00041545552450042414259535445505049C4
:1008C0004E470041524353004D4F54494F4E5F4DE8
:1008D0004F44455300544845524D414C5F50524F90
:1008E00054454354494F4E004C4F4E475F46494C88
:1008F000454E414D45004155544F5245504F52547D
:100900005F53445F53544154555300534443415241
:10091000440050524F4D50545F535550504F525415
:1009200000454D455247454E43595F50415253454E
:100930005200434153455F4C494748545F42524936
:100940004748544E45535300544F47474C455F4C1E
:10095000494748545300534F4654574152455F50FE
:100960004F574552004255494C445F50455243450C
:100970004E54004C4556454C494E475F4441544106
:10098000005A5F50524F42450052554E4F55540049
:100990004155544F4C4556454C005052494E545FBA
:1009A0004A4F420050524F4752455353004155540D
:1009B0004F5245504F52545F54454D5000564F4C86
:1009C000554D45545249430042494E4152595F46A4
:1009D000494C455F5452414E53464552005345528F
:1009E00049414C5F584F4E5F584F4646004649526A
:1009F0004D574152455F4E414D453A4D61726C69CC
:100A00006E20322E302E372E32202844656320325D
:100A10003820323032302031323A32393A353629C4
:100A200020534F555243455F434F44455F55524C09
:100A30003A68747470733A2F2F6769746875622E00
:100A4000636F6D2F4D61726C696E4669726D77616F
:100A500072652F4D61726C696E2050524F544F4336
:100A60004F4C5F56455253494F4E3A312E30204D30
:100A7000414348494E455F545950453A416E796368
:100A800075626963204B6F7373656C2045585452CF
:100A9000554445525F434F554E543A3120555549C0
:100AA000443A63656465326132662D343161322DBA
:100AB000343734382D396231322D6335356336326F
:100AC0006633363766660A002F2F20004D313435E5
:100AD00020533C696E6465783E206F7574206F66A4
:100AE0002072616E67652028302D31290A0041632C
:100AF00063656C65726174696F6E3A20500057418E
:100B0000524E494E4721204C6F77205A204A657239
:100B10006B206D6179206C65616420746F20756E47
:100B200077616E746564207061757365732E0A0059
:100B300046523A0020466C6F773A200020643A0013
:100B400020693A0020703A006469730043290A0062
:100B500061626C656420286D696E2074656D70201B
:100B600000436F6C642065787472756465732061EE
:100B7000726520004D34323120696E636F72726588
:100B8000637420706172616D657465722075736144
:100B900067650A00454550524F4D204F4B0A004DA6
:100BA000383420582059205A204500446F6E652063
:100BB0007072696E74696E672066696C650A004DB3
:100BC0003737004D33310032072D0726071F071135
:100BD00007204A0020204D34323120490020204790
:100BE000323920493939390A006163746976650AF6
:100BF000002053797374656D2076312E30312000DA
:100C00002020207C0A004E414E0020202E20202053
:100C100000207C004C43443A0A004353563A0A00F1
:100C200020666F7220003A0A0A000A426564205466
:100C30006F706F677261706879205265706F72743F
:100C40000050726F62696E67204661696C65640A64
:100C50000050726F62696E67204661696C6564005E
:100C6000446F6E652E0A003F496E76616C696420A0
:100C700073746F7261676520736C6F742E0A3F55D1
:100C80007365203020746F200047323920503220A5
:100C900066696E69736865642E0A005859206F751D
:100CA0007473696465207072696E7461626C65202A
:100CB0007261646975732E0A003F4572726F72200B
:100CC000696E20427573696E657373204361726447
:100CD000206D6561737572656D656E742E0A004DC9
:100CE000616E75616C6C792070726F62696E6720DD
:100CF000756E726561636861626C6520706F696EA4
:100D000074732E0A0050726F62696E672061726F91
:100D1000756E642028004D65736820696E76616C7D
:100D20006964617465642E2050726F62696E672019
:100D30006D6573682E0A004D657368207A65726F61
:100D400065642E0A0044656661756C742073746F67
:100D50007261676520736C6F7420302073656C65F9
:100D6000637465642E0A004C6F6164696E67207459
:100D70006573745F7061747465726E2076616C75F2
:100D800065732E0A0A00496E76616C696420746589
:100D900073745F7061747465726E2076616C7565D2
:100DA0002E20282D3120746F2032290A0A004C6F22
:100DB000636174696F6E7320696E76616C696461DA
:100DC0007465642E0A0A00456E74697265204D656B
:100DD000736820696E76616C6964617465642E0A5B
:100DE0000A00554E4C4F41442046494C414D454E1A
:100DF000540046494C414D454E54204348414E47CE
:100E00004500436F6E66696775726174696F6E0045
:100E10004D37303220542564004D3630302042307A
:100E200020542564004D373032203B2564004D3777
:100E3000303120542564004D373032004D37303189
:100E4000004D36303020423000436F6E74696E754D
:100E500065005075726765206D6F7265005245536D
:100E6000554D45204F5054494F4E533A005052492A
:100E70004E54205041555345440020204E6F7A7AFD
:100E80006C653A2000313530004245443A204154E7
:100E9000432031303447542D320052756E617761F2
:100EA000792057617463683A204F4E004D61782075
:100EB00054656D7000323735004D696E2054656D94
:100EC000700045313A204154432031303447542D8D
:100ED00032005053550047656E6572696300507269
:100EE0006F746F636F6C00312E3000426175640067
:100EF00032353030303000416E796375626963207D
:100F000052414D505320312E34004578747275642F
:100F100065727300416E796375626963204B6F730C
:100F200073656C00323032302D31302D3135005444
:100F30006865726D6973746F727300426F61726479
:100F400020496E666F005072696E74657220496E3A
:100F5000666F0053746F70004368616E6765204D63
:100F600065646961004D3231004175746F7374615D
:100F700072740041626F7574205072696E7465728C
:100F800000526573756D65205072696E74004E6F06
:100F9000204D656469610054756E650053746F700F
:100FA000205072696E7400506175736520507269CB
:100FB0006E74005061726B696E672E2E2E000000F9
:100FC0005761697420666F720066696C616D656E49
:100FD00074206368616E676500746F20737461725A
:100FE00074005761697420666F720066696C616D88
:100FF000656E7420756E6C6F616400004E6F7A7A56
:101000006C652068656174696E6700506C6561731A
:101010006520776169742E2E2E00005072657373FF
:1010200020627574746F6E00746F2068656174203F
:101030006E6F7A7A6C650000496E73657274206613
:10104000696C616D656E7400616E642070726573A9
:101050007320627574746F6E00746F20636F6E74AA
:10106000696E7565005761697420666F7200666904
:101070006C616D656E74206C6F6164000050726508
:10108000737320427574746F6E00746F2072657391
:10109000756D65207072696E740000576169742007
:1010A000666F72207072696E7400746F207265735F
:1010B000756D652E2E2E00005761697420666F7263
:1010C0000066696C616D656E74207075726765008D
:1010D0000050726F6265205A204F66667365740017
:1010E000416476616E6365642053657474696E67EC
:1010F0007300547A00547900547800457A00457999
:1011000000457800526573746F72652044656661AE
:10111000756C7473004C6F61642053657474696EF0
:1011200067730053746F72652053657474696E67DA
:10113000730050726568656174202420436F6E6689
:101140000044656C74612043616C6962726174690A
:101150006F6E00436F6E74726F6C6C6572204661C7
:101160006E004465627567204D656E750044696167
:101170006720526F64005261646975730043616C4B
:10118000696272617465205A0043616C69627261C0
:10119000746520590043616C6962726174652058FE
:1011A0000044656C74612053657474696E677300E4
:1011B00043616C6962726174652043656E74657227
:1011C000004175746F2043616C6962726174696F6C
:1011D0006E0047333300504944204175746F747575
:1011E0006E65202A005049442D44202A005049446D
:1011F0002D49202A005049442D50202A0020022049
:1012000046616374002002204D6178002002204D69
:10121000696E004175746F74656D7000565472612B
:1012200076204D696E00566D696E00566D617820AE
:101230004500566D6178204300566D61782042006C
:10124000566D6178204100416D6178204500416D07
:101250006178204300416D6178204200416D6178E2
:10126000204100412D54726176656C00412D52651C
:10127000747261637400416363656C0056652D4A46
:1012800065726B0056432D4A65726B0056422D4ABB
:1012900065726B0056412D4A65726B00456E636C3A
:1012A0006F73757265004D6F76696E672E2E2E0016
:1012B0004C6F6164206D6D00556E6C6F6164206DC4
:1012C0006D0046696C2E204469612E004520696ED0
:1012D000206D6DC2B3004D3330332055312045258C
:1012E000692053256900473239205034205239395A
:1012F000392054004732380A473239205031004DE6
:101300006F74696F6E00473238004F666620507206
:10131000696E746572204261636B75700047323983
:1013200020532D31004F757470757420666F7220D4
:1013300043535600473239205431004F757470754D
:101340007420666F7220486F7374004732392054DE
:10135000300045646974204D657368004D616E7599
:10136000616C6C79204275696C64204D657368000E
:1013700047323920493939390A4732392050322029
:101380004220543000372E20536176652042656438
:10139000204D65736800362E2046696E65205475B1
:1013A0006E6520416C6C00352E2056616C6964615D
:1013B0007465204D65736800342E2046696E652083
:1013C00054756E6520416C6C00332E2056616C693B
:1013D00064617465204D65736800322E20536D6121
:1013E00072742046696C6C2D696E0047323920504A
:1013F0003320543000312E204275696C6420436FD5
:101400006C64204D657368004F7574707574205559
:10141000424C20496E666F004732392057005542D2
:101420004C20546F6F6C73004F7574707574204D41
:10143000657368204D6170004D6573682053746F4B
:1014400072616765004D6573682045646974005377
:101450007465702D42792D537465702055424C008F
:1014600041637469766174652055424C0047323996
:10147000204100446561637469766174652055425A
:101480004C004732392044002568753A25303268CF
:10149000750025303268753A25303268750053443E
:1014A0000050726F7465637465642050696E0A0041
:1014B000726F746174696F6E206D61747269783ACD
:1014C0000A005A5F6D6F76655F636F6D700A00206A
:1014D0006D61783A00206D696E3A00417869732039
:1014E00000534C4F57005072696E746572207374CC
:1014F0006F707065642064756520746F206572720A
:101500006F72732E20466978207468652065727248
:101510006F7220616E6420757365204D39393920F2
:10152000746F20726573746172742E202854656D17
:101530007065726174757265206973207265736578
:10154000742E20536574206974206166746572205E
:1015500072657374617274696E67290A00457272EC
:101560006F722077726974696E6720746F204545C9
:1015700050524F4D210A004D343130004D3131323F
:10158000004D3130380053544F505045442E200008
:101590004E6F20436865636B73756D20776974685F
:1015A000206C696E65206E756D6265722C204C61D1
:1015B0007374204C696E653A2000636865636B73D1
:1015C000756D206D69736D617463682C204C617357
:1015D00074204C696E653A20004C696E65204E752A
:1015E0006D626572206973206E6F74204C61737434
:1015F000204C696E65204E756D6265722B312C2012
:101600004C617374204C696E653A20004D31313065
:101610000053442072656164206572726F720A0023
:101620002121204B494C4C20636175736564206215
:1016300079204B494C4C20627574746F6E2F706921
:101640006E0A002121204B494C4C20636175736563
:101650006420627920746F6F206D75636820696EF5
:101660006163746976652074696D65202D206375EA
:101670007272656E7420636F6D6D616E643A2000E6
:10168000627573793A2070617573656420666F7254
:1016900020696E7075740A00627573793A20706102
:1016A0007573656420666F7220757365720A0062D7
:1016B0007573793A2070726F63657373696E670A28
:1016C000004D656469612052656D6F766564004DFB
:1016D0006564696120496E73657274656400506C5D
:1016E00065617365205265736574005052494E54AC
:1016F00045522048414C5445440025533A20255337
:10170000004B494C4C45442E20005072696E746564
:10171000722068616C7465642E206B696C6C28297A
:101720002063616C6C6564210A006563686F3A0030
:101730004572726F723A000000B4420000B4420079
:1017400000A0430000B4C20000B4C20000000002C8
:1017500002020000F0410000F0410000F0410000F2
:10176000A0400000A0400000A04000003443000062
:1017700034430000A043010101000000010000000B
:101780000100008000555555000000400033333300
:1017900000AAAA2A004992240000002000C7711C58
:1017A0000099991900D1451700555515003BB11303
:1017B000002449120011111100000010000F0F0F3A
:1017C00000E3380E0043790D00CCCC0C00C3300C84
:1017D00000E8A20B0064210B00AAAA0A00703D0ACF
:1017E000009DD80900427B090092240900DCD3083F
:1017F00000888808001042080000000800F0C107B7
:10180000008787070075500700711C07003EEB0634
:1018100000A1BC06006990060066660600703E06E0
:10182000006118060017F4050074D105005BB005CF
:1018300000B2900500627205005555050078390523
:1018400000B81E0500050505004EEC040087D40411
:1018500000A1BD040090A7040049920400C17D04CA
:1018600000EE690400C7560400444404005C3204DE
:10187000000821040041100400000004003FF003B0
:1018800000F8E0030026D20300C3C30300CCB50375
:10189000003AA803000A9B0300388E0300C08103AE
:1018A000009F750300D0690300505E03001D5303C1
:1018B0000034480300913D0300333303001629032D
:1018C00000381F030097150300300C0300030303C7
:1018D000000BFA020049F10200BAE802005CE002E3
:1018E000002DD802002DD0020059C80200B0C0025D
:1018F0000031B90200DAB10200AAAA0200A0A302D4
:1019000000BC9C0200FA9502005C8F0200DF880296
:101910000082820200457C020027760200277002C6
:1019200000436A02007C640200D05E02003F59025C
:1019300000C8530200FFFDFCFAF8F6F4F2F0EEECFA
:10194000EAE9E7E5E3E1E0DEDCDAD9D7D5D4D2D0C5
:10195000CFCDCBCAC8C7C5C3C2C0BFBDBCBAB9B75B
:10196000B6B4B3B2B0AFADACAAA9A8A6A5A4A2A1C3
:10197000A09E9D9C9A99989795949392908F8E8D06
:101980008B8A8988878684838281807F7E7D7B7A2B
:10199000797877767574737271706F6E6D6C6B6A2F
:1019A000696867666564636261605F5E5D5C5B5A1F
:1019B0005958585756555453525150504F4E4D4CFC
:1019C0004B4A4A4948474646454443424241403FC4
:1019D0003E3E3D3C3B3B3A3938383736353534337B
:1019E00032323130302F2E2E2D2C2B2B2A29292824
:1019F000272726252524232322212120201F1E1EC0
:101A00001D1C1C1B1B1A191918181716161515144E
:101A1000131312121111100F0F0E0E0D0D0C0C0BD3
:101A20000A0A09090808070706060505040403034E
:101A300002020100005761726E696E673A20486FBA
:101A40006D696E672042756D702044697669736FA9
:101A500072203C20310A00496E666F205363726524
:101A6000656E00473239204A2569004C6576656C01
:101A7000204D657368005369646520506F696E740A
:101A8000730047726964204D657368204C65766504
:101A90006C696E6700332D506F696E74204C6576EB
:101AA000656C696E6700473239204A300047323929
:101AB000205033205220432E2569004D616E756100
:101AC0006C2046696C6C2D696E0046696C6C2D69E2
:101AD0006E20416D6F756E74004D65736820696E80
:101AE00076616C6964617465642E0A00496E766182
:101AF0006C696461746520436C6F7365737400472F
:101B00003239204900496E76616C696461746520E0
:101B1000416C6C00436F6E74696E7565204265643C
:101B2000204D65736800473239205031204300460C
:101B3000696C6C2D696E204D657368004275696C27
:101B40006420437573746F6D204D65736800473270
:101B5000380A4D3139302049310A4D313039204968
:101B6000310A4732392050310A4D31303420533058
:101B70000A4D313430205330004275696C64204D79
:101B800065736820282429004732380A4D313930DE
:101B90002049300A4D3130392049300A4732392046
:101BA00050310A4D3130342053300A4D3134302019
:101BB00053300047323920256325690A4D313137CA
:101BC00020004D657368202569204C6F6164656451
:101BD000004D657368202569205361766564004C6B
:101BE0006F616420426564204D657368004D656DCA
:101BF0006F727920536C6F74004E6F2053746F7244
:101C000061676500473239205034205825732059C8
:101C100025732052256900202D2D2D2D2D00486F74
:101C20006D696E672058595A004361703A003F5AF7
:101C3000206F7574206F662072616E6765202800C2
:101C40003F59206F7574206F662072616E67652042
:101C5000282D003F58206F7574206F662072616ECA
:101C6000676520282D0050726F6265204F6666738D
:101C70006574205800656E7175657565696E6720BD
:101C800022006F6B00526573656E643A2000236416
:101C90006566696E652044454641554C545F004B6E
:101CA0006420004B6920004B7020005049442041C3
:101CB00075746F74756E652066696E6973686564A6
:101CC000212050757420746865206C617374204BFA
:101CD000702C204B6920616E64204B6420636F6E12
:101CE0007374616E74732066726F6D2062656C6FC1
:101CF0007720696E746F20436F6E666967757261D5
:101D000074696F6E2E680A00504944204175746FE3
:101D100074756E65206661696C6564212074696DF7
:101D2000656F75740A000A20436C617373696320E0
:101D3000504944200A00204B643A2000204B693A65
:101D40002000204B703A20000A204E6F206F7665ED
:101D50007273686F6F740A002054753A2000204B2C
:101D6000753A2000206D61783A2000206D696E3A46
:101D7000200020643A200020626961733A200050FC
:101D80004944204175746F74756E65207374617277
:101D9000740A00504944204175746F74756E652053
:101DA0006661696C6564212054656D70657261744B
:101DB00075726520746F6F20686967680A00504902
:101DC00044204175746F74756E650050494420411C
:101DD00075746F74756E65206661696C6564212029
:101DE000426164206578747275646572206E756DE9
:101DF0006265720A007C4D61726C696E7C002D2DEB
:101E00002D2D2D2D00A10000006900A2000000630F
:101E100000B00000000900C10000004100C2000045
:101E2000004100C30000004100C40000004100C5A3
:101E30000000004100C60000004145C7000000430B
:101E400000C80000004500C90000004500CD0000AA
:101E5000004900D10000004E00D50000004F00D620
:101E60000000004F00D70000007800DC00000055A3
:101E700000DD0000005900E00000006100E100000A
:101E8000006100E20000006100E30000006100E486
:101E90000000006100E50000006100E60000006154
:101EA00065E70000006300E80000006500E900004D
:101EB000006500EA0000006500EB0000006500EC32
:101EC0000000006900ED0000006900EE00000069FC
:101ED00000EF0000006900F10000006E00F2000059
:101EE000006F00F30000006F00F40000006F00F5C9
:101EF0000000006F00F60000006F00F80000006FA7
:101F000000F90000007500FA0000007500FB0000F9
:101F1000007500FC0000007500FD0000007900FF66
:101F2000000000790004010000410005010000618B
:101F3000000601000043000701000063000C0100DF
:101F40000043000D01000063000E01000044000F7B
:101F50000100006400110100006400190100006527
:101F6000001A01000045001B01000065001F010070
:101F700000670030010000490031010000690041A4
:101F80000100004C00420100006C00430100004EC3
:101F900000440100006E00480100006E005801007E
:101FA0000052005901000072005A01000053005B0A
:101FB00001000073005F0100007300600100005326
:101FC000006101000073006501000074006F0100F2
:101FD0000075007C0100007A007D0100005A007E3F
:101FE0000100007A00920100006600E30200007820
:101FF00000222000002E001E210000507822210027
:1020000000544D902100003C2D922100002D3EB047
:102010002100000300BB21000004003C2200007EE0
:1020200000482200007E3D60220000213D61220028
:10203000003D00642200003C3D652200003E3DF171
:102040002300000700A03000003D0021F301000242
:1020500000C2F401000500A2000000EC00B0000086
:1020600000DF00E4000000E100F6000000EF00F7F0
:10207000000000FD00FC000000F500E3020000EBA2
:102080000087030000A5008F030000F40098030000
:1020900000F2009E030000E300A3030000F600A985
:1020A000030000F400AC030000E000AD030000E317
:1020B00000B1030000E000B2030000E200B503003D
:1020C00000E300B8030000F200BC030000E400BE1F
:1020D000030000E300C0030000F700C1030000E6B6
:1020E00000C3030000E500902100007F0092210062
:1020F000007E001A220000E8001E220000F3008883
:10210000250000FF0002300000A1000C300000A2FA
:10211000000D300000A3009B300000DE009C30006A
:1021200000DF00A03000003D00A1300000A700A2A9
:10213000300000B100A3300000A800A4300000B2BD
:1021400000A5300000A900A6300000B300A73000B1
:1021500000AA00A8300000B400A9300000AB00AA1B
:10216000300000B500AB300000B600AC300000B667
:10217000DEAD300000B700AE300000B7DEAF30009B
:1021800000B800B0300000B8DEB1300000B900B2D5
:10219000300000B9DEB3300000BA00B4300000BA3D
:1021A000DEB5300000BB00B6300000BBDEB730004B
:1021B00000BC00B8300000BCDEB9300000BD00BA81
:1021C000300000BDDEBB300000BE00BC300000BEF1
:1021D000DEBD300000BF00BE300000BFDEBF3000FB
:1021E00000C000C0300000C0DEC1300000C100C22D
:1021F000300000C1DEC3300000AF00C4300000C2B8
:1022000000C5300000C2DEC6300000C300C7300089
:1022100000C3DEC8300000C400C9300000C4DECAFC
:10222000300000C500CB300000C600CC300000C735
:1022300000CD300000C800CE300000C900CF300013
:1022400000CA00D0300000CADED1300000CADFD2A0
:10225000300000CB00D3300000CBDED4300000CB08
:10226000DFD5300000CC00D6300000CCDED7300007
:1022700000CCDFD8300000CD00D9300000CDDEDA50
:10228000300000CDDFDB300000CE00DC300000CEBF
:10229000DEDD300000CEDFDE300000CF00DF3000BA
:1022A00000D000E0300000D100E1300000D200E2B8
:1022B000300000D300E3300000AC00E4300000D474
:1022C00000E5300000AD00E6300000D500E730004A
:1022D00000AE00E8300000D600E9300000D700EA88
:1022E000300000D800EB300000D900EC300000DAFC
:1022F00000ED300000DB00EF300000DC00F23000C9
:1023000000A600F3300000DD00F4300000B3DEF77B
:10231000300000DCDEFA300000A6DEFB300000A555
:1023200000FC300000B000FD300000A400074E00AB
:1023300000FB0086510000FC0043530000FA0064DB
:10234000FF0000A40065FF0000A50066FF0000A6D6
:102350000067FF0000A70068FF0000A80069FF00F9
:1023600000A9006AFF0000AA006BFF0000AB006C30
:10237000FF0000AC006DFF0000AD006EFF0000AE7E
:10238000006FFF0000AF0070FF0000B00071FF00A1
:1023900000B10072FF0000B20073FF0000B30074D0
:1023A000FF0000B40075FF0000B50076FF0000B626
:1023B0000077FF0000B70078FF0000B80079FF0049
:1023C00000B9007AFF0000BA007BFF0000BB007C70
:1023D000FF0000BC007DFF0000BD007EFF0000BECE
:1023E000007FFF0000BF0080FF0000C00081FF00F1
:1023F00000C10082FF0000C20083FF0000C3008410
:10240000FF0000C40085FF0000C50086FF0000C675
:102410000087FF0000C70088FF0000C80089FF0098
:1024200000C9008AFF0000CA008BFF0000CB008CAF
:10243000FF0000CC008DFF0000CD008EFF0000CE1D
:10244000008FFF0000CF0090FF0000D00091FF0040
:1024500000D10092FF0000D20093FF0000D300944F
:10246000FF0000D40095FF0000D50096FF0000D6C5
:102470000097FF0000D70098FF0000D80099FF00E8
:1024800000D9009AFF0000DA009BFF0000DB009CEF
:10249000FF0000DC009DFF0000DD009EFF0000DE6D
:1024A000009FFF0000DF00E5FF00005C000010104F
:1024B000101010100000141414141414000015153A
:1024C0001515151500001C1F11111F00000006191D
:1024D0001803130C00040E1F041C000000000E1350
:1024E00015110E00001C10181705060500040A0A35
:1024F0000A0A11110E0C12120C00000000001F1528
:1025000011151F000000000000010204040000007B
:102510001C1C0C040404020100000000000408104C
:10252000000000000054656D70657261747572651D
:102530000046616E205370656564004D61696E00F0
:102540005072656865617420242042656400507291
:102550006568656174202420456E6400436F6F6C6C
:10256000646F776E00466C6F77005A2056616C7509
:1025700065004732380A4D313930205325690A4DFC
:10258000313039205325690A473239205031004211
:1025900065642054656D7000486F74656E642054E6
:1025A000656D70004732392050362043202D004899
:1025B000656967687420416D6F756E740041646A67
:1025C000757374204D657368204865696768740089
:1025D00046696E652054756E6520436C6F73657334
:1025E00074004732392050342054004732380A47AB
:1025F0003236204320502048256920422569005664
:10260000616C696461746520437573746F6D204DEE
:10261000657368004732380A47323620432050201D
:1026200049310056616C6964617465204D65736859
:1026300020282429004732380A47323620432050C8
:102640002049300050726F62652059204F666673D2
:1026500065740050726F62652058204F666673651E
:102660007400452073746570732F6D6D00432053A3
:10267000746570732F6D6D00422053746570732FF5
:102680006D6D00412053746570732F6D6D00496E40
:1026900069740050726F6265204F6666736574736B
:1026A00000416363656C65726174696F6E005665A5
:1026B0006C6F636974790050726F67726573732011
:1026C00042617220546573740049646C65205065E2
:1026D00072696F6400416374697665205370656543
:1026E00064004175746F204D6F64650049646C65CA
:1026F000205370656564005072696E742066726F55
:102700006D204D656469610020746F6F206C6F6E81
:102710006720657874727573696F6E207072657664
:10272000656E7465640A0020636F6C64206578745C
:10273000727573696F6E2070726576656E7465640C
:102740000A00486F6D65202573257325732046693F
:1027500072737400496E736572742066696C616D82
:10276000656E7420616E642070726573732062758B
:1027700074746F6E0A00220A00556E6B6E6F776E6E
:1027800020636F6D6D616E643A20220020453A002F
:10279000205A3A0020593A007879007A7800797AFC
:1027A00000207A002079002078002E2020202000B0
:1027B000456E64204452592D52554E004E6F206391
:1027C0006F6E76657267656E6365004974657261E8
:1027D00074696F6E203A2025303269005361766546
:1027E0002077697468204D35303020616E642F6F1A
:1027F0007220636F707920746F20436F6E66696713
:1028000075726174696F6E2E680A00253033692E07
:102810007800302E253033690043616C6962726143
:1028200074696F6E2073643A007374642064657613
:102830003A00726F6C6C696E67206261636B2E0088
:1028400043616C6962726174696F6E204F4B004323
:102850006F72726563742064656C74612073657453
:1028600074696E67732077697468204D3636352039
:10287000616E64204D3636360A0020284452592DA8
:1028800052554E2900436865636B696E672E2E2E84
:10289000204143003F4265642063616C696272615C
:1028A00074696F6E2072616469757320696D706CF4
:1028B00061757369626C652E0A0047333320417578
:1028C000746F2043616C6962726174650A003F280D
:1028D00056296572626F7365206C6576656C206938
:1028E0006D706C61757369626C652028302D3329B9
:1028F0002E0A003F2846296F72636520697465724D
:102900006174696F6E20696D706C61757369626C5A
:10291000652028302D3330292E0A003F28432961B5
:102920006C6962726174696F6E207072656369733D
:10293000696F6E20696D706C61757369626C65207A
:10294000283E3D30292E0A003F2850296F696E74B9
:102950007320696D706C61757369626C65202830D5
:102960002D3130292E0A0053746F77205A2D507262
:102970006F6265004465706C6F79205A2D50726FDC
:1029800062650053657474696E67732053746F7267
:102990006564002062797465733B20637263200074
:1029A00053657474696E67732053746F7265642025
:1029B00028004E6F20454550524F4D2E0A00454588
:1029C00050524F4D206461746173697A652065725D
:1029D000726F722E0A003F4D65736820746F6F200E
:1029E00062696720666F7220454550524F4D2E0A2E
:1029F0000055424C2072657365740A00206C6F614B
:102A00006465642066726F6D2073746F72616765B0
:102A10002E0A004D65736820003F43616E277420C5
:102A2000656E61626C65200020696E697469616C15
:102A3000697A65642E0A0A002073746F72656420D7
:102A400073657474696E67732072657472696576F4
:102A50006564202800202863616C63756C6174656F
:102A60006429210A0020213D2000454550524F4D48
:102A700020435243206D69736D61746368202D207B
:102A80002873746F726564292000496E6465783A12
:102A9000200044494749504F5453204C6F616465AE
:102AA000640A0044494749504F5453204C6F6164B5
:102AB000696E670A00204D61726C696E3D5638324E
:102AC000290A00454550524F4D2076657273696F53
:102AD0006E206D69736D617463682028454550529E
:102AE0004F4D3D0024F4D43050C38E20C2A2401775
:102AF000828B7011127A910D816CD90AA861E1085C
:102B0000C7586607615143061E4B5D05C145A704C2
:102B10001A411104093D9803713931034036DB0233
:102B200065339102D4305402802E1D02632CEE01D5
:102B3000752AC501B028A001102781018F256401E5
:102B40002B244B01E0223401AC211F018D200D010B
:102B5000801FFC00841EED00971DDF00B81CD20012
:102B6000E61BC600201BBC00641AB200B219A80004
:102B70000A19A0006A189900D117910040178B001C
:102B8000B516840031167E00B31579003A1573002E
:102B9000C7146F0058146A00EE13660088136300B0
:102BA00025135E00C7125B006C125700151254000B
:102BB000C111510070114F0021114B00D610490076
:102BC0008D1047004610440002104200C00F400024
:102BD000800F3E00420F3C00060F3B00CB0E38003A
:102BE000930E37005C0E3500270E3400F30D3200D3
:102BF000C10D3100900D3000600D2E00320D2D0002
:102C0000050D2C00D90C2B00AE0C2900850C2900D9
:102C10005C0C2700350C27000E0C2600E80B240066
:102C2000C40B2400A00B23007D0B23005A0B2100B2
:102C3000390B2100180B2000F80A1F00D90A1E00CA
:102C4000BB0A1E009D0A1D00800A1D00630A1C00AD
:102C5000470A1B002C0A1B00110A1A00F7091A0068
:102C6000DD091900C4091900AB0919009209170000
:102C70007B091800630917004C0916003609160075
:102C8000200916000A091500F5081500E0081400CF
:102C9000CC081400B8081400A4081400900813000D
:102CA0007D0812006B081300580812004608120035
:102CB0003408110023081100120811000108110046
:102CC000F0071000E0071000D0071000C007100048
:102CD000B0070F00A107100091070E0083070F0037
:102CE00074070F0065070E0057070E0049070E0016
:102CF0003B070D002E070E0020070D0013070D00E7
:102D000006070D00F9060C00ED060D00E0060C00AC
:102D1000D4060C00C8060C00BC060C00B0060C0063
:102D2000A4060B0099060C008D060B0082060B0012
:102D300077060B006C060B0061060A0057060B00B5
:102D40004C060A0042060A0038060A002E060A004F
:102D500024060A001A060A001006090007060A00DF
:102D6000FD050900F4050900EB050900E20509006D
:102D7000D9050900D0050900C7050900BE050900ED
:102D8000B5050800AD050800A50509009C0508006B
:102D9000940508008C050800840508007C050800DF
:102DA000740508006C050700650508005D0507004F
:102DB000560508004E0507004705070040050800B6
:102DC00038050700310507002A050700230507001D
:102DD0001C050600160507000F050700080506007C
:102DE00002050700FB040600F5040700EE040600D8
:102DF000E8040600E2040700DB040600D504060030
:102E0000CF040600C9040600C3040600BD04060082
:102E1000B7040600B1040500AC040600A6040600D1
:102E2000A00405009B04060095040500900406001C
:102E30008A04050085040500800406007A04050064
:102E400075040500700405006B04050066040500A8
:102E5000610405005C0405005704050052040500E8
:102E60004D04050048040500430405003E04040029
:102E70003A04050035040500300404002C04050064
:102E800027040400230405001E0404001A0404009F
:102E900016040500110404000D04040009040500D3
:102EA0000404040000040400FC030400F80304000C
:102EB000F4030400F0030400EC030400E80304003E
:102EC000E4030400E0030400DC030400D80304006E
:102ED000D4030400D0030400CC030400C80303009F
:102EE000C503030024F404D9201BC40C5C0E980411
:102EF000C4095F0265077101F405F900FB04B30022
:102F000048048700C10369005803550003034500C6
:102F1000BE023A008402310053022A002902250031
:102F200004022000E4011C00C8011900AF011700D1
:102F30009801140084011300710110006101100058
:102F400051010E0043010D0036010B002B010B0057
:102F500020010B00150109000C0109000301080004
:102F6000FB000800F3000800EB000700E400060087
:102F7000DE000600D8000600D2000600CC000500E6
:102F8000C7000500C2000500BD000400B900040030
:102F9000B5000400B1000400AD000400A900040065
:102FA000A5000300A20003009F0004009B00030093
:102FB00098000300950002009300030090000300B6
:102FC0008D0002008B0003008800020086000200D2
:102FD00084000300810002007F0002007D000200E7
:102FE0007B000200790002007700010076000200F9
:102FF0007400020072000100710002006F00020004
:103000006D0001006C0002006A000100690002000E
:103010006700010066000100650001006400020015
:103020006200010061000100600001005F00020019
:103030005D0001005C0001005B0001005A0001001E
:10304000590001005800010057000100560001001E
:10305000550001005400010053000000530001001E
:103060005200010051000100500001004F0001001A
:103070004E0000004E0001004D0001004C00010018
:103080004B0000004B0001004A0001004900010014
:103090004800000048000100470001004600000011
:1030A0004600010045000000450001004400010009
:1030B0004300000043000100420000004200010004
:1030C0004100000041000100400001003F000000FD
:1030D0003F0001003E0000003E0001003D000000F6
:1030E0003D0001003C0000003C0000003C000100ED
:1030F0003B0000003B0001003A0000003A000100E4
:1031000039000000390001003800000038000000DC
:1031100038000100370000003700010036000000D1
:1031200036000000360001003500000035000000C8
:1031300035000100340000003400000034000100BC
:1031400033000000330000003300010032000000B3
:1031500032000000320001003100000031000000A8
:10316000310001003000000030000000300001009C
:103170002F0000002F0000002F0000002F00010092
:103180002E0000002E0000002E0001002D00000087
:103190002D0000002D0000002D0001002C0000007B
:1031A0002C0000002C0000002C0001002B0000006F
:1031B0002B0000002B0000002B0001002A00000063
:1031C0002A0000002A0000002A0001002900000057
:1031D000290000002900000029000000290001004A
:1031E000280000002800000028000000280000003F
:1031F0002800010027000000270000002700000031
:103200002700000027000100260000002600000023
:103210002600000026000000260001002500000016
:10322000250000002500000025000000250000000A
:1032300025000100240000002400000024000000FC
:1032400024000000240001002300000023000000EF
:1032500023000000230000002300000023000000E2
:1032600023000100220000002200000022000000D4
:1032700022000000220000002200010021000000C6
:1032800021000000210000002100000021000000BA
:1032900021000000210001002000000020000000AB
:1032A000200000002000000020000000200000009E
:1032B00020000000200001001F0000001F0000008F
:1032C0001F0000001F0000001F0000001F00000082
:1032D0001F0001001E0000001E0000001E00000074
:1032E0001E0000003930000033250000871900005F
:1032F000B00F0000DB080000BD04000074020000F5
:103300003F0100005374616E64617264204465760D
:10331000696174696F6E3A20004465766961746909
:103320006F6E0025533A2025730046696E697368F5
:103330006564210A003A207A3A2000206F66200056
:10334000476F696E6720746F3A2058004D6F766939
:103350006E6720696E776172643A20580043570A9D
:1033600000206469723A0020616E676C653A005310
:1033700074617274207261646975733A004D3438F7
:1033800020506F696E740025533A2025642F256400
:1033900000506F736974696F6E696E672074686539
:1033A0002070726F62652E2E2E0A003F4C65677387
:1033B000206F66206D6F76656D656E7420696D7027
:1033C0006C61757369626C652028302D3135292E4A
:1033D0000A003F2028582C5929206F7574206F66E9
:1033E00020626F756E64732E0A0050726F626520E2
:1033F0006F7574206F6620626F756E6473003F5343
:10340000616D706C652073697A65206E6F742070D1
:103410006C61757369626C652028342D3530292EF6
:103420000A004D3438205A2D50726F626520526563
:10343000706561746162696C697479205465737434
:103440000A003F2856296572626F7365206C6576A5
:10345000656C20696D706C61757369626C6520289C
:10346000302D34292E0A002052616E67653A200003
:10347000205369676D613A20004D65616E3A200006
:10348000204D393220580020204D61783A2000200C
:10349000204D696E3A2000536F667420656E647328
:1034A000746F70733A200025290A00252000203B04
:1034B00020280020204D3731302053003B20436F1F
:1034C0006E74726F6C6C65722046616E0A002049E2
:1034D0006E76616C696420657874727564657220BB
:1034E000003F454550524F4D2073746F72616765C0
:1034F000206E6F7420617661696C61626C652E0A62
:10350000004732362048656174696E67204E6F7AD5
:103510007A6C65004732362048656174696E6720B1
:103520004265640057616974696E6720666F722036
:103530006865617475702E0A004669786564204C70
:10354000656E677468205072696D6500446F6E65C2
:10355000205072696D696E67004D616E75616C20F7
:103560007072696D696E672E2E2E004732362043C9
:10357000616E63656C6564004C656176696E672099
:10358000473236003F537065636966696564205849
:103590002C5920636F6F7264696E617465206F755A
:1035A00074206F6620626F756E64732E0A003F2868
:1035B000522965706561742076616C7565206E6F47
:1035C0007420706C61757369626C653B206D7573F6
:1035D00074206265206174206C6561737420312EE3
:1035E0000A003F537065636966696564206E6F7A8F
:1035F0007A6C652074656D70657261747572652092
:103600006E6F7420706C61757369626C652E0A0050
:103610003F5370656369666965642066696C616DB6
:10362000656E742073697A65206E6F7420706C61AA
:10363000757369626C652E0A003F53706563696635
:10364000696564207072696D65206C656E67746869
:10365000206E6F7420706C61757369626C652E0AE0
:10366000003F537065636966696564206E6F7A7A9E
:103670006C652073697A65206E6F7420706C61755B
:103680007369626C652E0A003F52657472616374DF
:10369000696F6E204D756C7469706C696572206D10
:1036A000757374206265207370656369666965640B
:1036B0002E0A003F53706563696669656420526530
:1036C0007472616374696F6E204D756C7469706C8F
:1036D000696572206E6F7420706C61757369626CBD
:1036E000652E0A003F537065636966696564206CE6
:1036F0006179657220686569676874206E6F7420EF
:10370000706C61757369626C652E0A0043292E0A1C
:10371000003F537065636966696564206265642073
:1037200074656D7065726174757265206E6F74205A
:10373000706C61757369626C65202834302D0047A8
:103740003236207374617274696E672E2E2E0A00F1
:10375000426564204C6576656C696E672000466141
:10376000696C656420746F20656E61626C652042CF
:103770006564204C6576656C696E670A00496E76F3
:10378000616C6964206D6573682E0A0076616C69EE
:10379000640A53746F7261676520736C6F743A20AA
:1037A000004D65736820697320003F496E76616C37
:1037B00069642073746F7261676520736C6F742E17
:1037C0000A0020205261646975733A002E486569C9
:1037D0006768743A001000C90210012C01400122F0
:1037E0000170011801B0010E01F00104015002FA4C
:1037F00000B002F0003003E600D003DC009004D2F9
:10380000007005C800A006BE000008B400B009AAF8
:1038100000D00BA000600E960060118C0000158295
:103820000020197800C01D6E00A0226400B0275A45
:1038300000902C500000314600E0343C001038323B
:1038400000903A2800603C1E00A03D1400803E0A13
:1038500000203F000020583A0068747470733A2FBB
:103860002F6D61726C696E66772E6F726700203201
:103870002E302E372E32002020506C616E6E657215
:1038800042756666657242797465733A2000204617
:10389000726565204D656D6F72793A2000436F6DDA
:1038A00070696C65643A2044656320323820323098
:1038B00032300A00204C6173742055706461746565
:1038C000643A20323032302D31302D3135207C2099
:1038D000417574686F723A2028466F785F65786525
:1038E000290A00322E302E372E320A004D61726CBA
:1038F000696E0020536F667477617265205265733C
:1039000065740A00205761746368646F67205265AC
:103910007365740A002042726F776E206F75742091
:1039200052657365740A002045787465726E616C27
:103930002052657365740A00506F77657255700A7E
:10394000006175746F25632E6700473237004D3173
:10395000303031006572726F722077726974696EEF
:103960006720746F2066696C650A00446F6E65207D
:10397000736176696E672066696C652E0A004D3248
:1039800039002553202563202563202563202563E6
:1039900000656E6473746F7073206869743A2000F8
:1039A000022053697A653A200043616E6E6F74207D
:1039B0006F70656E207375626469722000534420D5
:1039C000496E6974204661696C00534420636172DA
:1039D00064206F6B0A006F70656E526F6F742066A3
:1039E00061696C65640A00766F6C756D652E696E31
:1039F0006974206661696C65640A004E6F205344E7
:103A000020636172640A004D3233202573006F70A9
:103A1000656E206661696C65642C2046696C653A48
:103A2000200046696C652073656C65637465640A83
:103A30000046696C65206F70656E65643A200045CC
:103A40004E4420535542524F5554494E450A002288
:103A500020706F73002220706172656E743A2200CC
:103A6000535542524F5554494E452043414C4C20EA
:103A70007461726765743A220053756263616C6C9D
:103A8000204F766572666C6F770045786365656474
:103A90006564206D617820535542524F5554494E0C
:103AA000452064657074683A310A00577269746918
:103AB0006E6720746F2066696C653A2000667265D7
:103AC000736800646F696E67004E6F7720004D6504
:103AD000616E204D657368204865696768743A2097
:103AE0000023206F662073616D706C65733A20004F
:103AF0000A4D657368206F6E6C792070617274690D
:103B0000616C6C7920706F70756C617465642E0ADD
:103B10000A0050726F62696E6720506F696E7400A0
:103B20000A50726F62696E67206D65736820706FEE
:103B3000696E74200020616E642074616B65206181
:103B4000206D6561737572656D656E742E0A006D0A
:103B50006D20746869636B2E0A00427573696E6527
:103B600073732043617264206973200052656D6F26
:103B700076652026204D6561737572652042656407
:103B80000052656D6F7665207368696D00506C61D9
:103B90006365207368696D20756E646572206E6F51
:103BA0007A7A6C65004D65736820506F696E742079
:103BB0004D656173757265642061743A20000A4D29
:103BC000657368206F6E6C79207061727469616CC6
:103BD0006C7920706F70756C617465642E0A00508A
:103BE0006C616365205368696D2026204D656173A3
:103BF000757265004D6F76696E6720746F206E6513
:103C00007874004D6573682045646974696E672037
:103C100053746F7070656400446F6E65204564690D
:103C200074696E67204D6573680A00446F6E652085
:103C300045646974696E67204D6573680046696EF6
:103C4000652054756E696E67204D6573680028584D
:103C50002C5929206F757473696465207072696EC0
:103C60007461626C65207261646975732E0A004F1D
:103C70006666736574206F7574206F6620626F7559
:103C80006E64732E20283020746F2031306D6D29C2
:103C90000A0A00496E76616C6964206D6170207457
:103CA0007970652E0A0A003F43616E2774206163B4
:103CB00074697661746520616E6420646561637403
:103CC0006976617465206174207468652073616D24
:103CD000652074696D652E0A0A00426F7468205869
:103CE00020262059206C6F636174696F6E73206D9C
:103CF00075737420626520737065636966696564B5
:103D00002E0A0A003F496E76616C69642067726909
:103D1000642073697A6520284A2920737065636975
:103D2000666965642028322D39292E0A0A003F2849
:103D30005029686173652076616C756520696E76BF
:103D4000616C69642028302D36292E0A0A003F282C
:103D500056296572626F7365206C6576656C2069A3
:103D60006D706C61757369626C652028302D342923
:103D70002E0A0A003F285229657065746974696FBC
:103D80006E20636F756E7420696E76616C69642055
:103D900028312B292E0A0A00446F696E67204732AA
:103DA000390000000000000000000000A043486F40
:103DB0006D696E67204661696C6564006F70656E41
:103DC00000545249474745524544007A5F6D617837
:103DD000007A5F6D696E00795F6D617800785F6D64
:103DE0006178005265706F7274696E6720656E64E9
:103DF00073746F70207374617475730A00646F6EEE
:103E0000650A00496E73756666696369656E74203C
:103E1000646174610A004578747261706F6C6174DA
:103E2000696E67206D6573682E2E2E00486F74656D
:103E30006E6420746F6F20636F6C640A005072654B
:103E4000737320627574746F6E20746F2072657363
:103E5000756D650A00507265737320627574746FB6
:103E60006E20746F2068656174206E6F7A7A6C655D
:103E70000A000000A0C2000020C2000000000000F4
:103E800020420000A04243616E63656C004F66668D
:103E9000004F6E004175746F20486F6D650053745C
:103EA000617274205072696E740043616E6E6F743B
:103EB00020656E746572207375626469723A2000C1
:103EC000052E2E00486F74656E6420746F6F20633A
:103ED0006F6C640050726F6365656400467265655F
:103EE00020585900536F667420456E6473746F7068
:103EF000730044697361626C65205374657070650A
:103F00007273004D3834004D34382050726F626542
:103F1000205465737400473238204F0A4D343820DE
:103F200050313000496E76616C6964206578747236
:103F3000756465720A0020573A007C3C3E5E2B3D5A
:103F40003F2F5B5D3B2C2A225C000009121B242DB5
:103F5000363F48415A536C657E7719100B023D3449
:103F60002F265158434A757C676E323B2029161F15
:103F7000040D7A7368615E574C452B2239300F0669
:103F80001D14636A7178474E555C646D767F4049B5
:103F9000525B2C253E3708011A137D746F66595009
:103FA0004B42353C272E1118030A565F444D727B55
:103FB00060691E170C053A3328214F465D546B6229
:103FC0007970070E151C232A31384148535A656C05
:103FD000777E09001B122D243F3658514A437C75C9
:103FE0006E671019020B343D262F737A6168575E95
:103FF000454C3B3229201F160D046A6378714E47E9
:104000005C55222B3039060F141D252C373E010834
:10401000131A6D647F7649405B523C352E27181188
:104020000A03747D666F5059424B171E050C333AD4
:1040300021285F564D447B7269600E071C152A23A8
:104040003831464F545D626B707920433A0020420C
:104050003A0020436F756E7420413A00453100628A
:104060006564002C2073797374656D2073746F70B0
:1040700070656421204865617465725F49443A2027
:104080000048656174696E67204661696C6564000B
:1040900048656174696E67206661696C65640020BB
:1040A0002D20496E76616C69642065787472756440
:1040B0006572206E756D62657220210A004572720C
:1040C0003A204D415854454D50004D415854454DAE
:1040D0005020747269676765726564004572723A50
:1040E000204D494E54454D50004D494E54454D507C
:1040F0002074726967676572656400202F00204232
:10410000403A0020403A00005072696E74205061BD
:1041100075736564003F00496E697469616C697A02
:104120006520454550524F4D00416E796375626977
:1041300063204B6F7373656C2052656164792E0048
:104140005072696E74696E672E2E2E005072696E01
:10415000742041626F72746564004D323520500ADC
:104160004D32340050617573696E672E2E2E0045F6
:104170004550524F4D2056657273696F6E204572DF
:10418000726F7200454550524F4D20496E646578FC
:10419000204572726F7200454550524F4D20435278
:1041A00043204572726F720049676E6F72650041FD
:1041B000425300504C41004D6F76652025736D6D64
:1041C000004D6F766520302E316D6D004D6F766538
:1041D00020316D6D004D6F76652031306D6D004D75
:1041E0006F766520417869730045787472756465EF
:1041F00072004D6F7665205A004D6F76652059002C
:104200004D6F76652058004368616E67652046698A
:104210006C616D656E7400556E6C6F6164204669EB
:104220006C616D656E74004C6F61642046696C61F1
:104230006D656E74005072656865617420437573B6
:10424000746F6D005072656865617420240042616E
:10425000636B0000000A0B02090C0D0E0807030433
:10426000010000000000000000000000000000004D
:10427000000000000000000000000000000000122C
:10428000111000000000000000000000000000000D
:10429000000000000000000000B341AF41205200C8
:1042A0004D65736820736176656420696E20736C58
:1042B0006F7420003F556E61626C6520746F2073CF
:1042C000617665206D65736820646174612E0A00F3
:1042D00020736C6F743D00206D65736865735F6556
:1042E0006E643D004532454E443D00206D65736867
:1042F00020736C6F747320617661696C61626C65A8
:104300002E0A003F496E76616C696420736C6F748D
:104310002E0A004D657368206C6F616465642066C9
:10432000726F6D20736C6F7420003F556E61626C0C
:104330006520746F206C6F6164206D657368206404
:104340006174612E0A0048617264636F6465642061
:1043500044656661756C742053657474696E677327
:10436000204C6F616465640A00556E696669656416
:1043700020426564204C6576656C696E67003B2061
:104380000020204D363033200020550046696C61F6
:104390006D656E74206C6F61642F756E6C6F6164F7
:1043A000206C656E677468733A0020204D38353193
:1043B0002058005A2D50726F6265204F66667365F3
:1043C000740020204D33303420500020204D3330F5
:1043D000312050005049442073657474696E6773CE
:1043E0003A0020460020204D3134352053004D61E5
:1043F00074657269616C20686561747570207061A4
:1044000072616D65746572733A0020480020204D1A
:10441000363635204C0044656C74612073657474C5
:10442000696E67733A204C3C646961676F6E616CBA
:1044300020726F643E20523C7261646975733E2045
:10444000483C6865696768743E20533C7365676DD6
:10445000656E747320706572207365633E205859D1
:104460005A3C746F77657220616E676C6520747258
:10447000696D3E204142433C726F64207472696DE5
:104480003E0020204D363636205800456E64737449
:104490006F702061646A7573746D656E743A002084
:1044A0006D65736865732E0A0A00454550524F4D7D
:1044B0002063616E20686F6C6420004163746976CC
:1044C00065204D65736820536C6F743A200020207E
:1044D0004D34323020530020204D32303520420000
:1044E000416476616E6365643A20423C6D696E5F3B
:1044F0007365676D656E745F74696D655F75733E36
:1045000020533C6D696E5F66656564726174653EDB
:1045100020543C6D696E5F74726176656C5F666590
:104520006564726174653E20583C6D61785F785FA8
:104530006A65726B3E20593C6D61785F795F6A6590
:10454000726B3E205A3C6D61785F7A5F6A65726B70
:104550003E20453C6D61785F655F6A65726B3E0029
:1045600020204D323034205000416363656C657209
:104570006174696F6E2028756E6974732F733229A8
:104580003A20503C7072696E745F616363656C3E83
:1045900020523C726574726163745F616363656C21
:1045A0003E20543C74726176656C5F616363656C38
:1045B0003E0020204D3230312058004D6178696D29
:1045C000756D20416363656C65726174696F6E20FF
:1045D00028756E6974732F7332293A0020204D328A
:1045E00030332058004D6178696D756D20666565C2
:1045F0006472617465732028756E6974732F7329F2
:104600003A0053746570732070657220756E69741A
:104610003A0020204D32303020530020446973612D
:10462000626C65640A0046696C616D656E74207326
:10463000657474696E67733A0020204D31343920F7
:1046400043203B20556E69747320696E2043656C6E
:10465000736975730A0020286D6D29002020473288
:1046600031202020203B20556E69747320696E2014
:104670006D6D000000C8420000C8420000C8420042
:1046800000C8420000A0420000A0420000A042007A
:1046900000C042B80B0000B80B0000B80B0000B817
:1046A0000B0000544845524D414C2052554E415745
:1046B000415900546865726D616C2052756E617766
:1046C00061790000002200250028002B002E003117
:1046D00000340002010000050108010B0100002167
:1046E00000240027002A002D0030003300010100C3
:1046F00000040107010A010505050507050808086A
:1047000008020202020A0A08080404040401010162
:10471000010101010103030303030303030407076A
:10472000070C0C0C0C0C0C0C0C0202020206060608
:1047300006060606060B0B0B0B0B0B0B0B010210F0
:1047400020200808102040102040800201020108AB
:10475000040201010204081020408080402010085B
:1047600004020180040201804020100804020108B4
:104770000402010102040810204080010204081014
:1047800020408000002110422063308440A550C6A4
:1047900060E770088129914AA16BB18CC1ADD1CE7F
:1047A000E1EFF13112100273325222B5529442F706
:1047B00072D662399318837BB35AA3BDD39CC3FFCF
:1047C000F3DEE36224433420040114E664C774A4D6
:1047D0004485546AA54BB528850995EEE5CFF5AC1F
:1047E000C58DD55336722611163006D776F66695E6
:1047F00056B4465BB77AA719973887DFF7FEE79D6F
:10480000D7BCC7C448E5588668A778400861180235
:10481000282338CCC9EDD98EE9AFF9488969990ABE
:10482000A92BB9F55AD44AB77A966A711A500A3345
:104830003A122AFDDBDCCBBFFB9EEB799B588B3B0E
:10484000BB1AABA66C877CE44CC55C222C033C6095
:104850000C411CAEED8FFDECCDCDDD2AAD0BBD685E
:104860008D499D977EB66ED55EF44E133E322E5125
:104870001E700E9FFFBEEFDDDFFCCF1BBF3AAF59AE
:104880009F788F8891A981CAB1EBA10CD12DC14E1F
:10489000F16FE18010A100C230E3200450254046B2
:1048A000706760B9839893FBA3DAB33DC31CD37FD1
:1048B000E35EF3B1029012F322D232354214527702
:1048C000625672EAB5CBA5A89589856EF54FE52CA1
:1048D000D50DC5E234C324A0148104667447642452
:1048E000540544DBA7FAB79987B8975FE77EF71DB1
:1048F000C73CD7D326F2369106B0165766767615A2
:104900004634564CD96DC90EF92FE9C899E9898A00
:10491000B9ABA94458654806782768C018E10882F1
:1049200038A3287DCB5CDB3FEB1EFBF98BD89BBB10
:10493000AB9ABB754A545A376A167AF10AD01AB341
:104940002A923A2EFD0FED6CDD4DCDAABD8BADE860
:104950009DC98D267C076C645C454CA23C832CE091
:104960001CC10C1FEF3EFF5DCF7CDF9BAFBABFD9F0
:104970008FF89F176E367E554E745E932EB23ED1E1
:104980000EF01E04000005010003000501000504EF
:104990000000000500030092498D4988498349259C
:1049A000532025692F2569005D0A00626564207027
:1049B0006C616E65206E6F726D616C203D205B00D6
:1049C000436F756C64206E6F7420636F6D706C65DF
:1049D0007465204C5346210054696C74696E6720DD
:1049E0006D65736820706F696E7420003F45727248
:1049F0006F722070726F62696E6720706F696E747B
:104A00002E2041626F7274696E67206F70657261EB
:104A100074696F6E2E0A00255320332F33005469BA
:104A20006C74696E67206D6573682028332F332995
:104A30000A00255320322F330054696C74696E6765
:104A4000206D6573682028322F33290A00436F7266
:104A50007265637465645F5A3D0054696C74696E75
:104A60006720506F696E7400255320312F33005436
:104A7000696C74696E67206D6573682028312F3307
:104A8000290A0000D201D40111241FBECFEFD1E2C8
:104A9000DEBFCDBF00E00CBF13E0A0E0B2E0E4E277
:104AA000FCE703E00BBF02C007900D92AA33B107E9
:104AB000D9F725E1AAE3B3E001C01D92A738B207F8
:104AC000E1F715E2C3E4D5E200E006C02197010951
:104AD000802FFE010F94C3B8C234D10780E00807CD
:104AE000A9F70F945EA10D9400BE0C9400002F92C4
:104AF0003F924F925F926F927F928F929F92AF926E
:104B0000BF92CF92DF92EF92FF920F931F93CF93BA
:104B1000DF93CDB7DEB7E1970FB6F894DEBF0FBED7
:104B2000CDBF89AB2091560528AB21E020935605D7
:104B30008091DF048D3409F414C3843511F40C948E
:104B40003137873411F00C9443378091DD04909114
:104B5000DE048B31910509F431C1BCF48430910538
:104B60003CF4823091050CF04BC097FF3DC0F5C27C
:104B70008531910511F40C9445378A31910509F47A
:104B800019C1049709F0E9C2D6C08132910509F430
:104B9000C2C154F48D31910509F43AC10CF428C115
:104BA0004E9709F439C1D9C28A35910509F4B7C1C4
:104BB00024F48A9709F41FC2D0C28B35910509F4F9
:104BC000B2C18C35910509F0C8C2A9E92A2EA2E02C
:104BD0003A2EBAE5EB2EB5E0FB2E13E5C12E12E01E
:104BE000D12E00E010E0D9C18091190E813011F072
:104BF0000C9445370F9412100E94F7950C9445378A
:104C00002091190E213011F00C94453711E00297D4
:104C100009F010E00F94121019821A821B821C8274
:104C20001D821E821F82188682E50E94573D8823BE
:104C300009F44BC00E94D03C6B017C0120E030E0C5
:104C4000A9010F94C8B1882309F455C0809153027B
:104C500090915402A0915502B09156028CA39DA34D
:104C6000AEA3BFA38091570290915802A091590220
:104C7000B0915A0288A799A7AAA7BBA7809044051C
:104C800090904505A0904605B09047054090480596
:104C90005090490560904A0570904B05A50194011C
:104CA0006CA17DA18EA19FA10F94C8B181110C941C
:104CB0004E37A301920168A579A58AA59BA50F94FB
:104CC000C8B18823C1F00C944E3789E40E94573D47
:104CD000882331F00E94D03C69837A838B839C8344
:104CE0008AE40E94573D882331F00E94D03C6D83B6
:104CF0007E838F83988720E030E0A90169817A81E3
:104D00008B819C810F94C8B181110C94023820E0F2
:104D100030E0A9016D817E818F8198850F94C8B1A3
:104D200081110C9402380E942C8487E397E00E9442
:104D30000A840C94453780E50E94573D882329F06A
:104D40000F9402106B017C0103C0C12CD12C7601A1
:104D500083E50E94573D882361F00E94D03C20E00B
:104D600030E04AE754E40F942EB20F943FBA6B013F
:104D70007C010E94848E80917E0F811105C060E0CD
:104D80008DE497E00F9469830F942F8DC60ED71E84
:104D9000E81EF91E0F942F8DDC01CB018C199D09A3
:104DA000AE09BF09B7FD02C00C94453780E00E94F0
:104DB0007386F0CF0F94FD190C9445370E9418D9D3
:104DC00081110C9445378CE0EDE8F2E0DE0111969C
:104DD00001900D928A95E1F760E070E080E50F9414
:104DE0007C0EBE016F5F7F4F0F94964E0C9445373B
:104DF0008091A9048770873011F00C94153860E019
:104E00008FE40F94385481110C9445370C94153865
:104E10000E945D450C9445372091A4103091A51057
:104E20004091A6105091A7106091530270915402C6
:104E300080915502909156020F94CCB8AB01BC0101
:104E400088E50E9472A869837A838B839C83209172
:104E5000A8103091A9104091AA105091AB10609108
:104E60005702709158028091590290915A020F9402
:104E7000CCB8AB01BC0189E50E9472A86D837E832A
:104E80008F839887BE016B5F7F4FCE0101960E9492
:104E9000D33D882311F40C94453780E00E942245CD
:104EA0000E94069884E690E090932E0280932D0253
:104EB00061E085E40F94385401E021E041E0682F7F
:104EC000CE0101960E94C9406B017C019B01AC019F
:104ED0000F946DBC811119C049815A816B817C810D
:104EE00080E697E00E9436864D815E816F817885ED
:104EF0008BE597E00E943686B701A60186E597E02C
:104F00000E9436868AE00E94F8830E94ED970F94F3
:104F100061410C9445370E9414DF0C944537109280
:104F200043030C9445378FE0809343030C9445373B
:104F30000E94D03C2B013C01133049F0F701208145
:104F40003181428153810F94CBB82B013C01D601B2
:104F50002D913D914D915C91C301B2010F94CBB85D
:104F60004B015C012DEB37E346E855EB0F9480BB1A
:104F700087FD1BC02DEB37E346E855E3C501B401BF
:104F80000F94C8B118168CF01F5FB4E0EB0EF11C43
:104F9000E4E0CE0ED11C143021F1D1018D911D0120
:104FA0000E94573D882381F3C3CF133051F44092C0
:104FB0005F0250926002609261027092620201E0B0
:104FC000E3CFA5019401F701608171818281938112
:104FD0000F94CCB8D7016D937D938D939C931397C9
:104FE000D3CF002321F08FE592E00E942F920F94FF
:104FF00061410C9445378091190E813011F00C9469
:10500000453789E40E94573D082F882321F00E94EC
:10501000CC3CE82E01C0E12C8AE40E94573D182FB9
:10502000882321F00E94CC3CF82E01C0F12C0023F3
:1050300019F0F4E0FE1528F0112349F024E02F15B3
:1050400030F488E697E00E940A840C94453780E1AA
:10505000E3E5F2E0A4E4B5E001900D928A95E1F772
:10506000002359F08E2D0E94743E60934405709386
:1050700045058093460590934705112359F08F2DE0
:105080000E94743E609348057093490580934A05D9
:1050900090934B0560E080E50F9438548823C1F16C
:1050A0000023D1F02091A4103091A5104091A610BA
:1050B0005091A71060914405709145058091460577
:1050C000909147050F94CBB86093440570934505C4
:1050D00080934605909347051123D1F02091A810A5
:1050E0003091A9104091AA105091AB1060914805E1
:1050F0007091490580914A0590914B050F94CBB86A
:10510000609348057093490580934A0590934B0539
:1051100040E050E0BA0186E40E9472A86B017C0175
:1051200020E030E0A9010F9480BB18164CF420E079
:1051300030E040E752E4C701B6010F94C6B903C09E
:1051400060E070E0CB0169837A838B839C83CE011E
:1051500001960F946E510C9445370E942FD80C94F1
:1051600045378091DD049091DE048837910511F474
:105170000C94D1300CF06CC18D34910509F415C537
:105180000CF05DC08931910509F44BC31CF58431E5
:10519000910509F4C2C27CF48131910509F4A9C2D8
:1051A0002CF4029708F46CC20C942E37429709F441
:1051B000B0C60C942E378631910509F4E3C20CF485
:1051C000DDC28731910509F4E7C2489709F4F9C2B5
:1051D0000C942E378E31910509F490C3ACF48B31C9
:1051E000910509F430C30CF420C38C31910509F406
:1051F0007DC34D9711F00C942E37809134158E7F1E
:10520000809334150C9445378033910509F4C5C457
:105210004CF48F31910509F415C4809709F4CFC37C
:105220000C942E378B34910509F4BBC48C34910552
:1052300011F00C942E370F94FA4A0C9445378C36A3
:10524000910509F4BCC50CF047C08535910509F4FA
:1052500096C64CF58235910509F44DC6D4F48135D6
:10526000910511F00C942E370F94D6760F940F4BB6
:105270000E94958E0E94B88368EE73E080E090E013
:105280000E94188360E08DE898E00F9469830C9485
:1052900045378335910509F435C68435910509F400
:1052A00038C60C942E378936910509F4D3C454F4CA
:1052B0008C35910509F486C68836910509F479C4C0
:1052C0000C942E378A36910509F4D8C48B36910593
:1052D00009F412C50C942E378137910509F479C56C
:1052E000C4F48E36910509F412C50CF489C48F36C6
:1052F000910509F41FC58037910511F00C942E37E4
:1053000041E060E070E08AE598E00E9434840C940B
:1053100045378537910509F4FAC60CF08CC0823701
:10532000910509F4EDC68337910511F00C942E37E1
:105330008DEE99E00E940A8460E08DED99E00E9474
:10534000A7B560E088EC99E00E94A7B561E082E231
:1053500091E40E94A7B561E08DEB99E00E94A7B5AA
:1053600061E08DEA99E00E94A7B560E084EA99E0E7
:105370000E94A7B561E08AE999E00E94A7B561E0C3
:1053800080E999E00E94A7B560E089E899E00E9471
:10539000A7B561E081E899E00E94A7B561E083E7E5
:1053A00099E00E94A7B560E085E699E00E94A7B564
:1053B00060E086E599E00E94A7B560E088E499E0A6
:1053C0000E94A7B560E082E399E00E94A7B560E083
:1053D00081E299E00E94A7B560E082E199E00E9435
:1053E000A7B561E08BE099E00E94A7B560E086EF89
:1053F00098E00E94A7B560E088EE98E00E94A7B50B
:1054000061E085ED98E00E94A7B560E088EC98E047
:105410000E94A7B561E083EC98E00E94A7B560E028
:1054200086EB98E00E94A7B560E082EA98E00E94CF
:10543000A7B50C9445378637910509F478C68737A8
:10544000910511F00C942E370F94D6450C944537E6
:10545000813931E0930711F40C9408340CF07AC0D0
:105460008C3C910509F4C4C7B4F58B39910509F456
:1054700018C5E4F48D37910509F43AC56CF4893701
:10548000910511F00C942E371092500C10924F0C85
:105490000F94F8450C9445378C38910509F4BEC437
:1054A0008139910509F484C60C942E37883C910506
:1054B00009F4F2C634F48E3B910509F4D0C40C947F
:1054C0002E37893C910509F451C78B3C910509F4AD
:1054D00070C70C942E378C32B1E09B0711F40C94FA
:1054E000B932ACF4833D910509F4C3C734F48D3C63
:1054F000910509F4AEC70C942E378C3D910509F443
:10550000BBC78D3D910509F4DEC70C942E378F3251
:10551000F1E09F0711F40C9405346CF48D3231E006
:10552000930711F40C94CE328E32914011F40C9406
:10553000C1330C942E378033B1E09B0711F40C94E7
:105540004E338039914011F00C942E370E94848E96
:105550000C9445378835F2E09F0711F40C94D3344E
:105560000CF048C0843F31E0930711F40C94A6344A
:10557000F4F48A39B1E09B0709F427C45CF482395A
:10558000914011F00C942E370E94C03D0F94614160
:105590000C944537843A21E0920711F40C940D34B1
:1055A000853A914011F40C9410340C942E37873FB7
:1055B000A1E09A0711F40C94AC347CF4853FE1E04F
:1055C0009E0711F40C94A934863F914011F00C947D
:1055D0002E370F94668F0C944537883F21E0920751
:1055E00011F40C94B5348C30924011F40C94C63400
:1055F0000C942E378E3BA2E09A0711F40C940836D7
:10560000ECF48939E2E09E0711F40C944D353CF43A
:105610008B35924011F40C94D6340C942E378A3981
:1056200032E0930711F40C94E6358D3B924011F073
:105630000C942E370F94C3100C944537803AB3E086
:105640009B0709F4F1C17CF4863CF2E09F0711F45A
:105650000C94C7368335934011F00C942E370E947A
:10566000FAAE0C944537873E33E0930711F40C945F
:105670000637893E934011F40C9414370C942E375E
:1056800080E50E94573D882329F00F9402106B019A
:105690007C0103C0C12CD12C760183E50E94573DCB
:1056A000882361F00E94D03C20E030E04AE754E4D7
:1056B0000F942EB20F943FBA6B017C010E94848E2E
:1056C0008091DB049091DC04009721F061E00F945D
:1056D000FB8305C060E081E897E00F94698340E0B8
:1056E000C701B6010E94F08B80E00F9427840C94D0
:1056F00045378091E00484FF02C00C9446388091C5
:10570000E20487FF02C00C9446388091E304837062
:1057100011F00C9446380C9462388091341583FF54
:1057200025C08CEA97E00E940A848091341583FF9B
:1057300017C082E893E10F94D16C8BE1E2E8F3E1CA
:10574000DE01119601900D928A95E1F760E070E01C
:10575000CE0101960F94D42ECE0101960F94D66CF3
:105760008DE997E00E940A840C9445370E943084AA
:105770008DEB97E00E940A840C9445370F948C2897
:105780000C9445370F94CD2780913415877F806224
:10579000809334150C944537E091DB04F091DC04E0
:1057A0008081882329F0803209F410823196F8CF65
:1057B00060E08091DB049091DC040F94BB2D0C948D
:1057C000453780911D0E8823F9F080E090E0A6E136
:1057D000B3E488A399A3AAA3BBA31C8E1D8E1E8E1F
:1057E0001F8E19821A821B821C8200E010E020E0CA
:1057F000AE01405E5F4FBE01645E7F4FCE010196F9
:105800000F94DA540C9445370E949483882321F036
:105810000F94DE270F94D64A80E00F9427840C94CF
:1058200045370F94FA120C9445378091341583FD57
:1058300002C00C94453783E50E94573D81110C94BA
:1058400070380C94453783E40E94093D882319F190
:1058500081ED97E00E940A8480912C13882391F0B7
:10586000BE016F5F7F4F89E293E10F94986B8E01C9
:105870000F5F1F4FF80181918F01882339F00E943B
:10588000F883F8CF87EC97E00E940A848AE00E94B0
:10589000F8830C9445378091341582FF21C080EE47
:1058A00097E00E940A8460913015709131158091C3
:1058B0003215909133154AE00E94FB848FE20E94DA
:1058C000F88360912C1570912D1580912E15909173
:1058D0002F154AE00E94FB840E9447860C944537AE
:1058E00082EF97E00E940A840C9445378091DB0494
:1058F0009091DC040F94732D0C94453780913415EE
:1059000083FD02C00C9445370E9418D8809134154D
:1059100083FD02C00C9445374091DB045091DC04B8
:10592000BE01645E7F4F80E00F94CC998C0100979C
:1059300011F40C9445376C8D7D8D19821C8222E008
:10594000AC01CE0101960F947671811102C0F12C49
:1059500014C0CE0101960F943A998823C1F361E0F7
:10596000CE0101960F947C6B009789F325EEDC0144
:105970002C931C820F94EF29F82ECE0101960F94E0
:10598000D66CB801FF2089F08BE198E00E94198461
:105990008AE00E94F883109230151092311510920F
:1059A0003215109233150C94453783E098E00E942D
:1059B000198484E699E20E940A840C944537809108
:1059C000341582FD0E94848E8091341583FD02C0BF
:1059D0000C94453760E080E50F943854182F682FF9
:1059E0008091DB049091DC040F94BB2D83E50E9431
:1059F000573D882381F00E94BC3CAB01BC01409321
:105A0000301550933115609332157093331589E238
:105A100093E10F94152C0F94DE2711110C94453748
:105A20000F94D64A0C9445372091DB043091DC0466
:105A300090913415926090933415C9010F94732D91
:105A40000C9445370F94874A7B018C0120E831E59F
:105A500041E050E00F941EB8C9016DE671E00F946B
:105A60009BB84B015C01C801B70120E13EE040E07A
:105A700050E00F941EB8CA01B90128E130E040E0BF
:105A800050E00F941EB8762E672EC62ED72EFCE35C
:105A90002F2E312C412C512CC801B701A2019101AC
:105AA0000F941EB8F62EE72ECA01B901A20191018A
:105AB0000F941EB8CB018E010F5F1F4F811491040C
:105AC00099F0EF92FF927F936F936F927F92BF92C4
:105AD000AF929F928F9289E298E09F938F931F934A
:105AE0000F930F9460B113C0A114B104B1F0EF9201
:105AF000FF927F936F936F927F92BF92AF928DE2EE
:105B000098E09F938F931F930F930F9460B10FB6FC
:105B1000F894DEBF0FBECDBF30C0CD2879F0EF9234
:105B2000FF927F936F936F927F9281E398E09F93B0
:105B30008F931F930F930F9460B1E9CF892B69F076
:105B4000EF92FF927F936F9385E398E09F938F93FB
:105B50001F930F930F9460B1DACFEF92FF9289E316
:105B600098E09F938F931F930F930F9460B10F90C2
:105B70000F900F900F900F900F9060E0C8010F945E
:105B8000FB830E943084B8018DE398E00E94198461
:105B90008AE00E94F8830C9445370F94CE130C943E
:105BA00045370F94D64A0C9445370F940F4B0C94FD
:105BB00045378091520B83FF02C00C9445370F94F8
:105BC000530E87FF02C00C94453789E40E94573D6D
:105BD000882311F40C9481380F94145490E0181613
:105BE000190614F481E090E026E0289FF001299F37
:105BF000F00D1124E055FF4E808191810C948B387B
:105C00008091520B83FF02C00C9445370F94530EC2
:105C1000F82E87FF02C00C94453789E40E94573D57
:105C2000082F882311F40C9494380F94145490E0A6
:105C30001816190614F481E090E026E0289FF00180
:105C4000299FF00D1124E055FF4E8081918110E0D5
:105C50000C94A4380F94530E182F87FD0AC082E8C5
:105C60009CE10E940A84812F0F942C768AE00E9486
:105C7000F883B8A9B09356050C94313A60E080E5FA
:105C80000F94861881110C94453781E40E94093DD8
:105C9000882329F060918E05062F10E002C00FEFD7
:105CA00010E089E40E94573D882399F00F94145422
:105CB00090E01816190614F481E090E026E0289F81
:105CC000F001299FF00D1124E055FF4E048115814C
:105CD00008C083E50E94573D882319F00E94BC3C10
:105CE0008B01B8010F3F110519F010F06FEF70E054
:105CF00060938E050C94453760E080E50F9486181C
:105D000081110C94453710928E050C9445378EE422
:105D10000E94573D882311F40C9445370E94BC3CE7
:105D20006093E6047093E7048093E8049093E90499
:105D30000C94453783E50E94093D882331F060E0EB
:105D400083E50F9486188093520B0E94308483E57C
:105D500098E00E940A848091520B882369F1E7EC55
:105D6000EE2EEBE0FE2E00E010E020E08091520BE2
:105D700090E0A0E0B0E0002E04C0B695A7959795FE
:105D800087950A94D2F780FF0EC0DD24D394D20EFB
:105D9000222319F08CE20E94F883F70185919491F7
:105DA0000E940A842D2D0F5F1F4FE2E0EE0EF11CC2
:105DB00005301105D9F66ACD8FE498E065CD1092D3
:105DC0005505109272020C9445370E946F830C9413
:105DD000453783E50E94573D882381F00F94145482
:105DE000282F30E02D33310524F4809300020C94E9
:105DF00045378CE3809300020C9445370E94308431
:105E00004091000250E060E070E088E698E00E9477
:105E100068858AE00E94F8830C9445378091520B84
:105E200083FF02C00C94453789E40E94573D8823C4
:105E300011F40C94EE380F94145490E018161906CF
:105E400014F481E090E026E0289FF001299FF00DF6
:105E50001124E055FF4E828193810C94F938809192
:105E6000520B83FF02C00C94453789E40E94573DD2
:105E7000882311F40C9400390F94145490E01816F0
:105E8000190614F481E090E026E0289FF001299F94
:105E9000F00D1124E055FF4E8281938110E00C94A7
:105EA000113983E50E94573D882311F40C9445373E
:105EB0000F941454182F90E0CD970CF01CE310931E
:105EC0003E030F942F8D6B017C01212F30E0A8EE53
:105ED000B3E00F9472B8C60ED71EE81EF91EC0922A
:105EE0003A03D0923B03E0923C03F0923D03CDC7CE
:105EF0000F94FA12CAC7809143038F7D806180930B
:105F00004303C3C7809143038F7E80628093430322
:105F1000BCC783E50E94573D8823E9F00F942F8D7D
:105F20006093F80E7093F90E8093FA0E9093FB0E27
:105F30000E94D03C20E030E04AE754E40F942EB2B7
:105F40000F943FBA609301027093020280930302A0
:105F5000909304029AC78091E00484FF02C00C94DD
:105F60003A398091E20487FF02C00C943A3980915B
:105F7000E304837011F00C943A390C946C3983E586
:105F80000E94093D882309F480C70F942F8D6093E8
:105F9000F80E7093F90E8093FA0E9093FB0E0E9408
:105FA000D03C20E030E04AE754E40F942EB20F9446
:105FB0003FBA60933F0370934003809341039093F3
:105FC000420363C70F94530E87FD5FC79091E004AF
:105FD00094FD04C09091E20497FF0AC069E9C62EBF
:105FE00062E0D62E73E5E72E7BE0F72E10E009C0C5
:105FF0009091E304937091F7682F81E00F94C70F9D
:1060000044C7D6018D916D010E94573D882309F444
:106010006DC0133009F063C00E94D03C4B015C019D
:1060200020E030E040EA51E40F94C8B187FF4EC051
:10603000A50194016091730B7091740B8091750BA5
:106040009091760B0F94C6B92B013C019B01AC01DA
:10605000609172057091730580917405909175053A
:106060000F942EB26093720570937305809374053C
:1060700090937505A30192016091830B7091840B3D
:106080008091850B9091860B0F942EB26093830BB9
:106090007093840B8093850B9093860B609182059F
:1060A0007091830580918405909185050F94CDB101
:1060B000A30192010F942EB20F943FBA6093820510
:1060C0007093830580938405909385058092730B6C
:1060D0009092740BA092750BB092760B07C00E9441
:1060E000D03CF701648B758B868B978B1F5FF4E038
:1060F000EF0EF11C143009F084CF0E94608EC5C6EB
:106100000E942DD78AED93E10F94967EBEC68091B2
:10611000DB049091DC04009709F47ECBDC012C9128
:10612000222309F479CB60E00F94FB83AEC6009183
:10613000DB041091DC0494E0F12C40E0915021F15B
:10614000F8018081282F2B7F213421F421812133F4
:10615000D9F407C08035C1F4818180538A3048F07A
:1061600013C0813421F0853421F441E002C0FF24C2
:10617000F39498012E5F3F4F89012F5F3F4FF80145
:1061800080818032C9F3DACF41110E943084FF2030
:1061900021F088EC9AE00E940A84C8010E944D8692
:1061A00074C62093500C20934F0C0F94F8456DC685
:1061B00060E070E083E50E94643D823038F00E9428
:1061C0002C848CEC9AE00E940A845FC68C01112713
:1061D00088E40E94573D8823E1F00E94CC3C8A3A33
:1061E000910544F00E94CC3C8530914034F40E94EB
:1061F000CC3C05C08AEA90E002C084E091E026E051
:10620000209FF001219FF00D1124E055FF4E918356
:10621000808382E40E94573D8823D9F00E94CC3CC1
:10622000059744F00E94CC3C8D38910534F40E94CF
:10623000CC3C05C085E090E002C08CE890E026E010
:10624000209FF001219FF00D1124E055FF4E938314
:10625000828386E40E94573D882309F416C60E9473
:10626000CC3C97FD09C00E94CC3C8F3F910509F0C2
:1062700034F40E94CC3C05C080E090E002C08FEF77
:1062800090E026E0209FF001219FF00D1124E055C1
:10629000FF4E95838483F9C50F94530E182F87FD05
:1062A000F4C50091F61084E40E94573D882311F450
:1062B0000C946F390E94D03C6B017C0120E030E0EF
:1062C000A9010F94C8B1882309F44AC024E012023E
:1062D000F0011124EE50FF4EC082D182E282F3829F
:1062E00020E030E0A901C701B6010F9480BB181669
:1062F000D4F420E030E040E05FE3C701B6010F9442
:106300002EB29B01AC010F942EB22BED3FE049E47D
:1063100050E40F942EB260930502709306028093AE
:1063200007029093080220E030E0A9016091F2108A
:106330007091F3108091F4109091F5100F94C8B102
:1063400081110CC080E090E0A0EEBFE38093F210DA
:106350009093F310A093F410B093F51001E0BFC731
:1063600080E08093F6100E94828D8FC50F94530EAB
:1063700087FD8BC559E9E52E52E0F52E03E51BE0BC
:10638000D7018D917D010E94093D882359F00E941B
:10639000D03C0F943FBAF80160837183828393836A
:1063A0000E94198E0C5F1F4FFBE003361F0741F759
:1063B0006CC50F94530E87FD68C549E9E42E42E091
:1063C000F42E03E51BE0D7018D917D010E94093D6C
:1063D000882339F00E94D03CF80164A375A386A3FA
:1063E00097A30C5F1F4FFBE003361F0761F74DC5F6
:1063F0008091E10487FD78C78091E2048E7009F0F6
:1064000073C74091870B5091880B6091890B7091F5
:106410008A0B8EEE9AE00E94368640918B0B50914B
:106420008C0B60918D0B70918E0B8DE992E40E9424
:10643000368640918F0B5091900B6091910B70912B
:10644000920B88EE95E20E9436868AE00E94F883DD
:106450001CC58091E004827109F08CC78091E20430
:106460008C7809F087C78091E304837009F082C7B4
:106470000CC50F94D80E09C583E50E94573D8823AB
:1064800031F00E94CC3C90932E0280932D0280919B
:10649000E0049091E104A091E204B091E304892B1F
:1064A0008A2B8B2B09F0F1C460912D0270912E0282
:1064B00080E39BE00E94B28585E20E94F8838AE037
:1064C0000E94F883E2C40F94530EF82E87FDDDC4BA
:1064D00083E50E94573D0F2D0F2C000C110B8823D4
:1064E00069F10E94CC3CF801EE0FFF1FED5CFD4FFF
:1064F00091838083000F111F000F111F9801235BF0
:106500003D4F7901BC01990F880B990B0F94CFB1C6
:106510002AE037ED43E25CE30F942EB2F801E65532
:10652000FB4F20813181428153810F942EB2D701DC
:106530006D937D938D939C931397A7C40E94308491
:1065400085E40E94F88380E38F0D0E94F883000F9A
:10655000111FF801ED5CFD4F6081718184E39BE0C8
:106560000E94B28585E20E94F8838AE00E94F88347
:106570008CC464E071E083E50F947C0E8C0168EEBE
:1065800073E080E50F947C0E8938B3E19B0710F02F
:1065900088E893E1B8010F94328377C460E085E422
:1065A0000F948618811173C080E50E94093D8823ED
:1065B00051F00E94D03C609312117093131180939C
:1065C00014119093151189E40E94093D882381F0EC
:1065D0000E94D03C2CEA35EC47E25EE30F942EB2E9
:1065E00060931611709317118093181190931911DD
:1065F00084E40E94093D882381F00E94D03C2CEA6B
:1066000035EC47E25EE30F94C6B960931A117093BC
:106610001B1180931C1190931D110E943084409196
:10662000121150911311609114117091151184E49D
:106630009BE00E9436862CEA35EC47E25EE36091EF
:1066400016117091171180911811909119110F94D2
:10665000C6B9AB01BC0180E49BE00E9436862CEAFF
:1066600035EC47E25EE360911A1170911B11809145
:106670001C1190911D110F942EB2AB01BC018CE343
:106680009BE00E9436868AE00E94F883FEC30E9447
:106690002C8484E29FE30E940A84F7C380E50E9471
:1066A000093D882351F00E94D03C6093070F7093FE
:1066B000080F8093090F90930A0F89E40E94093D07
:1066C000882381F00E94D03C2CEA35EC47E25EE35F
:1066D0000F942EB260930B0F70930C0F80930D0FDD
:1066E00090930E0F84E40E94093D882381F00E945C
:1066F000D03C2CEA35EC47E25EE30F94C6B96093D8
:106700000F0F7093100F8093110F9093120F0E9430
:1067100030844091070F5091080F6091090F7091DC
:106720000A0F84E49BE00E9436862CEA35EC47E2AF
:106730005EE360910B0F70910C0F80910D0F9091A3
:106740000E0F0F94C6B9AB01BC0180E49BE00E9420
:1067500036862CEA35EC47E25EE360910F0F7091CC
:10676000100F8091110F9091120F0F942EB2AB0168
:10677000BC018CE39BE00E9436868AE00E94F8838D
:1067800084C383E50E94093D182F882371F00E947D
:10679000D03C0F9438BA709352026093510221E0BA
:1067A000672B09F020E020939F0580E50E94093DBA
:1067B000882359F02091510230915202232B11F07D
:1067C0000F94285480939F0560C311115EC30E94EB
:1067D000308481E69BE00E940A8480919F05882393
:1067E00019F080E69AE102C088E49BE00E940A84E6
:1067F000609151027091520280E59BE00E94B28547
:106800008CE49BE00E940A8440C30E9489A83DC397
:106810000E94C93D0F94614138C30F94921835C34B
:106820006FEF7FEF89E40E94643DB82E6FEF7FEF3A
:106830008AE40E94643D182F83E40E94093DE82EFB
:106840008EE40E94093DC82E8AE50E94093DF82E7B
:10685000811105C081E50E94093DD82E01C0D12CCF
:10686000EE2081F020E030E040E063E572E081E07E
:106870000F94933529833A834B835C836D837E83A6
:10688000032F02C0012F2B2D8E2D90E0B7FC05C0E9
:106890001095111F1127111F01C010E0810F911DCC
:1068A000019731F4F1100BC0D11009C0C11007C01D
:1068B0000E942C8484E79BE00E940A84E6C2253073
:1068C00010F4053038F00E942C8488E697E00E948E
:1068D0000A84DBC2E22E220FFF08002E000C110BEF
:1068E000C1101DC00E94D03CDD2099F025E02E9DF6
:1068F000F0012F9DF00D1124E00FF11FEE0FFF1F8F
:10690000EE0FFF1FE85CFF4E2081318142815381F1
:1069100003C020E030E0A9010F94CCB804C060E0CF
:1069200070E080EC9FE725E02E9DF0012F9DF00D9B
:106930001124E00FF11FEE0FFF1FEE0FFF1FE85CA9
:10694000FF4E60837183828393839FC20E94B4F65B
:106950009CC20F94329299C261E083E50F9438543F
:1069600091E089270F94409290C281E08093371084
:106970000E940BFC10923710882309F486C20E94F3
:10698000308484E99BE00E940A847FC280913415A0
:1069900082FF04C080648093341577C283FF75C280
:1069A0000E9418D872C20F94F1116FC20F94530E47
:1069B000082F87FD6AC285E50E94093D8823A1F161
:1069C000E02E002E000CFF080E94D03C4B015C0121
:1069D00020E030E0A9010F9480BB87FF04C0B7FA24
:1069E000B094B7F8B094C70153E0880F991F5A9537
:1069F000E1F7FC01E456FF4E7F0180829182A28282
:106A0000B38220E030E84BE354E4C501B4010F94B5
:106A100080BB18164CF480E090E8ABE3B4E4F701D7
:106A200080839183A283B3838CE40E94093D8823F1
:106A300009F42BC2002E000C110B0E94D03C6B01FC
:106A40007C0120E030E0A9010F9480BB87FF04C0E7
:106A5000F7FAF094F7F8F09420E030E84BE354E4D0
:106A6000C701B6010F9480BB980143E0220F331F8A
:106A70004A95E1F7F901E456FF4E18162CF0C4824E
:106A8000D582E682F78201C280E090E8ABE3B4E40D
:106A900084839583A683B783F8C188E40E94093D67
:106AA000882351F00E94D03C6093D8107093D91085
:106AB0008093DA109093DB108CE40E94093D8823C8
:106AC00051F00E94D03C6093E0107093E1108093ED
:106AD000E2109093E31082E50E94093D882351F073
:106AE0000E94D03C6093DC107093DD108093DE1028
:106AF0009093DF1083E50E94093D882351F00E94A6
:106B0000D03C6093D4107093D5108093D61090939E
:106B1000D71088E50E94093D882351F00E94D03C9F
:106B20006093C8107093C9108093CA109093CB10D3
:106B300089E50E94093D882351F00E94D03C609372
:106B4000CC107093CD108093CE109093CF108AE527
:106B50000E94093D882351F00E94D03C6093D010E0
:106B60007093D1108093D2109093D31081E40E943F
:106B7000093D882351F00E94D03C6093BC10709373
:106B8000BD108093BE109093BF1082E40E94093D17
:106B9000882351F00E94D03C6093C0107093C110C4
:106BA0008093C2109093C31083E40E94093D882310
:106BB00051F00E94D03C6093C4107093C510809334
:106BC000C6109093C7100F94D2485FC124EEE22EF6
:106BD00020E1F22E18E5812F0E94093D882389F0DB
:106BE0000E94D03C4B015C0120E030E0A9010F94F1
:106BF000C8B1181634F0D7018D929D92AD92BC9217
:106C000013971F5FB4E0EB0EF11C1B3521F73DC15C
:106C10000F94530E182F87FD38C18AE50E94573D07
:106C2000882349F040E050E0BA018AE50E9472A84A
:106C30004B015C0106C0812C912C98E4A92E92E4B2
:106C4000B92E412F64E083E00E94DD5520E030E062
:106C5000A901C501B4010F9480BB18167CF580E032
:106C600090E0A0E7B2E489839A83AB83BC83209150
:106C70005B0230915C0240915D0250915E02C50161
:106C8000B4010F94CCB86B017C0120E030E040EA05
:106C900053E40F94C8B187FD06C0C12CD12C80EA03
:106CA000E82E83E4F82ECC8EDD8EEE8EFF8EBE01B4
:106CB0006F5F7F4FCE014C960E94429A85E50E94FD
:106CC000093D882329F00E94D03C6B017C010AC059
:106CD00028E01202F0011124E456FF4EC080D1805A
:106CE000E280F38020E030E0A901C701B6010F94F3
:106CF00080BB87FF04C0F7FAF094F7F8F094F7FA36
:106D0000F094F7F8F094C982DA82EB82FC8244E0D6
:106D100061E0CE0101960F94F65520E030E0A90124
:106D2000C501B4010F9480BB18165CF580E090E0BB
:106D3000A0E7B2E489839A83AB83BC83A501940165
:106D400060915B0270915C0280915D0290915E02A5
:106D50000F94CBB86B017C0120E030E0A9010F94C7
:106D600080BB18161CF0C12CD12C7601CC8EDD8E88
:106D7000EE8EFF8EBE016F5F7F4FCE014C960E945C
:106D8000429A40E060E089E00E94DD557EC082E5E5
:106D90000E94093DD82E81110F94205883E50E944E
:106DA000573DE82E882321F00F9414548093AE0BA6
:106DB00089E40E94573DF82E882321F00F94145443
:106DC0008093AF0B81E40E94573D082F882321F068
:106DD0000F9428548093B20B84E40E94573D182FDF
:106DE000882331F00E94BC3C7093B10B6093B00BD0
:106DF000D1104BC0E11049C0F11047C0011145C08E
:106E0000111143C080E00F948F0E3FC081E080934A
:106E1000190E1092CF0F60E083E50F943854811162
:106E200034C00E945BAE31C00F94874A6D33710548
:106E30008105910520F083EC9BE00E94F1B58FEB7A
:106E40009BE00E94F1B58BEA9BE00E940A848FE9E7
:106E50009BE09093550C8093540C17C00E942FD840
:106E600014C01091DD040F942F8D6093F80E709371
:106E7000F90E8093FA0E9093FB0E112331F0812FBF
:106E80000F94677202C00E942FD839A9311102C035
:106E90000E944BAE88A980935605E3C220E030E003
:106EA000A901C701B6010F94C8B1881F8827881FA0
:106EB000181709F4A2C080E090E0A0E8BFEB8CA70F
:106EC0009DA7AEA7BFA72CA13DA14EA15FA1C50163
:106ED000B4010F94CBB820E030E040E05FE30F94C2
:106EE0002EB26CA37DA38EA39FA328A539A54AA586
:106EF0005BA5C301B2010F94CBB820E030E040E0C5
:106F00005FE30F942EB22B013C012CA13DA14EA1B9
:106F10005FA1CA01B9010F942EB24B015C01A3011C
:106F20009201C301B2010F942EB29B01AC01C501C5
:106F3000B4010F94CCB80F941EBC4B015C019B01B3
:106F4000AC01C701B6010F94CBB868A779A78AA78F
:106F50009BA7A5019401C701B6010F94CCB89B0172
:106F6000AC0168A579A58AA59BA50F942EB26B01EB
:106F70007C0120E030E0A9010F9480BB87FD07C0B1
:106F8000C701B6010F941EBC6B017C0103C0C12C6C
:106F9000D12C7601C301B2019058A50194010F9440
:106FA000C6B92CA53DA54EA55FA50F942EB2A7018D
:106FB00096010F942EB22CA13DA14EA15FA10F947A
:106FC000CCB869837A838B839C83A50194016CA1DF
:106FD0007DA18EA19FA10F94C6B92CA53DA54EA55C
:106FE0005FA50F942EB2A70196010F942EB2A301B4
:106FF00092010F94CCB80C94772680E090E0A0E842
:10700000BFE35DCF412FBE016F5F7F4F84E495E00A
:107010000E94B0B10F942F8D6093F80E7093F90E0B
:107020008093FA0E9093FB0E30CF0E94848E1092C4
:1070300014021091F11080E00E9422450F942F8DD0
:107040006093F80E7093F90E8093FA0E9093FB0EF6
:107050000E94069884E690E090932E0280932D0281
:1070600081E08093500C0F94F8450F941546809161
:107070004F0C8093500C812F0E9422450E94ED9767
:1070800083E0809388020F946141FFCE88E50E94DF
:10709000093D81115F9889E50E94093D81118A9817
:1070A0008AE50E94093D882329F0809108018170BA
:1070B0008093060185E40E94093D882309F4E5CE0A
:1070C0001298E3CE60E084E997E00F9469835F98BB
:1070D0008A98809108018170809306011298D5CE1C
:1070E0000E94BC3CAB01BC0140933015509331155C
:1070F000609332157093331589E293E10F94152C48
:10710000C4CE83E50E94573D882359F00E94D03CAD
:107110000F9438BACB010F947C7261E080E00F9439
:1071200029A80F94B2A0B1CE83E50E94573D182F35
:10713000811105C082E50E94573D882341F10E94DC
:10714000D03C0F9438BACB010F947C7261E081E09F
:107150000F9429A860910F1170911011072E000C47
:10716000880B990B0F94CFB14B015C0140900B1130
:1071700050900C1160900D1170900E11A3019201AE
:107180000F9480BB18163CF1112361F001E00F94BD
:10719000B2A0002309F479CE40E0612F8F2D0F9427
:1071A000237473CEA3019201C501B4010F9480BB77
:1071B00018168CF083E798E09F938F938AE498E009
:1071C0009F938F931F920F94DA830F900F900F90DD
:1071D0000F900F90DBCF82E898E0EECF83E50E941E
:1071E000573D882309F451CE0E94D03C0F9438BA01
:1071F000CB010F94605161E080E00F9429A845CE47
:1072000083E50E94573D182F811106C082E50E9438
:10721000573D882309F439CE0E94D03C0F9438BAE8
:10722000CB010F94605160E081E00F9429A8609138
:10723000040F7091050F072E000C880B990B0F940B
:10724000CFB12091000F3091010F4091020F50916A
:10725000030F0F9480BB181654F08FE698E060E09F
:107260000F94698360E0812F0F948C720ECE8EE7AD
:1072700098E0F5CF0E94848E88E50E94093D88231E
:1072800021F05F9A80E00E941C9589E50E94093DEB
:10729000882321F08A9A81E00E941C958AE50E9449
:1072A000093D882349F08091080180958170809381
:1072B000060182E00E941C9585E40E94093D81112F
:1072C0000E945A838091BC04882309F4DECD109279
:1072D000BC041092D00FD9CD0E94958EF3CF602FB1
:1072E00083E50F9438543DC883E50E94573D8823B9
:1072F00091F00E94D03C6093870B7093880B809331
:10730000890B90938A0B60938F0B7093900B8093F3
:10731000910B9093920B80E50E94573D882351F08A
:107320000E94D03C6093870B7093880B8093890BED
:1073300090938A0B82E50E94573D882351F00E946A
:10734000D03C60938B0B70938C0B80938D0B909340
:107350008E0B84E50E94573D882309F496CD0E9448
:10736000D03C60938F0B7093900B8093910B909314
:10737000920B8BCD82E40E94093D882351F00F943B
:1073800002106093630B7093640B8093650B909372
:10739000660B83E50E94093D882351F00E94D03C92
:1073A0006093930B7093940B8093950B9093960B33
:1073B00084E50E94093D882351F00E94D03C6093EF
:1073C000970B7093980B8093990B90939A0B88E589
:1073D0000E94093D882351F00E94D03C60936605CD
:1073E00070936705809368059093690589E50E940D
:1073F000093D882351F00E94D03C60936A05709348
:107400006B0580936C0590936D058AE50E94093D9C
:107410008823B1F00E94D03C60936E0570936F0595
:1074200080937005909371052DEC3CEC4CEC5DE382
:107430000F94C8B1181624F08EEF9AE00E940A84C7
:1074400085E40E94093D882309F41FCD0E94D03CA9
:10745000609372057093730580937405909375051E
:1074600014CDE1960FB6F894DEBF0FBECDBFDF910D
:10747000CF911F910F91FF90EF90DF90CF90BF9031
:10748000AF909F908F907F906F905F904F903F90C4
:107490002F900895CF92DF92EF92FF926B017C01C3
:1074A00020E030E0A9010F9480BB87FF04C0C70132
:1074B000B601905802C0C701B601FF90EF90DF906F
:1074C000CF9008951092CF0F089548E350E125E042
:1074D000A0E0B0E0FA01EA0FFB1F608371838283B2
:1074E00093831496A431B105A9F721504C5E5F4FE8
:1074F0002111EECF08959091440380934403892F86
:1075000008950F931F93CF938C0120E030E040EA61
:1075100052E4FC0160817181828193810F94CCB827
:1075200020E030E040EA51E40F94CCB82DEC3CEC84
:107530004CEC5CE30F942EB20F9438BA653010F423
:10754000C62F01C0CFEF20E030E040EA52E4F8015E
:1075500064817581868197810F94CCB820E030E0FA
:1075600040EA51E40F94CCB82DEC3CEC4CEC5CE3DD
:107570000F942EB20F9438BA653010F4962F01C0D4
:107580009FEF8C2FCF911F910F91089586E093E18B
:107590000C94F1B5CF92DF92EF92FF92CF93C82F68
:1075A00087E00E94FF83C12CD12C760180E20E94EB
:1075B000F883C701B6010E9486858C2F0E94FF8345
:1075C0008FEFC81AD80AE80AF80A85E0C816D1046D
:1075D000E104F10459F76AE070E080E090E0CF91B7
:1075E000FF90EF90DF90CF900C943C830F931F930C
:1075F000CF93DF938B01EA010E94FF8388E20E9410
:10760000F883043611054CF480E20E94F8830A30B6
:1076100011051CF480E20E94F883B801110F880B59
:10762000990B0E9486858CE20E94F883C436D105AE
:107630004CF480E20E94F883CA30D1051CF480E249
:107640000E94F883BE01DD0F880B990B0E9486858E
:1076500089E20E94F88365E070E080E090E0DF91CD
:10766000CF911F910F910C943C83CF92DF92EF92B8
:10767000FF920F931F93CF93DF930E94EC82882396
:1076800009F44AC00E9430848DED9BE00E940A8478
:1076900088E3C82E80E1D82EC0E0D0E0760100E07B
:1076A00010E0F70160817181828193819B01AC01BF
:1076B0000F946DBC811121C00E943084BE0184ED05
:1076C0009BE00E94B285B80181ED9BE00E94B285EB
:1076D00086E891E10E940A84F701608171818281CC
:1076E000938144E00E94BF858AE00E94F8836BE4A6
:1076F00070E080E090E00E943C830F5F1F4FF4E059
:10770000EF0EF11C0530110561F6219684E1C80EDB
:10771000D11CC530D10511F6DF91CF911F910F918A
:10772000FF90EF90DF90CF9008958F929F92AF924D
:10773000BF92CF92DF92EF92FF920F931F93CF935E
:10774000DF93EC017B018A016901FB01208131811A
:1077500042815381688179818A819B810F94CCB861
:10776000688379838A839B83F801208131814281F8
:1077700053816C817D818E819F810F94CCB86C8305
:107780007D838E839F83F6012081318142815381E5
:10779000688579858A859B850F94CCB868877987B9
:1077A0008A879B87F70160817181828193819B0128
:1077B000AC010F942EB29B01AC016C857D858E854A
:1077C0009F850F94CCB86C877D878E879F87F80143
:1077D00060817181828193819B01AC010F942EB2F3
:1077E0009B01AC01688979898A899B890F94CCB8FF
:1077F000688B798B8A8B9B8BF6016081718182818A
:1078000093819B01AC010F942EB29B01AC016C895A
:107810007D898E899F890F94CCB86C8B7D8B8E8BE4
:107820009F8BF8012081318142815381F701608172
:107830007181828193810F942EB29B01AC01688D7E
:10784000798D8A8D9B8D0F94CCB8688F798F8A8FB4
:107850009B8FF6012081318142815381F701608144
:107860007181828193810F942EB29B01AC016C8D4A
:107870007D8D8E8D9F8D0F94CCB86C8F7D8F8E8F6C
:107880009F8FF6012081318142815381F80160810F
:107890007181828193810F942EB29B01AC0168A10A
:1078A00079A18AA19BA10F94CCB868A379A38AA3DC
:1078B0009BA38CA09DA0AEA0BFA0F701C080D180EB
:1078C000E280F38020E030E0A901C701B6010F9407
:1078D00080BB87FF04C0F7FAF094F7F8F094A70193
:1078E0009601B401C5010F94C8B187FD02C06401BF
:1078F0007501CCA2DDA2EEA2FFA288A499A4AAA43D
:10790000BBA4F801C080D180E280F38020E030E0A9
:10791000A901C701B6010F9480BB87FF04C0F7FA25
:10792000F094F7F8F0949401A501C701B6010F9403
:1079300080BB181614F064017501C8A6D9A6EAA682
:10794000FBA620E030E040E85FE368AD79AD8AADAA
:107950009BAD0F94CCB868AF79AF8AAF9BAFDF9186
:10796000CF911F910F91FF90EF90DF90CF90BF903C
:10797000AF909F908F90089580910F0C9091100C74
:10798000009731F04AE050E060E070E00D9471AE95
:1079900060E070E0CB0108950E94BC3CCB010895EB
:1079A0000F931F93CF9380910F0C9091100C009721
:1079B00011F1FC018F01C1912C2F2F7DA9F0C5344D
:1079C00011F0C536B9F7F801108260E070E08091DF
:1079D0000F0C9091100C0F9415ADF801C083562F29
:1079E000472F382F292F0BC060E070E0CF911F91F7
:1079F0000F910D9415AD50E040E030E020E0652F90
:107A0000742F832F922FCF911F910F9108950C9473
:107A1000D03C81548A3108F047C0E82FF0E0409113
:107A2000E0045091E1046091E2047091E30404C029
:107A300076956795579547958A95D2F7842F8170EB
:107A400040FF34C0EF53FB4F9081992341F1E09107
:107A50005805F0915905E90FF11D908120ED290F8E
:107A60002A3098F09E3211F491810CC09D3211F0B1
:107A70009B3271F4918120ED290F2A3030F09E3233
:107A800039F4928190539A3018F42E2F9F2F02C010
:107A900020E090E020930F0C9093100C089510922A
:107AA000100C10920F0C089580E0089508950E9424
:107AB000093D882341F081E020910F0C3091100C9A
:107AC000232B09F480E00895CF93DF93EB010E940C
:107AD000573D882321F0DF91CF910C94CC3CCE010F
:107AE000DF91CF9108958F929F92AF92BF92CF92E4
:107AF000DF92EF92FF926091A4107091A510809197
:107B0000A6109091A710C090A810D090A910E09056
:107B1000AA10F090AB109B01AC010F942EB24B0158
:107B20005C01A7019601C701B6010F942EB29B011B
:107B3000AC01C501B4010F94CCB80F941EBC6B010D
:107B40007C0120E030E040EF51E40F94C8B187FFA2
:107B500006C0C12CD12C80EFE82E81E4F82EA701BD
:107B6000960160E070E084EB92E40F94CBB8FF9054
:107B7000EF90DF90CF90BF90AF909F908F9008953F
:107B80008091520C882319F080E00F94D90280E094
:107B900008958091520C811103C081E00F94D902A5
:107BA00080E0089508954F925F926F927F928F9236
:107BB0009F92AF92BF92CF92DF92EF92FF92CF93BC
:107BC000DF9300D01F92CDB7DEB79A838983FB0184
:107BD00040805180628073802091A8103091A9105C
:107BE0004091AA105091AB10C301B2010F94CBB8D1
:107BF0004B015C01E981FA81C080D180E280F38091
:107C00002091A4103091A5104091A6105091A7107A
:107C1000C701B6010F94CBB89B01AC010F942EB2F3
:107C200069837A838B839C83A5019401C501B40188
:107C30000F942EB29B01AC0169817A818B819C816A
:107C40000F94CCB825E230E24DEF55E40F94C8B163
:107C50001816F4F0A7019601C701B6010F942EB2D1
:107C60006B017C01A3019201C301B2010F942EB2FA
:107C70009B01AC01C701B6010F94CCB8F1E0F983C8
:107C800021E330E041E655E40F94C8B118160CF436
:107C9000198289810F900F900F900F90DF91CF91F3
:107CA000FF90EF90DF90CF90BF90AF909F908F901C
:107CB0007F906F905F904F9008958091780F82FB36
:107CC000882780F90895FC01208127FD06C0818165
:107CD0008095881F8827881F089580E008952FEFDA
:107CE000FC01208321830895E82FF0E0853078F4AB
:107CF000EE0FFF1FEE0FFF1FEE58F14C459155910F
:107D000065917491F42FE52F362F272F16C0BF01F0
:107D1000FF0F880B990B0F94CFB120E030E040E2C9
:107D200052E40F942EB220E030E040EA52E40F9487
:107D3000CBB8F62FE72F382F292F6F2F7E2F832FC9
:107D4000922F08950F931F93CF93DF93CDB7DEB794
:107D500028970FB6F894DEBF0FBECDBF8C01FC0193
:107D600080810E94743E69837A838B839C83F801AF
:107D700081810E94743EE62F462F572FBC014D8310
:107D80005E836F83788729813A814B815C816E2F76
:107D90007E818F81988528960FB6F894DEBF0FBE3E
:107DA000CDBFDF91CF911F910F9108952F923F92F8
:107DB0004F925F926F927F928F929F92AF92BF92FB
:107DC000CF92DF92EF92FF920F931F93CF93DF93A7
:107DD000CDB7DEB762970FB6F894DEBF0FBECDBF4A
:107DE0009A838983788B6F8720E030E040EA52E401
:107DF000FC0160817181828193810F94CCB82DEC5C
:107E00003CEC4CEC5CE30F942EB20F9438BA698BC7
:107E100065301CF0F4E0F98B03C0298927FD198A2D
:107E200020E030E040EA52E4EF85F889608171811A
:107E3000828193810F94CCB82DEC3CEC4CEC5CE34C
:107E40000F942EB20F9438BA6A8B65301CF0F4E0B0
:107E5000FA8B03C02A8927FD1A8A3989232E330F0A
:107E60003308C10144E02416310414F083E090E0AB
:107E7000FC013196FE87ED87F989FF5FFD838F2F27
:107E80000E94743E69877A878B879C8789890E94C4
:107E9000743E6B017C0185E0829DF001839DF00DB5
:107EA00011242A89022F220F110BE00FF11FEE0F70
:107EB000FF1FEE0FFF1FE85CFF4E40805180628085
:107EC00073804D855E85849FF001859FF00D1124A0
:107ED000E00FF11FEE0FFF1FEE0FFF1FE85CFF4EDC
:107EE000A301920160817181828193810F94CBB84B
:107EF0004B015C01A7019601E981FA8160817181E2
:107F0000828193810F94CBB89B01AC01C501B40170
:107F10000F942EB24B015C01A701960169857A8509
:107F20008B859C850F94CBB89B01AC01C501B40136
:107F30000F94C6B9A30192010F94CCB869877A87D0
:107F40008B879C87C8010430110514F083E090E012
:107F50005C01FFEFAF1ABF0A8D810E94743E6D83F2
:107F60007E838F83988789890E94743E6B017C0190
:107F700025E0229DC001239D900D1124FC01EA0DF6
:107F8000FB1DEE0FFF1FEE0FFF1FE85CFF4E408052
:107F90005180628073804D855E85249FC001259F3E
:107FA000900D1124FC01EA0DFB1DEE0FFF1FEE0FDB
:107FB000FF1FE85CFF4EA301920160817181828105
:107FC00093810F94CBB84B015C01A7019601E98125
:107FD000FA8160817181828193810F94CBB89B017A
:107FE000AC01C501B4010F942EB24B015C01A70195
:107FF00096016D817E818F8198850F94CBB89B010E
:10800000AC01C501B4010F94C6B9A30192010F944C
:10801000CCB82B013C018A898F5F0E94743E698332
:108020007A838B839C838A890E94743E6B017C01D6
:108030009B01AC01EF85F889608171818281938118
:108040000F94CBB84B015C0129853A854B855C8543
:10805000C301B2010F94CBB89B01AC01C501B401BF
:108060000F942EB24B015C01A701960169817A81C0
:108070008B819C810F94CBB89B01AC01C501B401ED
:108080000F94C6B929853A854B855C850F94CCB889
:108090006B017C019B01AC010F946DBC882319F02E
:1080A000C12CD12C7601C701B60162960FB6F894A7
:1080B000DEBF0FBECDBFDF91CF911F910F91FF901B
:1080C000EF90DF90CF90BF90AF909F908F907F9078
:1080D0006F905F904F903F902F9008954F925F92D6
:1080E0006F927F928F929F92AF92BF92CF92DF92C8
:1080F000EF92FF92CF93FC014080518062807380A9
:1081000084809580A680B7809A01AB0160E070E022
:1081100084EB92E40F94CBB827E137EB41ED58E3C1
:108120000F94CCB86B017C01A3019201C301B20191
:108130000F942EB22B013C01A5019401C501B4019D
:108140000F942EB29B01AC01C301B2010F94CCB8C5
:108150004B015C01A7019601C701B6010F942EB235
:108160009B01AC01C1E0C501B4010F94C8B1181660
:108170000CF4C0E08C2FCF91FF90EF90DF90CF9068
:10818000BF90AF909F908F907F906F905F904F9037
:1081900008952F923F924F925F926F927F928F92AB
:1081A0009F92AF92BF92CF92DF92EF92FF920F9386
:1081B0001F93CF93DF93CDB7DEB7A7970FB6F89491
:1081C000DEBF0FBECDBF9EA38DA36FA3242E302E86
:1081D0008E010F5F1F4F8CE0F80111928A95E9F72D
:1081E000EDA1FEA1408051806280738049825A8255
:1081F0006B827C8284809580A680B7808D829E82EF
:10820000AF82B886222351F1BE016B5F7F4FC80158
:108210000E94D33D882309F4E1C12091A41030913C
:10822000A5104091A6105091A710C301B2010F9460
:10823000CBB869837A838B839C832091A81030917B
:10824000A9104091AA105091AB10C501B4010F9430
:10825000CBB86D837E838F83988709C040E050E060
:10826000BA01C8010E946E40882309F4B7C140904A
:108270000F025090100260901102709012028090D4
:108280005B0290905C02A0905D02B0905E0294014F
:10829000A501B201C3010F9480BB181614F042016E
:1082A0005301C401D50189879A87AB87BC87409069
:1082B0002F0250903002609031027090320280E0C4
:1082C00090E0A8E4B2E480932F0290933002A09350
:1082D0003102B09332021D861E861F86188ABE01A7
:1082E000635F7F4FC8010E94FD9A0E94C93D8111C2
:1082F00053C18091A90482FF11C02091AC1030912C
:10830000AD104091AE105091AF1060E070E080EA87
:1083100090EC0F94CBB86B017C0106C0C12CD12C22
:1083200020E2E22E21ECF22E8090AC109090AD1065
:10833000A090AE10B090AF1020E030E0A901C501D0
:10834000B4010F94C8B187FF0BC0A501940160E090
:1083500070E08CE592E40F94CBB84B015C0106C051
:10836000812C912C9CE5A92E92E4B92EA5019401B3
:1083700060915B0270915C0280915D0290915E025F
:108380000F9480BB1816ECF5898E9A8EAB8EBC8E3E
:10839000812C912C80E7A82E81E4B82E8D8A9E8AAC
:1083A000AF8AB88EBE016B5E7F4FCE0149960E94A8
:1083B000429A1091180E1092180E82E00F94AB4161
:1083C0000F945F4112FF1DC08D869E86AF86B88ACE
:1083D00020E030E040EA50E460915B0270915C0282
:1083E00080915D0290915E020F94CCB8698B7A8B7C
:1083F0008B8B9C8BBE01635F7F4FCE0141960E94A9
:10840000429AC98ADA8AEB8AFC8A80E090E0A0EF7F
:10841000B0E48D879E87AF87B88BBE01635F7F4FC7
:10842000CE0141960E94429A1091180E147010923B
:10843000180E82E00F94AB410F945F41332009F492
:10844000DFC02091AC103091AD104091AE10509132
:10845000AF1060E070E080EA90E40F94CBB89B012D
:10846000AC0160915B0270915C0280915D02909121
:108470005E020F9480BB18160CF0C2C060E070E082
:1084800080EC9FE72091AC103091AD104091AE1080
:108490005091AF100F94CCB85B018C019B01AC01E3
:1084A0000F946DBC81117CC08FA18250823050F539
:1084B00080E090E0A0E7B1E48D8F9E8FAF8FB8A3EE
:1084C00060915B0270915C0280915D0290915E020E
:1084D000FFA1F33029F020E030E040EA50E404C08E
:1084E00020E030E048EC51E40F94CCB869A37AA3C3
:1084F0008BA39CA3BE01635E7F4FCE0181960E9439
:10850000429A07C02FA1213021F40E94C03D811161
:1085100005C082E0821508F043C008C0F2E0F21501
:1085200008F061C0A12CB12C00EC1FE720915A0586
:1085300030915B0540915C0550915D05EDA1FEA178
:1085400060817181828193810F94CCB8AB01BC01B1
:1085500080E697E00E94368620915E0530915F05A7
:108560004091600550916105EDA1FEA16481758186
:10857000868197810F94CCB8AB01BC018BE597E065
:108580000E943686A501B80186E597E00E943686EE
:108590008AE00E94F88304C0A12CB12C00EC1FE7F4
:1085A00040922F0250923002609231027092320259
:1085B0009501A801B501C8010F946DBC882361F134
:1085C0000E94C03D60E081E59CE00F9469830E94B9
:1085D0002C8481E49CE00E940A841EC0A12CB12C52
:1085E00000EC1FE719C040922F02509230026092B7
:1085F000310270923202A12CB12C00EC1FE7E0CFC7
:10860000112309F43BCF60915B0270915C02809171
:108610005D0290915E0236CFB501C801A7960FB6F4
:10862000F894DEBF0FBECDBFDF91CF911F910F91A8
:10863000FF90EF90DF90CF90BF90AF909F908F9082
:108640007F906F905F904F903F902F900895CF93C1
:1086500089E693E40E940A84C091F11081EF9BE0C7
:108660000E940A84C11103C087EC9AE102C08DEA1E
:108670009DE00E940A8489EE9BE00E940A8462E3E6
:1086800070E080E090E0CF910C943C8381E00C940A
:108690007386CF92DF92EF92FF92CF93DF93CDB7A5
:1086A000DEB7EC970FB6F894DEBF0FBECDBF9CAF20
:1086B0008BAF81E00E947B3A8B8388E08C8386E1DC
:1086C0008D838BAD9CAD8370992721E0892B09F0B8
:1086D00020E02E8321E08BAD9CAD019709F020E0D6
:1086E0002F8321E08BAD9CAD029709F020E0288715
:1086F0008BAD9CAD8470992721E0892B09F420E093
:1087000029878AE29CE00E940A848E818823C9F02E
:1087100086E29CE00E940A8440E550E060EB7FEF37
:1087200084E00E94F63A40E550E060E570E086E1C2
:108730000E94F63A8AE00E94F88386E00E94CA3AD4
:108740000EC080E29CE00E940A848F81882319F089
:108750008AE19CE002C084E19CE00E940A8480914E
:10876000F2029091F30223E532E048E0F901DE01E4
:10877000919601900D924A95E1F79B878A8789A18E
:108780009AA1ABA1BCA1898B9A8BAB8BBC8B8DA121
:108790009EA1AFA1B8A58D8B9E8BAF8BB88F8A851C
:1087A0009B85FC0180819181A281B38129893A89CD
:1087B0004B895C89BC01CD010F94CCB8DC01CB01A5
:1087C0006C017D018A859B85FC0184819581A68150
:1087D000B7812D893E894F89588DBC01CD010F94F9
:1087E000CCB8DC01CB01C98EDA8EEB8EFC8E8D8F7E
:1087F0009E8FAF8FB8A388E0FE017996DE01D396F5
:1088000001900D928A95E1F788E0FE01F396DE0172
:10881000999601900D928A95E1F7CE0189960E9472
:10882000813A9AAB89AB988581E08927882319F032
:108830008AE00E94F88384E08983898188230CF48C
:10884000D4C08E81882391F089818A301CF480E223
:108850000E94F8838981082E000C990B6AE070E071
:108860000E94A28581E19CE00E940A841A828A818A
:10887000853008F09FC08A81282F30E089A9082E12
:10888000000C990B2817390731F49AA98981981798
:1088900011F481E001C080E08C878E81882341F053
:1088A0008C85882311F08BE501C080E20E94F8835B
:1088B0008A81282F30E08981482F880F550BC90104
:1088C000880F991F880F991F820F931F840F951F80
:1088D000880F991F880F991F885C9F4EFC0180812B
:1088E0009181A281B3818D879E87AF87B88B888560
:1088F000882309F045C02D853E854F8558896D85B3
:108900007E858F8598890F946DBC882359F08E8160
:10891000882319F08AE09CE002C086E09CE00E9477
:108920000A842EC08E81882319F48F81882341F117
:108930008E818823D9F020E030E0A9016D857E8505
:108940008F8598890F9480BB882384F020E030E0E5
:10895000A9016D857E858F8598890F9480BB181637
:1089600014F48BE201C080E20E94F8838D859E851D
:10897000AF85B88943E050E0BC01CD010E94348648
:108980008F81882331F08A81843018F489E00E9435
:10899000F8838E81882341F08C85882311F08DE542
:1089A00001C080E20E94F8830E9446438A818F5F63
:1089B0008A835DCF988581E08927882319F08AE032
:1089C0000E94F8838981882361F08E81882349F091
:1089D000998581E08927882321F080E09CE00E942E
:1089E0000A8489818150898328CF8E818823D1F0A0
:1089F00086E00E94CA3A8AE00E94F88340EB5FEF6B
:108A000060EB7FEF84E00E94F63A40EB5FEF60E5B9
:108A100070E086E10E94F63A8AE00E94F8838AE0DC
:108A20000E94F8838B810E947B3AEC960FB6F894F3
:108A3000DEBF0FBECDBFDF91CF91FF90EF90DF90F3
:108A4000CF9008959091F1109817B1F00E94848E04
:108A50008091F110882339F083E592E00E94C28E64
:108A60001092F11007C081E08093F11083E592E04D
:108A70000E94A78E0D945F41089580E00E942245D8
:108A800060E070E080EC9FE70C94653ACF93C09172
:108A9000F11080E00E9422458FEF8093F01084E671
:108AA000E8E3F0E1DF011D928A95E9F7CC2319F0A4
:108AB000CF910D946141CF9108956F927F928F92E3
:108AC0009F92AF92BF92CF92DF92EF92FF920F935D
:108AD0001F93CF93DF93CDB7DEB7CF55D1090FB634
:108AE000F894DEBF0FBECDBF19860F945E31882388
:108AF00009F0CDC66FEF7FEF80E50E94643D8A8765
:108B00008A85813059F08A85823041F08A858430A7
:108B100029F08AE40E94093D882311F081E001C018
:108B200080E08B878B85882371F00E94848E87E09C
:108B30000E942E95982F81E0992309F480E08823E4
:108B400011F00E94C63A89E40E94093D882309F485
:108B5000A0C0198280910F0C9091100C21E0892BFC
:108B600009F420E0222319F00E94CC3C02C081E0ED
:108B700090E090939B0E80939A0E80919A0E909124
:108B80009B0E49973CF060E070E080EC9FE70E940C
:108B9000653A7BC080919A0E90919B0E9C0121506A
:108BA000310930939B0E20939A0E21E0892B09F412
:108BB00020E0222309F469C08981853120F01982DF
:108BC00080E00E94738620E030E040E06EE87EE0C6
:108BD00081E00F949335A22EB32EC42ED52EE62E0F
:108BE000F72E082F192F2A2D3B2D4C2D5D2D6E2D84
:108BF0007F2D802F912FFE01E65AFF4F2083318376
:108C00004283538364837583CE01865A9F4F9D8729
:108C10008C878C859D85FC01808188235CF460E0D5
:108C200070E080EC9FE70E94653A87EC9DE00E942F
:108C30000A842BC08C859D85FC018081282F880F9C
:108C4000330B8C859D85FC018181482F880F550B46
:108C5000C901880F991F880F991F820F931F840FD6
:108C6000951F880F991F880F991F9C01285C3F4E04
:108C700080E090E0A0ECBFE7F90180839183A283BC
:108C8000B38389818F5F898385CF8EEA9DE00E94BF
:108C90000A8481E50E94093D882309F4F3C180918B
:108CA0000F0C9091100C21E0892B09F420E0222375
:108CB00019F00E94CC3C02C08DE99FEF9B8B8A8B00
:108CC0008A899B898F3F9F4F24F08A899B890397CC
:108CD0002CF086E89DE00E940A84D9C587E69DE0D5
:108CE0000E940A848A899B898130910509F4BDC05C
:108CF0008230910509F462C1892B09F0C3C11A823F
:108D00008A81853008F0BEC11B828B81853008F0D6
:108D1000A8C08A81882F90E0092E000CAA0BBB0BFB
:108D2000BC01CD010F94CFB1DC01CB019C01AD01A1
:108D300060E070E080E290E40F94CBB8DC01CB01FE
:108D40008C8B9D8BAE8BBF8B8B81882F90E0092EF7
:108D5000000CAA0BBB0BBC01CD010F94CFB1DC0101
:108D6000CB019C01AD0160E070E080E290E40F94E3
:108D7000CBB8DC01CB01888F998FAA8FBB8F8A81FA
:108D8000082F10E08B81A82EB12C8A81282F30E08B
:108D90008B81482F50E0C901880F991F880F991FB8
:108DA000820F931F840F951F880F991F880F991F9B
:108DB000885C9F4EFC01C080D180E280F3802C89CA
:108DC0003D894E895F896C897D898E899F890F9441
:108DD0002EB2DC01CB013C014D01288D398D4A8D2D
:108DE0005B8D688D798D8A8D9B8D0F942EB2DC0101
:108DF000CB019C01AD01C401B3010F94CCB8DC01DF
:108E0000CB01BC01CD010F941EBCDC01CB019C0148
:108E1000AD01BC01CD010F94CCB8DC01CB019C01AC
:108E2000AD01C701B6010F94CCB8DC01CB019C01A8
:108E3000AD01C801880F991F880F991F800F911FDE
:108E40008A0D9B1D880F991F880F991F885C9F4E64
:108E5000FC0120833183428353838B818F5F8B831B
:108E600054CF8A818F5F8A834BCF1C828C8185305F
:108E700008F008C18C81082F10E08C81E82EF12CBD
:108E80008C81282F30E08C81482F50E0C901880F59
:108E9000991F880F991F820F931F840F951F880FAA
:108EA000991F880F991F885C9F4EFC0180819181DA
:108EB000A281B38127EE3BEF4FE151E4BC01CD012C
:108EC0000F94CCB8DC01CB019C01AD01C801880F27
:108ED000991F880F991F800F911F8E0D9F1D880F5E
:108EE000991F880F991F885C9F4EFC012083318356
:108EF000428353838C81E82EF12C8C81282F30E023
:108F000081E09C81943008F080E0882F90E0820F0F
:108F1000931F892B19F001E010E002C00FEF1FEF43
:108F20008C81482F50E08C81282F30E081E09C819B
:108F3000943008F080E0882F90E0820F931F892BF7
:108F400019F021E030E002C02FEF3FEFCA01880F97
:108F5000991F880F991F840F951F820F931F880FE9
:108F6000991F880F991F885C9F4EFC018081918119
:108F7000A281B38127EE3BEF4FE151E4BC01CD016B
:108F80000F94CCB8DC01CB019C01AD01C701880F67
:108F9000991F880F991F8E0D9F1D800F911F880F9D
:108FA000991F880F991F885C9F4EFC012083318395
:108FB000428353838C818F5F8C8358CF81E08D8374
:108FC0008D81833008F05EC081E08E838E81833096
:108FD00008F054C083E40E94093D882349F0809141
:108FE0009C0E90919D0EA0919E0EB0919F0E04C07C
:108FF0008AE097EDAFE1B1E42D81C22ED12C2E8114
:10900000A22EB12C2D81422F50E02E81622F70E0D4
:109010009A01220F331F220F331F240F351F260FF3
:10902000371F220F331F220F331F285C3F4EF901D9
:10903000E080F180028113819C01AD01C801B7017C
:109040000F94CCB8DC01CB019C01AD01C601880FA7
:10905000991F880F991F8C0D9D1D8A0D9B1D880FD0
:10906000991F880F991F885C9F4EFC0120833183D4
:10907000428353838E818F5F8E83A8CF8D818F5FD4
:109080008D839ECF8AE40E94093D882399F00F9436
:10909000573180917F159091801521E0892B09F03F
:1090A00020E0822F0F944D9B0F944D310F9461411E
:1090B00081E0898780E50E94093D882309F415C372
:1090C0008091980E9091990E992384F08091980E3A
:1090D0009091990E029754F48091F0108F3F31F4E3
:1090E0001092F01085E49DE00E940A848091980E11
:1090F0009091990E092E000CAA0BBB0B40E050E09A
:1091000026E030E0841B950B2817390708F4EDC2E0
:10911000FC018827EE58FF4F8F4F0D94C3B80E9473
:10912000464587E39DE00E940A84DFC283E40E94F3
:10913000093D982F81E08927882331F00E943D4521
:1091400086E19DE00E940A8480917D1590917E15B4
:10915000029724F180918E0E90918F0EA091900E27
:10916000B091910E25E03DE0AC01BD01C9010E9426
:1091700036868CE20E94F8838091920E9091930E35
:10918000A091940EB091950E42E050E0BC01CD014B
:109190000E94348683E99DE30E940A848091F20252
:1091A0009091F30299A388A380918E0E90918F0ED7
:1091B000A091900EB091910E8C8F9D8FAE8FBF8F2E
:1091C0008091920E9091930EA091940EB091950E75
:1091D0008E879F87A88BB98B88A199A1FC0180817C
:1091E0009181A281B3812C8D3D8D4E8D5F8DBC010F
:1091F000CD010F94CCB8DC01CB016C017D0188A1BD
:1092000099A1FC0184819581A681B7812E853F8536
:1092100048895989BC01CD010F94CCB8DC01CB0140
:10922000C8AAD9AAEAAAFBAA8CAB9DABAEABBFABCE
:10923000CE018E5A9F4F28E0FE01F096DC0101908E
:109240000D922A95E1F7CE01865B9F4F9E012E5A23
:109250003F4F48E0F901DC0101900D924A95E1F79A
:1092600085E50E94093D082F85E40E94093D182FDD
:1092700084E50E94093D382FCE01865B9F4F202F49
:10928000412F632F0F94143F0F94614181E0898730
:109290002CC28FED9CE00E940A8480E090E0A0EA5E
:1092A000B0E488AF99AFAAAFBBAFCE01C89620E0BB
:1092B00041E061E00E94659A83E40E94093D8823B1
:1092C00099F08091960E882331F48091970E88232F
:1092D00021F480E003C081E001C081E091E08927B2
:1092E000882311F081E001C080E0882381F0109292
:1092F0008E0E10928F0E1092900E1092910E109270
:10930000920E1092930E1092940E1092950E82E48B
:109310000E94093D882309F442C080910F0C90916E
:10932000100C21E0892B09F420E0222329F00E946F
:10933000D03CDC01CB0108C060E070E080EA90E442
:109340000F942E33DC01CB018093470390934803A5
:10935000A0934903B0934A03809147039091480337
:10936000A0914903B0914A03BC01CD010E944A3A41
:10937000DC01CB0111E020E030E040EC5FE3BC0118
:10938000CD010F9480BB18160CF010E0112329F0CA
:1093900089EB9CE00E940A847AC281E0898740E0E0
:1093A00050E0BA018EE89EE00E946E40982F81E066
:1093B0008927882329F08BE99CE00E940A8467C2F0
:1093C00040E050E060EA70E488E40E9472A8DC01AA
:1093D000CB019E012A5B3F4FF90180839183A283D9
:1093E000B38384E50E94093D282FCE018A5B9F4FFD
:1093F00047E453E0BC018EE89EE00F94513D89E8BC
:109400009CE00E940A840F9461416FC180918D0E8F
:10941000882309F4E6C080919A0E90919B0E49979B
:109420006CF080919C0E90919D0EA0919E0EB0913B
:109430009F0EBC01CD010E94653A56C180919A0EE3
:1094400090919B0E9C012150310930939B0E2093EB
:109450009A0E21E0892B09F420E0222309F444C16B
:1094600020E030E040E06EE87EE080E00F9493354D
:10947000A22EB32EC42ED52EE62EF72E082F192F8E
:109480002A2D3B2D4C2D5D2D6E2D7F2D802F912F64
:10949000FE01E05CFF4F2083FE01EF5BFF4F308356
:1094A000FE01EE5BFF4F4083FE01ED5BFF4F5083FB
:1094B000FE01EC5BFF4F6083FE01EB5BFF4F7083AF
:1094C000CE01805C9F4F9BA38AA38AA19BA1FC0134
:1094D000808188230CF05AC01F828F81853008F06C
:1094E00003C118868885853008F04CC08F81282FED
:1094F00030E08885482F50E0C901880F991F880FF8
:10950000991F820F931F840F951F880F991F880F33
:10951000991F885C9F4EFC0180819181A281B3815B
:1095200011E09C01AD01BC01CD010F946DBC8823FD
:1095300009F410E0112311F18F81482F50E0888544
:10954000682F70E080919C0E90919D0EA0919E0ED0
:10955000B0919F0E9A01220F331F220F331F240F49
:10956000351F260F371F220F331F220F331F285C92
:109570003F4EF90180839183A283B38388858F5FF7
:109580008887B0CF8F818F5F8F83A7CF8AA19BA160
:10959000FC018081482F880F550B8AA19BA1FC01FB
:1095A0008181682F880F770B80919C0E90919D0E82
:1095B000A0919E0EB0919F0E9A01220F331F220F91
:1095C000331F240F351F260F371F220F331F220F83
:1095D000331F285C3F4EF90180839183A283B383BC
:1095E0002DCF0E94D03CDC01CB018CA39DA3AEA368
:1095F000BFA320E030E040E251E46CA17DA18EA148
:109600009FA10F942EB2DC01CB01BC01CD010F94C0
:1096100062BCDC01CB01BC01CD010F9438BADC0186
:10962000CB014E97019709F040C026E636E646E4A6
:1096300050E46CA17DA18EA19FA10F94CBB8DC0159
:10964000CB0120E030E048EC52E4BC01CD010F94A6
:109650002EB2DC01CB0188A799A7AAA7BBA720E05F
:1096600030E0A90168A579A58AA59BA50F94C8B18A
:10967000882379F088A599A5AAA5BBA59C01AD0171
:1096800060E070E080E291E40F94C0BBDC01CB01AC
:1096900003C080E090E0DC018CAF9DAFAEAFBFAF08
:1096A000CE01CC960F94B45D20C00F94D49A1DC007
:1096B00084E50E94093D682F8EE89EE00F94873A6A
:1096C00014C080919C0E90919D0EA0919E0EB09121
:1096D0009F0E20918D0EAC01BD01822F0F946B3433
:1096E00004C00F94193401C000008CE40E94093DAD
:1096F000882309F455C080910F0C9091100C21E043
:10970000892B09F420E0222319F00E94CC3C05C0EB
:109710008091F010082E000C990B909346038093D3
:1097200045030F944C919DA78CA78CA59DA5892BD3
:1097300029F481EE94E30E940A84A9C08091450334
:1097400090914603992364F08CA59DA59C0121501E
:10975000310980914503909146032817390774F425
:109760008CA59DA59C012150310987E69CE0B9019B
:109770000E94B2858AE00E94F88389C080914503E7
:109780009091460360E070E00F94589180914503FA
:10979000909146038093F01080E69CE00E940A843A
:1097A00083E50E94093D882309F45CC080910F0C79
:1097B0009091100C21E0892B09F420E0222319F06C
:1097C0000E94CC3C05C08091F010082E000C990B33
:1097D00090934603809345038091450390914603FF
:1097E000019619F40E94353B52C00F944C919FA7EB
:1097F0008EA78EA59FA5892B29F481EE94E30E9464
:109800000A843BC08091450390914603992364F0FC
:109810008EA59FA59C01215031098091450390910F
:1098200046032817390774F48EA59FA59C01215083
:10983000310987E69CE0B9010E94B2858AE00E9466
:10984000F8831BC080914503909146030F94BD910E
:1098500080914503909146038093F01080E69CE050
:109860000E940A8484E50E94093D882331F080919A
:109870008B0E90918C0E0E9449430E94623A81E0C7
:109880000F94178580E00F9427841092760FC15AA9
:10989000DF4F0FB6F894DEBF0FBECDBFDF91CF9183
:1098A0001F910F91FF90EF90DF90CF90BF90AF90FE
:1098B0009F908F907F906F9008950C94EE6FCF9251
:1098C000DF92EF92FF920F931F9385E1C82E81E400
:1098D000D82EE12CF12C0CE91FE02DE53CE444EE00
:1098E00051E06EE472E483E59FE00E9483721F9171
:1098F0000F91FF90EF90DF90CF900895CF92DF927D
:10990000EF92FF921F93CF93DF9361E081E00E947B
:10991000F46EC0911310D0E011E089E4E82E8EE0DF
:10992000F82E92E5C92E9EE0D92EC1112AC011232E
:10993000D9F0809112101816BCF040911E10509171
:109940001F1060912010709121104F5F5F4F6F4F7B
:109950007F4F40931E1050931F1060932010709300
:1099600021108F5F80931210809188028823E9F183
:1099700020E030E041E06DE57EE08D2F0E948377AE
:1099800034C0C13059F4809112108130D1F49091DB
:109990000D1010920D1091110EC013C0C23029F598
:1099A00080911210823081F590910D1010920D105F
:1099B000911124C029C0C093540590912E1091118B
:1099C00030C090918802992379F01F92DF92CF9254
:1099D000DF9391E0813019F59F930E9421C60F908B
:1099E0000F900F900F900F9010E0DF5FCF5FD4309B
:1099F00009F09BCF83E080930E1013C0C0935405F1
:109A000090912E1091110DC090918802992361F3CD
:109A10001F92FF92EF92DF9391E08230E9F290E0A3
:109A2000DBCFDF91CF911F91FF90EF90DF90CF9030
:109A30000895EF92FF920F931F93CF93DF93CDB7CB
:109A4000DEB765970FB6F894DEBF0FBECDBF80912D
:109A50000D1010920D10882319F00E94EE6F7AC03D
:109A600060E084E00E94F46E0091131010E08AE33D
:109A7000F82E90E2E92E01110AC080918802882315
:109A800061F120E030E043E06CEE78E323C0013088
:109A900051F480918802882301F120E030E041E018
:109AA0006FE678E317C0023051F480918802882372
:109AB000A1F020E030E041E064E27FE00BC0033041
:109AC000E9F580918802882341F020E030E041E010
:109AD00064E17FE0812F0E948377F982EA8242E18C
:109AE00050E063E273E1CE0103960F94FAB08C89E3
:109AF00087FD1C8A053059F4809188028823A9F0DB
:109B00009E012F5F3F4F41E06AE07FE00BC00630CF
:109B100061F480918802882341F020E030E041E048
:109B200069E673E4812F0E9483771F5F0F5F143013
:109B300009F0A1CF87E080930E100CC0043069F6C5
:109B400080918802882349F220E030E041E069E515
:109B500078E3C0CF65960FB6F894DEBF0FBECDBFD9
:109B6000DF91CF911F910F91FF90EF900895EF92A9
:109B7000FF920F931F93CF93DF93CDB7DEB7659717
:109B80000FB6F894DEBF0FBECDBF80910D101092BE
:109B90000D10882319F00E94EE6F74C060E084E01D
:109BA0000E94F46E0091131010E08AE3F82E90E208
:109BB000E92E01110CC080918802882341F020E039
:109BC00030E043E067EF7EE0812F0E948377F982E7
:109BD000EA8242E150E060EF7EE0CE0103960F940E
:109BE000FAB08C8987FD1C8A013069F48091880263
:109BF000882349F09E012F5F3F4F41E06BEE7EE0EE
:109C0000812F0E948377F982EA8242E150E067EE79
:109C10007EE0CE0103960F94FAB08C8987FD1C8AF2
:109C2000023069F480918802882349F09E012F5FF9
:109C30003F4F41E06EED7EE0812F0E948377F982F5
:109C4000EA8242E150E066ED7EE0CE0103960F9499
:109C5000FAB08C8987FD1C8A033069F480918802F0
:109C6000882349F09E012F5F3F4F41E062ED7EE087
:109C7000812F0E9483771F5F0F5F143009F099CF07
:109C800010930E1065960FB6F894DEBF0FBECDBFD1
:109C9000DF91CF911F910F91FF90EF900895EF9278
:109CA000FF920F931F93CF93DF93CDB7DEB76597E6
:109CB0000FB6F894DEBF0FBECDBF80910D1010928D
:109CC0000D10882319F00E94EE6FB5C060E084E0AB
:109CD0000E94F46E0091131010E08AE3F82E90E2D7
:109CE000E92E01110CC080918802882341F020E008
:109CF00030E042E062EC7EE0812F0E948377F982BF
:109D0000EA8242E150E06DE27FE0CE0103960F94DB
:109D1000FAB08C8987FD1C8A013069F48091880231
:109D2000882349F09E012F5F3F4F40E069EB7EE0C2
:109D3000812F0E948377F982EA8242E150E065EB4D
:109D40007EE0CE0103960F94FAB08C8987FD1C8AC1
:109D5000023059F480918802882309F19E012F5F17
:109D60003F4F40E06CEA7EE017C0033051F4809131
:109D700088028823A1F020E030E040E06AE97EE03C
:109D80000BC0043061F480918802882341F020E008
:109D900030E042E069E87EE0812F0E948377F9821B
:109DA000EA8242E150E06DE27FE0CE0103960F943B
:109DB000FAB08C8987FD1C8A053069F4809188028D
:109DC000882349F09E012F5F3F4F40E069EB7EE022
:109DD000812F0E948377F982EA8242E150E065E8B0
:109DE0007EE0CE0103960F94FAB08C8987FD1C8A21
:109DF000063059F4809188028823A9F09E012F5FD4
:109E00003F4F40E06CEA7EE00BC0073061F4809188
:109E10008802882341F020E030E040E06AE97EE0FB
:109E2000812F0E9483771F5F0F5F143009F059CF95
:109E300088E080930E1065960FB6F894DEBF0FBED3
:109E4000CDBFDF91CF911F910F91FF90EF900895BB
:109E50002F923F924F925F926F927F928F929F923A
:109E6000AF92BF92CF92DF92EF92FF920F931F9328
:109E7000CF93DF9300D01F92CDB7DEB76C010F9464
:109E8000D9B001967601E80EF91EC7010F94D9B03A
:109E9000F7012080F1E0F983211001C01982F70158
:109EA000E80FF91F21E02B838181811101C01B8202
:109EB00060E084E00E94F46E0091131010E039819C
:109EC000832F90E00196FC012B81E20FF11DFA83B4
:109ED000E983011117C080918802882301F1E09184
:109EE0000902E250E33040F4F0E0EE0FFF1FE356CA
:109EF000FD4F6081718102C06DE67EE020E030E0C0
:109F000043E00AC0013059F480918802882339F077
:109F100020E030E041E0B601812F0E9483772220CB
:109F200081F0023089F480918802882381F020E05A
:109F300030E041E0B701812F0E94837733E03C831A
:109F400008C042E04C8305C083E08C8302C093E0EC
:109F50009C83E981FA81319719F4FC81FF5FFC83CE
:109F60002C812013B6C080918802882309F4AEC0EA
:109F700020E030E042E06AE77EE0812F0E948377B4
:109F800030914B033B83612F8BE00E94FBA70E9423
:109F90001179382E4B8147FF0DC04090000F509033
:109FA000010F6090020F7090030F6091040F709189
:109FB000050F0CC040900B1150900C1160900D11CA
:109FC00070900E1160910F1170911011072E000CFE
:109FD000880B990B0F94CFB14B015C0162E070E0EC
:109FE00080E090E00E9450A720E030E040E05FE396
:109FF000C301B2010F94CCB80F9438BACB010F94BF
:10A000009E4D0E9497A76FE270E080E090E00E9472
:10A0100050A731107EC08B818F3F49F0082E000C75
:10A02000990B97FF02C080E090E08B8302C091E023
:10A030009B8325E03B81239FF0011124E950FF4ED3
:10A040008481882309F465C060E270E080E090E0DC
:10A050000E9450A720E030E040E251E4C501B40185
:10A060000F9480BB87FD06C060E270E080E090E066
:10A070000E9450A720E030E048EC52E4C501B40152
:10A080000F9480BB87FD06C060E270E080E090E046
:10A090000E9450A761E070E080E090E00E9450A72D
:10A0A00060E270E080E090E00E9450A720E030E0A5
:10A0B00040E251E4C501B4010F94C8B187FF06C066
:10A0C00060E270E080E090E00E9450A742E04093A0
:10A0D00088021F5F0F5F143009F0FBCE8C818F5F09
:10A0E00080930E100F900F900F900F90DF91CF91F3
:10A0F0001F910F91FF90EF90DF90CF90BF90AF90A6
:10A100009F908F907F906F905F904F903F902F9097
:10A11000089520E030E040E05FE3C501B4010F9412
:10A12000CCB80F9438BACB010F94734D0E9497A707
:10A13000B1CF83EB9FE00C94284F80EC9FE00C9410
:10A14000284F82EE9FE00C94284F8DE790E10C940D
:10A15000284F88E390E10C94284F85E690E10C9419
:10A16000284F88EB90E10C94284F8BE990E10C94F8
:10A17000284F8BE190E10C94284F8CEF9FE00C94DA
:10A18000284F84E00D94638A83E00D94638A82E013
:10A190000D94638A2F923F924F926F927F928F928B
:10A1A0009F92AF92BF92CF92DF92EF92FF920F9366
:10A1B0001F93CF93DF930E944883382E80913415EC
:10A1C00083FBDD27D0F983FF04C00E949483282EEF
:10A1D00001C0212C61E081E00E94F46E1091131007
:10A1E000412C8AEE682E82E0782E9EE8E92E9FE0D0
:10A1F000F92E25E6822E2FE0922E34E8C32E31E090
:10A20000D32E49E6A42E4FE0B42E11110BC080913D
:10A21000121081113BC080910D1010920D10811110
:10A220002FC034C0332009F443C0113061F4809151
:10A230001210813009F0BBC180910D1010920D10E9
:10A240008111AFC1B4C1123061F48091121082301B
:10A2500009F0A3C080910D1010920D10811195C0CE
:10A260009CC0133009F0BFC180911210833009F0F7
:10A27000C4C180910D1010920D108111B6C1BDC1E5
:10A280000E94EE6F80912E10811107C2809188028A
:10A29000882361F081E090911210911180E003E039
:10A2A00023E047E55AE1642D0E940E7631109BC1F0
:10A2B0000E94A283882371F0113071F480911210F2
:10A2C000813009F0B0C180910D1010920D108111F4
:10A2D000A4C1A9C1C1E001C0C2E0C11322C08091E4
:10A2E00012108C130EC080910D1010920D10882347
:10A2F00041F086E492E00E94D97E80912E10811177
:10A30000CCC180918802882361F081E09091121085
:10A31000911380E00EE32EE34FEF52E1642D0E9493
:10A320000E76CF5FC11322C0809112108C130EC025
:10A3300080910D1010920D10882341F08BE79EEB59
:10A340000E94D97E80912E108111A7C18091880230
:10A35000882361F081E090911210911380E00EE368
:10A360002EE345E255E2642D0E940E7681E08C0FCB
:10A37000811326C08091121081137BC180910D1032
:10A3800010920D1081116DC174C18FE59CE40E9483
:10A39000D97E80912E10811180C1809188028823FE
:10A3A00009F479C181E090911210923009F080E0B7
:10A3B0000EE32EE34CE95FE0642D0E940E76C4E0CC
:10A3C00082E08C0F811322C08091121081130EC085
:10A3D00080910D1010920D10882341F08FE593E5C8
:10A3E0000E94D97E80912E10811157C180918802E0
:10A3F000882361F081E090911210911380E00EE3C8
:10A400002EE347E052E4642D0E940E7683E08C0F29
:10A41000811322C08091121081130EC080910D1003
:10A4200010920D10882341F082ED94E50E94D97EB0
:10A4300080912E10811131C180918802882361F0B2
:10A4400081E090911210911380E00EE32EE343E738
:10A450005FE0642D0E940E7684E08C0F311099C06D
:10A46000811327C08091121081130CC080910D10B0
:10A4700010920D10882331F00F94D92680912E1060
:10A4800081110BC180918802882399F0DF92CF92CD
:10A49000BF92AF924F9281E090911210911380E0A1
:10A4A0008F930E9421C60F900F900F900F900F90E6
:10A4B0000F9085E08C0FDD2309F44CC0211069C09A
:10A4C000811320C09091121091130EC080910D1035
:10A4D00010920D10882341F09092550C8092540CEC
:10A4E00080912E108111D9C080918802882351F06B
:10A4F00081E0911380E000E22EE348E55FE0642D07
:10A500000E940E7686E08C0F811322C0809112107B
:10A5100081130EC080910D1010920D10882341F010
:10A5200082EE91E00E94D97E80912E108111B5C0FB
:10A5300080918802882361F081E09091121091133C
:10A5400080E00EE32EE347EF56E2642D0E940E7684
:10A5500087E01EC081131BC080911210811302C0BE
:10A5600010920D1090918802992389F01F921F92EA
:10A57000FF92EF924F9291E0811390E09F930E949F
:10A5800021C60F900F900F900F900F900F9086E0C4
:10A590008C0F43941F5F94E0491237CE80930E10C6
:10A5A0007CC00F94AE8380912E10811176C0809173
:10A5B0008802882309F46FC07F926F9287EA9FE038
:10A5C0009F938F934F9281E090911210913009F0F8
:10A5D00080E08F930E9421C60F900F900F900F90F4
:10A5E0000F900F9058C0C4E09DCE8BE99AEB0E946B
:10A5F000D97E80912E10811150C0809188028823CD
:10A6000009F449C081E090911210933009F080E084
:10A610000EE32EE347E95FE0CFCE0F9454848091A0
:10A620002E1081113AC0809188028823C1F080E900
:10A6300091E09F938F9381E89FE09F938F934F9238
:10A6400081E090911210913009F080E08F930E9488
:10A6500021C60F900F900F900F900F900F90C2E0B7
:10A6600060CE8DE49EE50E94D97E80912E108111EE
:10A6700014C080918802882309F4A2CE81E09091D1
:10A680001210911380E00EE32EE342E05EE0642DB1
:10A690000E940E7695CEC4E069CEDF91CF911F91D6
:10A6A0000F91FF90EF90DF90CF90BF90AF909F9071
:10A6B0008F907F906F904F903F902F900895AF9222
:10A6C000BF92CF92DF92EF92FF920F931F93CF939F
:10A6D000DF930E94A283882311F081E001C082E011
:10A6E0008093D10F0E94E36F182F61E081E00E94F8
:10A6F000F46ED0911310C0E087E3E82E8EE0F82EC0
:10A700009CE3C92E9EE0D92E21E4A22E2EE0B22E8B
:10A71000D11120C08091121081110CC080910D10B8
:10A7200010920D10882331F00E94EE6F80912E1050
:10A7300081112DC180918802882361F081E0909180
:10A740001210911180E003E023E04BE355E26C2FFF
:10A750000E940E7680919F0581111BC080910F1180
:10A7600090911011209151023091520221503109E3
:10A770008217930774F4D13009F0E2C0809112106F
:10A780008130E9F480910D1010920D1081110FC0ED
:10A7900016C0D13029F590911210913009F0B3C054
:10A7A00080910D1010920D108111A5C0ACC087ECE6
:10A7B00090E50E94D97E80912E108111E8C0809191
:10A7C0008802882369F081E090911210913009F09D
:10A7D00080E00EE32EE347E052E46C2F0E940E76F9
:10A7E000112311F082E07FC080919F05811150C03C
:10A7F00080910F11909110112091510230915202CD
:10A8000021503109821793070CF0BAC0D23019F5E4
:10A8100080911210823071F480910D1010920D1001
:10A82000882341F084EC90E50E94D97E80912E101F
:10A830008111ADC080918802882369F081E09091F8
:10A840001210923009F080E00EE32EE347E252E46A
:10A850006C2F0E940E7620910F1130911011809173
:10A860009F05811118C08091510290915202019769
:10A870002817390784F4D330A9F58091121083305A
:10A8800001F580910D1010920D10811112C019C0A8
:10A89000D23009F458C0D33029F59091121093307A
:10A8A00009F044C080910D1010920D10811136C036
:10A8B0003DC081EC90E50E94D97E80912E108111DF
:10A8C00066C080918802882369F081E0909112101F
:10A8D000933009F080E00EE32EE347E152E46C2F61
:10A8E0000E940E7684E0CF5FDF5FC43009F010CFA6
:10A8F00080930E104CC0B092550CA092540C8091D5
:10A900002E10811144C080918802882309F468CFF9
:10A9100081E0913009F080E000E25CCFF092550CCC
:10A92000E092540C80912E10811131C080918802E8
:10A930008823C1F281E0933009F080E000E2CCCFBF
:10A94000111150CF59CF90911210923071F4809123
:10A950000D1010920D10882341F0D092550CC0922A
:10A96000540C80912E10811112C08091880288238E
:10A9700009F471CF81E0923009F080E000E265CF08
:10A98000D23009F320910F11309110116CCFDF916B
:10A99000CF911F910F91FF90EF90DF90CF90BF90DC
:10A9A000AF9008950F93CF93DF9361E081E00E9411
:10A9B000F46ED0911310C0E0D1110BC08091121031
:10A9C000811129C080910D1010920D1081111DC0B0
:10A9D00022C0D13059F480911210813091F58091CC
:10A9E0000D1010920D10811124C02BC0D23009F02F
:10A9F00041C080911210823009F051C080910D1039
:10AA000010920D10811143C04AC00E94EE6F8091D8
:10AA10002E1081116AC080918802882319F181E08B
:10AA200090911210911180E003E023E04BE355E296
:10AA300016C089E19DE40E94D97E80912E1081117B
:10AA400054C080918802882369F081E090911210AF
:10AA5000913009F080E00EE32EE346E45FE06C2FD6
:10AA60000E940E76CF5FDF5FC43009F0A5CFC093A0
:10AA70000E103BC0D330B1F780911210833031F506
:10AA800080910D1010920D10811118C01FC087EB1E
:10AA90009DE40E94D97E80912E10811126C0809164
:10AAA00088028823F9F281E090911210923009F027
:10AAB00080E00EE32EE34BE35FE0D1CF8FE49EE432
:10AAC0000E94D97E80912E1081110FC08091880242
:10AAD000882341F281E090911210933009F080E0D8
:10AAE0000EE32EE34FE25FE0BACFDF91CF910F91FB
:10AAF0000895EF92FF920F931F93CF93DF93CDB7FB
:10AB0000DEB72B970FB6F894DEBF0FBECDBF7C012A
:10AB100020911410422F022E000C550B809115101D
:10AB2000833051F0843019F089E19EE00AC027FF9C
:10AB300006C085E29EE005C08EE29EE002C080E194
:10AB40009EE05F932F939F938F938E010F5F1F4F14
:10AB50001F930F930F9460B1C7010F947C72C801CB
:10AB60000E94D86E0F900F900F900F900F900F9043
:10AB70002B960FB6F894DEBF0FBECDBFDF91CF91FD
:10AB80001F910F91FF90EF900895E091111087E1D0
:10AB9000E802F0011124E95FFE4E808591850C9456
:10ABA0007955E091111086E0E802F0011124E0559A
:10ABB000FF4E808191810C94795561116093090257
:10ABC00040934B03082E000C990BAA0BBB0B8C3047
:10ABD000910590F5FC018827E758FF4F8F4F0D94A2
:10ABE000C3B88DE990E51FC085EA90E51CC089EAED
:10ABF00090E519C08DEA90E516C081EB90E513C091
:10AC000085EB90E510C089EB90E50DC08DEB90E5EC
:10AC10000AC0109254058EE79CE405C089E990E5CE
:10AC200002C081EA90E521E02093D00F20E040E0CF
:10AC300060E070E00C944F6F0C94966FCF93DF93AD
:10AC4000EC01CB01BA010F94CFB120E030E0A901B3
:10AC50000F94CCB80F943FBA79836883DF91CF917A
:10AC60000895CF93DF93EC01CB01BA010F94CFB1DC
:10AC70002DEC3CEC4CEC5DE30F94C6B920E030E0E9
:10AC8000A9010F94CCB80F943FBA79836883DF9100
:10AC9000CF910895CF93DF93EC01CB01BA010F94CC
:10ACA000CFB129EC38EC48EC5EE30F94C6B920E054
:10ACB00030E040E05FE30F94CCB80F943FBA688374
:10ACC000DF91CF910895CF93DF93CDB7DEB728976B
:10ACD0000FB6F894DEBF0FBECDBF21E020934C032A
:10ACE00019821A821B821C8240E050E060EA70E404
:10ACF0004D835E836F837887AE014F5F5F4FBE01E8
:10AD00006B5F7F4F0E94249A10924C0380E090E08A
:10AD10000E942C708DEC9CECACE4BDE3809380022F
:10AD200090938102A0938202B093830220E040E0DE
:10AD300060E070E08EE491E00E944F6F28960FB6BD
:10AD4000F894DEBF0FBECDBFDF91CF910895CF93B2
:10AD5000DF93CDB7DEB728970FB6F894DEBF0FBEEE
:10AD6000CDBFCE01019628E0FC0111922A95E9F7AA
:10AD700020914C03211102C00E94635628960FB601
:10AD8000F894DEBF0FBECDBFDF91CF91089586E06E
:10AD900093E19093550C8093540C20E040E060E0E8
:10ADA00070E08FE49AE50C944F6F8F929F92AF9270
:10ADB000BF92CF92DF92EF92FF920F931F93CF93A8
:10ADC000DF9361E081E00E94F46ED0911310C0E047
:10ADD000D1110BC08091121081112AC080910D10E9
:10ADE00010920D1081111EC023C0D13061F48091EA
:10ADF0001210813009F05AC080910D1010920D1080
:10AE0000811128C053C0D23009F075C08091121052
:10AE1000823009F0A2C080910D1010920D108111A6
:10AE200086C09BC00E94EE6F80912E10811173C26C
:10AE300080918802882309F455C081E09091121016
:10AE4000911180E003E023E041E451E16C2F0E9486
:10AE50000E7648C0C090D810D090D910E090DA108B
:10AE6000F090DB1020E030E040E251E4C701B60191
:10AE70000F94CCB84B015C0120E030E040E251E49B
:10AE8000C701B6010F94CBB89B01AC0198E9C92E5C
:10AE900099E5D92E8501740168ED70E189EC95E2A0
:10AEA0000F94C3A880912E10811135C28091880221
:10AEB0008823C1F011E080911210813009F010E078
:10AEC0006091D8107091D9108091DA109091DB10B8
:10AED0000E94F76A00E09C0149EC55E26C2F812F3B
:10AEE0000E948775CF5FDF5FC43009F071CF8AE0C1
:10AEF00080930E1010C2D33061F480911210833011
:10AF000009F069C080910D1010920D1081114DC093
:10AF100062C0D430E1F580911210843009F099C0FC
:10AF200080910D1010920D1081117DC092C018E912
:10AF3000C12E19E5D12EE12CF12C00EA10E420E01D
:10AF400030E040EA50EC64EE70E181E091E10F9472
:10AF50000BAA80912E108111DEC180918802882376
:10AF600009F4C0CF11E080911210823009F010E096
:10AF70006091E4107091E5108091E6109091E710D7
:10AF80000E94886D00E09C0141E051E1A7CFD530DF
:10AF9000E1F580911210853009F0B0C080910D105C
:10AFA00010920D1081117EC0A9C0A8E9CA2EA9E592
:10AFB000DA2EE12CF12C00EA10E420E030E040EA47
:10AFC00050EC68EE70E18EEF90E10F940BAA809147
:10AFD0002E108111A0C180918802882309F482CFAC
:10AFE00011E080911210833009F010E06091E810B8
:10AFF0007091E9108091EA109091EB100E94886D99
:10B0000000E09C014EEF50E169CFD630E1F5809130
:10B010001210863009F0B0C080910D1010920D1002
:10B02000811194C0A9C0E8E9CE2EE9E5DE2EE12C1D
:10B03000F12C00EA10E420E030E040EA50EC6CEE45
:10B0400070E18BEF90E10F940BAA80912E1081118B
:10B0500062C180918802882309F444CF11E0809175
:10B060001210843009F010E06091EC107091ED1036
:10B070008091EE109091EF100E94886D00E09C018D
:10B080004BEF50E12BCFD73009F052C08091121016
:10B09000873009F0B0C080910D1010920D10811111
:10B0A00094C0A9C0C090DC10D090DD10E090DE10FC
:10B0B000F090DF1020E030E040EA50E4C701B60134
:10B0C0000F94CCB84B015C0120E030E040EA50E442
:10B0D000C701B6010F94CBB89B01AC0178E9C72E2C
:10B0E00079E5D72E850174016CED70E186E791E179
:10B0F0000F94C3A880912E1081110DC180918802F8
:10B10000882309F4EFCE11E080911210853009F008
:10B1100010E06091DC107091DD108091DE10909154
:10B12000DF100E94F76A00E09C0146E751E1D6CEAD
:10B13000D830E1F580911210883009F08CC08091F0
:10B140000D1010920D10811170C085C058E9C52EE8
:10B1500059E5D52EE12CF12C00EA10E420E030E096
:10B1600040EA50EC68EC70E188EF90E10F940BAA94
:10B1700080912E108111CFC080918802882309F41C
:10B18000B1CE11E080911210863009F010E060918C
:10B19000C8107091C9108091CA109091CB100E9474
:10B1A000886D00E09C0148EF50E198CED93009F05D
:10B1B00099CE80911210893009F093C080910D10C2
:10B1C00010920D10811161C08CC038E9C32E39E591
:10B1D000D32EE12CF12C00EA10E420E030E040EA2C
:10B1E00050EC6CEC70E185EF90E10F940BAA80912C
:10B1F0002E10811190C080918802882309F472CEAC
:10B2000011E080911210873009F010E06091CC10AD
:10B210007091CD108091CE109091CF100E94886DCA
:10B2200000E09C0145EF50E159CE98E9C92E99E51F
:10B23000D92EE12CF12C00EA10E420E030E040EAC5
:10B2400050EC60ED70E182EF90E10F940BAA8091D9
:10B250002E10811160C080918802882309F442CEAB
:10B2600011E080911210883009F010E06091D01048
:10B270007091D1108091D2109091D3100E94886D5E
:10B2800000E09C0142EF50E129CEC090E010D09048
:10B29000E110E090E210F090E31020E030E040EAAE
:10B2A00050E4C701B6010F94CCB84B015C0120E01B
:10B2B00030E040EA50E4C701B6010F94CBB89B01DF
:10B2C000AC0188E9C82E89E5D82E8501740160EEAD
:10B2D00070E18DE691E10F94C3A880912E10811149
:10B2E0001AC080918802882309F4FCCD11E0809176
:10B2F0001210893009F010E06091E0107091E110B7
:10B300008091E2109091E3100E94F76A00E09C01A6
:10B310004DE651E1E3CDDF91CF911F910F91FF9069
:10B32000EF90DF90CF90BF90AF909F908F90089557
:10B330000E9446450D94D2484F925F926F927F9241
:10B340008F929F92AF92BF92CF92DF92EF92FF9235
:10B35000CF93DF93CDB7DEB728970FB6F894DEBF53
:10B360000FBECDBF2BED3FE049E450E4FC0160810E
:10B370007181828193810F942EB220E030E044E30A
:10B3800053E40F94C6B96B017C010F94C1B94B0112
:10B390005C01C701B6010F9410BC2B013C010F9456
:10B3A00079486B017C019B01AC01C501B4010F948C
:10B3B0002EB269837A838B839C83A7019601C30194
:10B3C000B2010F942EB26D837E838F839887809114
:10B3D0004C03811104C0CE0101960E946356289649
:10B3E0000FB6F894DEBF0FBECDBFDF91CF91FF90B7
:10B3F000EF90DF90CF90BF90AF909F908F907F9015
:10B400006F905F904F900895CF93DF9300D01F927D
:10B41000CDB7DEB780E090E0A2E5B3E489839A83FC
:10B42000AB83BC83CE0101960E949C590F900F9074
:10B430000F900F90DF91CF910895CF93DF9300D0BD
:10B440001F92CDB7DEB780E090E0A5EAB3E4898330
:10B450009A83AB83BC83CE0101960E949C590F90C6
:10B460000F900F900F90DF91CF910895CF93DF93BE
:10B4700000D01F92CDB7DEB780E090E0A4EBB2E43D
:10B4800089839A83AB83BC83CE0101960E949C5929
:10B490000F900F900F900F90DF91CF9108958091B2
:10B4A0008802882341F020E030E041E06EE17CE159
:10B4B00081E00E9483778091A8048770873011F41F
:10B4C0000C94EE6F08950F94CFB120E030E0A90105
:10B4D0000F94CCB80F943FBACB010D94D44D0F9478
:10B4E000CFB12DEC3CEC4CEC5DE30F94C6B920E001
:10B4F00030E0A9010F94CCB80F943FBACB010D9462
:10B50000034E0F94CFB129EC38EC48EC5EE30F9476
:10B51000C6B920E030E040E05FE30F94CCB80F9470
:10B520003FBA862F0D94694E6EE176E583E69AE583
:10B530000C94E77461E376E58FE69AE50C94E77482
:10B540006AE476E581E89AE50C94E7743F924F92BD
:10B550005F926F927F928F929F92AF92BF92CF92A3
:10B56000DF92EF92FF920F931F93CF93DF93CDB7AC
:10B57000DEB728970FB6F894DEBF0FBECDBF309070
:10B58000111061E081E00E94F46E20911310288771
:10B590001F8211E0232D30E0C901880F991FAC01F3
:10B5A00047565D4B5A83498346E0429FC001439F03
:10B5B000900D1124FC01E055FF4E3F019F012C5FCF
:10B5C0003F4F3C832B832F0132E0430E511CAC01D3
:10B5D0004E545F4E5E834D83588551112CC011230C
:10B5E000D9F0809112101816BCF040911E105091A5
:10B5F0001F1060912010709121104F5F5F4F6F4FAF
:10B600007F4F40931E1050931F1060932010709333
:10B6100021108F5F8093121080918802882381F11E
:10B62000E981FA816591749120E030E043E08F81F7
:10B630000E94837725C08885813011F58091121092
:10B64000813061F480910D1010920D10882331F03B
:10B650000E94EE6F80912E1081112DC18091880281
:10B66000882369F081E090911210913009F080E018
:10B6700003E023E042E05EE06F810E940E7610E07E
:10B68000EB81FC8180818093D10FF885F23071F4D9
:10B690003092111080911210823009F040C08091D8
:10B6A0000D1010920D1081112EC039C02885233045
:10B6B00061F480911210833009F081C080910D10E7
:10B6C00010920D1081114FC07AC0F885F43061F4EA
:10B6D00080911210843009F0B4C080910D10109246
:10B6E0000D10811180C0ADC0F885F53079F58091DD
:10B6F0001210853009F0C0C080910D1010920D100D
:10B700008111B4C0B9C041EF5FEB61ED7FE081E32F
:10B7100095E20F94BFAA80912E108111CCC0809128
:10B720008802882391F011E080911210823009F094
:10B7300010E08091D10F0F94694E00E09C0141E32D
:10B7400055E26F81812F0E94877510E02F812F5F56
:10B750002F8338853F5F3887243009F03DCF86E05E
:10B7600080930E10A8C0F3016081718180E090E0A9
:10B770000F94CDB120E030E0A9010F94CCB820E0C7
:10B7800030E040EA50E40F94CBB80F943FBA812CDC
:10B79000912C24E9A22E2AE5B22E6B01E12CF12C8A
:10B7A0008701EA9425E030E040E050E0B3018DE00D
:10B7B00095E30F949E8880912E1081117CC080911A
:10B7C0008802882311F211E080911210833009F071
:10B7D00010E0F301808191810F94D44D00E09C0131
:10B7E0004DE055E3AECFF2016081718180E090E0E1
:10B7F0000F94CDB120E030E0A9010F94CCB820E047
:10B8000030E040EA50E40F94CBB80F943FBA812C5B
:10B81000912C84E9A82E8AE5B82E6B0117E8E12E59
:10B82000F12C00E010E025E030E040E050E06D81D8
:10B830007E818AE495E20F949E8880912E1081117A
:10B840003AC080918802882309F47FCF11E080916B
:10B850001210843009F010E0F201808191810F9480
:10B86000D44D00E09C014AE455E26BCF0F945C7F1D
:10B8700080912E1081111FC080918802882309F4C5
:10B8800064CF20EE31E03F932F9383E291E19F93C9
:10B890008F93FF81FF9381E090911210953009F012
:10B8A00080E08F930E9421C60F900F900F900F9011
:10B8B0000F900F904ACF28960FB6F894DEBF0FBEB8
:10B8C000CDBFDF91CF911F910F91FF90EF90DF904F
:10B8D000CF90BF90AF909F908F907F906F905F9030
:10B8E0004F903F9008956F927F928F929F92AF9268
:10B8F000BF92CF92DF92EF92FF920F931F93CF935D
:10B90000DF931091A804177061E081E00E94F46E4B
:10B91000D0911310C0E086ECE82E82E0F82E95E17D
:10B92000C92E91E1D92E20EEA22E21E0B22E33E2D3
:10B93000832E31E1932E42ED642E41E1742ED1111C
:10B940000BC080911210811128C080910D101092AF
:10B950000D1081111CC021C0D13059F490911210EA
:10B96000913091F580910D1010920D10811124C02D
:10B970002BC0D230D1F580911210823009F057C01F
:10B9800080910D1010920D1081114BC050C00E947B
:10B99000EE6F80912E10811171C1809188028823F1
:10B9A00009F4AAC081E090911210911180E003E0A7
:10B9B00023E04BE355E215C07092550C6092540C95
:10B9C00080912E1081115AC180918802882309F438
:10B9D00093C081E0913009F080E000E22EE341EC79
:10B9E00051E16C2F0E940E7687C0D33061F48091B4
:10B9F0001210833009F049C080910D1010920D1083
:10BA000081113DC042C0D43061F580911210843064
:10BA100009F0B1C080910D1010920D108111A3C0DA
:10BA2000AAC00F945C7F80912E10811127C1809154
:10BA30008802882309F460C0BF92AF929F928F92D0
:10BA4000CF9381E090911210923009F080E08F93B3
:10BA50000E9421C60F900F900F900F900F900F90A3
:10BA60004BC0D53009F048C080911210853071F577
:10BA700080910D1010920D10811120C027C00F94DD
:10BA8000717F80912E108111F9C0809188028823E6
:10BA900079F1FF92EF92DF92CF92CF9381E0909174
:10BAA0001210933009F080E08F930E9421C60F900E
:10BAB0000F900F900F900F900F901AC087EC96E5A3
:10BAC0000E94D97E80912E108111D8C08091880269
:10BAD000882309F461C081E090911210953009F03B
:10BAE00080E00EE32EE344E95EE36C2F0E940E76C5
:10BAF0001730D9F086E01AC01730E1F7D63029F5B3
:10BB0000809112108630D1F080918802882369F0EC
:10BB100081E090911210963009F080E00EE32EE360
:10BB200045E951E16C2F0E940E768AE0CF5FDF5F1E
:10BB3000C43009F004CF80930E10A0C080910D1086
:10BB400010920D10811139C0DFCFD73041F58091AF
:10BB50001210873009F052C080910D1010920D1014
:10BB6000811144C04BC085ED96E50E94D97E80913D
:10BB70002E10811183C080918802882369F081E0B2
:10BB800090911210943009F080E00EE32EE341EA28
:10BB900051E16C2F0E940E76173009F0ABCFD830F0
:10BBA000B1F480911210883009F040C080910D10DE
:10BBB00010920D10811132C039C084E09AE50E94C4
:10BBC000D97E80912E10882309F49ECF57C0D9309A
:10BBD00009F0ABCF80911210893009F03FC08091FD
:10BBE0000D1010920D10811131C038C08DE19AE511
:10BBF0000E94D97E80912E10811140C080918802D0
:10BC0000882309F492CF81E090911210973009F0C7
:10BC100080E00EE32EE349E851E184CF86E39AE524
:10BC20000E94D97E80912E10811128C080918802B7
:10BC3000882309F47ACF81E090911210983009F0AE
:10BC400080E00EE32EE34DE751E16CCF87EA96E505
:10BC50000E94D97E80912E10811110C0809188029F
:10BC6000882309F462CF81E090911210993009F095
:10BC700080E00EE32EE340EB51E154CFDF91CF9112
:10BC80001F910F91FF90EF90DF90CF90BF90AF90FA
:10BC90009F908F907F906F9008953F924F925F9208
:10BCA0006F927F928F929F92AF92BF92CF92DF92CC
:10BCB000EF92FF920F931F93CF93DF930E94E36F56
:10BCC000382E61E081E00E94F46EC0911310D0E044
:10BCD00036EC632E32E0732E45E1442E41E1542EC2
:10BCE000C1110BC080911210811129C080910D10DB
:10BCF00010920D1081111DC022C0C13059F48091E5
:10BD00001210813099F580910D1010920D10811153
:10BD100025C02CC0C23009F03CC080911210823086
:10BD200009F05CC080910D1010920D1081114EC071
:10BD300055C00E94EE6F80912E108111C9C1809173
:10BD40008802882309F4ACC081E09091121091110F
:10BD500080E003E023E04BE355E217C08AE496EC71
:10BD60000E94D97E80912E108111B2C180918802EB
:10BD7000882309F495C081E090911210913009F068
:10BD800080E00EE32EE342E651E16D2F0E940E7635
:10BD900087C0C33061F480911210833009F064C011
:10BDA00080910D1010920D10811128C05DC0C4301B
:10BDB00009F076C080911210843009F089C080911A
:10BDC0000D1010920D1081117BC082C087EA96EC95
:10BDD0000E94D97E80912E1081117AC180918802B3
:10BDE000882309F45DC081E090911210923009F02F
:10BDF00080E00EE32EE340EE50E1C7CF20E030E0DC
:10BE000048EC52E46091AC107091AD108091AE108E
:10BE10009091AF100F942EB220E030E0A9010F9462
:10BE2000CCB820E030E04AE755E40F94CCB80F944A
:10BE30003FBA812C912C81EDA82E84ECB82E6B0199
:10BE400010E7E12E17E1F12E00E010E020E630EFE0
:10BE50004FEF5FEF6CEA70E181ED90E10F949E8807
:10BE600080912E10811134C1809188028823C1F005
:10BE700011E080911210833009F010E06091AC1055
:10BE80007091AD108091AE109091AF100E94BB6D7B
:10BE900000E09C0141ED50E16D2F812F0E948775DC
:10BEA00031102BC0C53039F580911210853009F062
:10BEB000FCC080910D1010920D108111EEC0F5C0E4
:10BEC00082E091EC0E94D97E80912E10811100C1F8
:10BED00080918802882321F381E0909112109430A0
:10BEE00009F080E00EE32EE343E551E16D2F0E945F
:10BEF0000E76311002C016E001C015E029E9E22EED
:10BF000022E4F22ED12CC1132BC0F701859194911C
:10BF1000D09211109093101080930F1080911210F6
:10BF20008C130EC080910D1010920D10882341F0DB
:10BF300086EA9AE50E94D97E80912E108111C8C0B0
:10BF400080918802882361F081E090911210911312
:10BF500080E00EE32EE342E351E16D2F0E940E7666
:10BF6000012F11E0100FD39422E0E20EF11C82E0C9
:10BF7000D812C9CF1C132BC0809112108C130CC087
:10BF800080910D1010920D10882331F00F945C7F7A
:10BF900080912E1081119CC0809188028823B9F075
:10BFA00080EE91E09F938F9383E291E19F938F9333
:10BFB000DF9381E0909112109C1380E08F930E9498
:10BFC00021C60F900F900F900F900F900F9082E06E
:10BFD000800F31105AC08C1327C0809112108C131F
:10BFE0000CC080910D1010920D10882331F00F9429
:10BFF000717F80912E1081116BC0809188028823FF
:10C0000099F07F926F925F924F92DF9381E09091CF
:10C0100012109C1380E08F930E9421C60F900F9006
:10C020000F900F900F900F9013E0100F1C132BC068
:10C0300080911210C8130CC080910D1010920D1039
:10C04000882331F00F94757F80912E10811140C0AC
:10C05000809188028823B9F08AE291E09F938F93C0
:10C0600084E091E19F938F93DF9381E09091121090
:10C07000911380E08F930E9421C60F900F900F9034
:10C080000F900F900F9084E0800FDF5FCF5FD43070
:10C0900009F026CE80930E101BC083E79CE50E941A
:10C0A000D97E80912E10811113C08091880288233F
:10C0B00009F421CF81E090911210953009F080E0D1
:10C0C0000EE32EE341E451E16D2F0E940E7613CF73
:10C0D000DF91CF911F910F91FF90EF90DF90CF9064
:10C0E000BF90AF909F908F907F906F905F904F9098
:10C0F0003F900895CF92DF92EF92FF920F931F939C
:10C10000CF93DF9361E081E00E94F46ED091131031
:10C11000C0E0D1110BC08091121081112AC0809112
:10C120000D1010920D1081111EC023C0D13061F48A
:10C1300080911210813009F043C080910D1010924F
:10C140000D10811128C03CC0D23009F05EC0809132
:10C150001210823009F08AC080910D1010920D10DB
:10C1600081116FC083C00E94EE6F80912E108111EB
:10C17000F7C080918802882309F43EC081E0909145
:10C180001210911180E003E023E040EE50E16C2FAB
:10C190000E940E7631C00F94AA89E12C10E8F12E8E
:10C1A00007E714E420E030E040E85FE366E675E08E
:10C1B00084E992E10F940E8980912E108111D0C0F4
:10C1C000809188028823C1F011E0809112108130A3
:10C1D00009F010E06091660570916705809168052F
:10C1E000909169050E949F6E00E09C0144E952E134
:10C1F0006C2F812F0E948775CF5FDF5FC43009F0FD
:10C2000088CF85E080930E10ABC0D33061F480916D
:10C210001210833009F059C080910D1010920D104A
:10C2200081113EC052C0D43039F780911210843051
:10C2300009F07CC080910D1010920D1081115FC02B
:10C2400075C00F94AA89E12C10E8F12E07E714E4D9
:10C2500020E030E040E85FE36AE675E08CE892E1D8
:10C260000F940E8980912E1081117AC080918802DE
:10C27000882309F4C1CF11E080911210823009F0B7
:10C2800010E060916A0570916B0580916C0590914A
:10C290006D050E949F6E00E09C014CE852E1A8CF22
:10C2A0000F94AA89E12C10E8F12E07E714E420E0AE
:10C2B00030E040E85FE36EE675E084E892E10F94D9
:10C2C0000E8980912E1081114BC0809188028823A5
:10C2D00009F492CF11E080911210833009F010E040
:10C2E00060916E0570916F05809170059091710558
:10C2F0000E949F6E00E09C0144E852E179CF0F94C8
:10C30000AA89C12CD12CE12C10E8F12E07E714E406
:10C310002DEC3CEC4CEC5DE362E775E08CE792E1E0
:10C320000F94C3A880912E1081111AC080918802A9
:10C33000882309F461CF11E080911210843009F054
:10C3400010E0609172057091730580917405909171
:10C3500075050E94F76A00E09C014CE752E148CF66
:10C36000DF91CF911F910F91FF90EF90DF90CF90D1
:10C370000895EF92FF920F931F93CF93DF9361E0A5
:10C3800081E00E94F46ED0911310C0E0D1110BC077
:10C390008091121081112AC080910D1010920D1001
:10C3A00081111EC023C0D13061F480911210813000
:10C3B00009F043C080910D1010920D10811128C01A
:10C3C0003CC0D23009F05EC080911210823009F07A
:10C3D0008AC080910D1010920D1081116FC083C022
:10C3E0000E94EE6F80912E1081116EC180918802A3
:10C3F000882309F43EC081E090911210911180E0F1
:10C4000003E023E040EE50E16C2F0E940E7631C035
:10C410000F94AA89E12C10ECF12E09E714E420E036
:10C4200030E040E85FE367E77BE080E492E10F946F
:10C430000E8980912E10811147C180918802882336
:10C44000C1F011E080911210813009F010E060918C
:10C45000770B7091780B8091790B90917A0B0E94F9
:10C460009F6E00E09C0140E452E16C2F812F0E94FE
:10C470008775CF5FDF5FC43009F088CF87E0809396
:10C480000E1022C1D33061F480911210833009F074
:10C4900067C080910D1010920D1081114CC060C0CA
:10C4A000D430D9F580911210843009F097C0809172
:10C4B0000D1010920D1081117CC090C00F94AA89AC
:10C4C000E12C10ECF12E09E714E420E030E040E824
:10C4D0005FE36BE77BE089E392E10F940E89809143
:10C4E0002E108111F1C080918802882309F4C1CFF8
:10C4F00011E080911210823009F010E060917B0B06
:10C5000070917C0B80917D0B90917E0B0E949F6EB1
:10C5100000E09C0149E352E1A8CFD530D9F58091E4
:10C520001210853009F088C080910D1010920D1006
:10C5300081116EC081C00F94AA89E12C10ECF12EFC
:10C5400009E714E420E030E040E85FE36FE77BE0D8
:10C5500082E392E10F940E8980912E108111B4C074
:10C5600080918802882309F484CF11E08091121011
:10C57000833009F010E060917F0B7091800B809107
:10C58000810B9091820B0E949F6E00E09C0142E320
:10C5900052E16BCFD63009F06CCF8091121086300B
:10C5A00009F078C080910D1010920D1081115EC0BD
:10C5B00071C00F94AA89E12C10ECF12E09E714E464
:10C5C00020E030E040E85FE363E87BE08BE292E16B
:10C5D0000F940E8980912E10811176C0809188026F
:10C5E000882309F446CF11E080911210843009F0BD
:10C5F00010E06091830B7091840B8091850B90917A
:10C60000860B0E949F6E00E09C014BE252E12DCF11
:10C610000F94AA89E12C10ECF12E09E714E420E034
:10C6200030E0A90163E97BE086E292E10F940E8994
:10C6300080912E10811148C080918802882309F4CE
:10C6400018CF11E080911210853009F010E0609150
:10C65000930B7091940B8091950B9091960B0E9487
:10C660009F6E00E09C0146E252E1FFCE0F94AA8942
:10C67000E12C10ECF12E09E714E420E030E0A901F0
:10C6800067E97BE08CE192E10F940E8980912E1096
:10C6900081111AC080918802882309F4EACE11E042
:10C6A00080911210863009F010E06091970B709124
:10C6B000980B8091990B90919A0B0E949F6E00E0CD
:10C6C0009C014CE152E1D1CEDF91CF911F910F91AE
:10C6D000FF90EF9008950C94198E0C94198E0C9481
:10C6E000198E0C94198E6F927F928F929F92AF92B7
:10C6F000BF92CF92DF92EF92FF920F931F93CF934F
:10C70000DF9361E081E00E94F46ED0911310C0E0ED
:10C7100077247A94E3E06E2ED1110BC08091121031
:10C72000811129C080910D1010920D1081111DC032
:10C7300022C0D13059F4909112109130C1F58091FE
:10C740000D1010920D10811127C031C0D23009F0A8
:10C750009FC080911210823009F0CBC080910D10E3
:10C7600010920D108111B4C0C4C00E94EE6F809170
:10C770002E10811191C380918802882361F181E09C
:10C7800090911210911180E003E023E040EE50E11F
:10C790006C2F0E940E761FC08091F70E8D2780931C
:10C7A000F70E6092880280912E10811175C38091DE
:10C7B0008802882381F081E0913009F080E0909137
:10C7C000F70E911173C02DE83EE301E043E152E121
:10C7D0006C2F0E9487752CEA35EC47E25EE360918E
:10C7E00016117091171180911811909119110F94D1
:10C7F000C6B960935103709352038093530390938F
:10C8000054032CEA35EC47E25EE360911A11709113
:10C810001B1180911C1190911D110F942EB26093E9
:10C820004D0370934E0380934F0390935003D53084
:10C8300071F41092111080911210853009F0FBC034
:10C8400080910D1010920D108111E7C0F4C0D63008
:10C8500071F41092111080911210863009F0D0C13D
:10C8600080910D1010920D108111B1C1C9C1D73046
:10C8700009F027C11092111080911210873009F031
:10C88000E7C180910D1010920D108111D3C1E0C14C
:10C89000D33079F480911210833009F055C0809123
:10C8A0000D1010920D1081113EC04EC021E93EE3E3
:10C8B0008CCFD43009F08FCF80911210843009F0E2
:10C8C00090C080910D1010920D1081115BC089C035
:10C8D000E12CF12C02E813E420E030E0A9016DE343
:10C8E00072E08CE092E10F940E8980912E108111FC
:10C8F000D3C280918802882309F46DCF11E0809122
:10C900001210823009F010E060913D0270913E02F9
:10C9100080913F02909140020E949F6E00E09C0136
:10C920004CE052E12AC0E12CF12C02E813E420E0B3
:10C9300030E0A90169E372E085E092E10F940E898D
:10C9400080912E108111A8C280918802882309F459
:10C9500042CF11E080911210833009F010E0609115
:10C96000390270913A0280913B0290913C020E9400
:10C970009F6E00E09C0145E052E16C2F812F0E94E8
:10C98000877573C020E030E048EC52E460913502D6
:10C990007091360280913702909138020F942EB236
:10C9A00020E030E0A9010F94CCB80F943FBA812C5D
:10C9B000912C41EDA42E44ECB42E6B0118EEE12E27
:10C9C00013E0F12E00E010E020E030E0A90165E383
:10C9D00072E08DEF91E10F949E8880912E1081116D
:10C9E0005BC280918802882309F43FC011E08091E6
:10C9F0001210843009F010E0609135027091360217
:10CA000080913702909138020E94BB6D00E09C013A
:10CA10004DEF51E16C2F812FDCCE0F94AA8940E0BD
:10CA200050E062E171E185EF91E10F94C1A980913D
:10CA30002E10811131C280918802882309F463C0CD
:10CA400011E080911210853009F010E06091121110
:10CA50007091131180911411909115110E94AF6B78
:10CA600000E09C0145EF51E14AC02CEA35EC47E279
:10CA70005EE36091161170911711809118119091D9
:10CA800019110F94C6B960935103709352038093A8
:10CA90005303909354032CEA35EC47E25EE3609134
:10CAA0001A1170911B1180911C1190911D110F94FE
:10CAB0002EB260934D0370934E0380934F03909377
:10CAC0005003D83001F51092111080911210883067
:10CAD00009F476C080918802882309F451C111E0DD
:10CAE00080911210883009F010E080910C02909132
:10CAF0000D020F949E4D00E09C0146ED51E16C2F1C
:10CB0000812F0E9487752CEA35EC47E25EE3609145
:10CB10000B0F70910C0F80910D0F90910E0F0F94D1
:10CB2000C6B960935103709352038093530390935B
:10CB300054032CEA35EC47E25EE360910F0F7091ED
:10CB4000100F8091110F9091120F0F942EB26093DD
:10CB50004D0370934E0380934F0390935003D9304D
:10CB600071F47092111080911210893009F0B0C0E8
:10CB700080910D1010920D1081119CC0A9C0DA3067
:10CB800071F470921110809112108A3009F0D3C0A4
:10CB900080910D1010920D108111B4C0CCC0DB300B
:10CBA00009F01AC170921110809112108B3009F0A7
:10CBB00031C180910D1010920D1081111DC12AC13B
:10CBC00080910D1010920D10811160C083CF0F94D1
:10CBD000AA8921ECC22E2AE6D22EE12C18E1F12EF0
:10CBE0000CE116E42AE037ED43E25CE361E573E033
:10CBF0008DEE91E10F94C3A880912E1081114CC14C
:10CC000080918802882309F47ECF11E08091121070
:10CC1000863009F010E060915103709152038091C9
:10CC20005303909154030E94F76A00E09C014DEE7B
:10CC300051E127C00F94AA894AEA5AE66DE473E0ED
:10CC400085EE91E10F94C1A980912E10811124C12C
:10CC500080918802882309F456CF11E08091121048
:10CC6000873009F010E060914D0370914E03809180
:10CC70004F03909150030E94AF6B00E09C0145EE82
:10CC800051E16C2F812F0E9487757AC00F94AA8979
:10CC90000CED1FE624E031E046E950E06CE072E084
:10CCA00086ED91E10F94B68980912E10882309F4C6
:10CCB00011CFF2C00F94AA8940E050E067E07FE016
:10CCC00085EF91E10F94C1A980912E108111E4C0EC
:10CCD00080918802882309F44AC011E080911210E3
:10CCE000893009F010E06091070F7091080F809172
:10CCF000090F90910A0F0E94AF6B00E09C0145EF75
:10CD000051E131C00F94AA8983E9C82E8AE6D82E52
:10CD1000E12C18E1F12E0CE116E42AE037ED43E2B4
:10CD20005CE361E573E08DEE91E10F94C3A880911F
:10CD30002E108111B1C0809188028823C1F011E0CA
:10CD4000809112108A3009F010E0609151037091C7
:10CD5000520380915303909154030E94F76A00E0BC
:10CD60009C014DEE51E16C2F812F0E948775CF5FA2
:10CD7000DF5FC43009F0D0CC8DE080930E108CC002
:10CD80002CEA35EC47E25EE360910B0F70910C0FDB
:10CD900080910D0F90910E0F0F94C6B960935103BF
:10CDA0007093520380935303909354032CEA35EC11
:10CDB00047E25EE360910F0F7091100F8091110FA9
:10CDC0009091120F0F942EB260934D0370934E0307
:10CDD00080934F0390935003DC3049F6709211100A
:10CDE000809112108C3009F041C080910D1010928A
:10CDF0000D10811129C03AC00F94AA894CE75AE658
:10CE00006DE473E085EE91E10F94C1A980912E103D
:10CE1000811142C080918802882309F4A8CF11E0D3
:10CE2000809112108B3009F010E060914D037091E9
:10CE30004E0380914F03909150030E94AF6B00E02E
:10CE40009C0145EE51E18FCF0F94AA890BE517E6BF
:10CE50002CE830E04CE350E06AE072E086ED91E1CE
:10CE60000F94B68980912E10811116C0809188028E
:10CE7000882309F47CCF11E0809112108C3009F0E6
:10CE800010E080910A0290910B020F949E4D00E0F9
:10CE90009C0146ED51E167CFDF91CF911F910F913A
:10CEA000FF90EF90DF90CF90BF90AF909F908F90CA
:10CEB0007F906F9008958FEF9FEF0C949E6F4F922D
:10CEC0005F926F927F928F929F92AF92BF92CF921A
:10CED000DF92EF92FF920F931F93CF93DF9300D0D7
:10CEE00000D0CDB7DEB7C090570BD090580BE09074
:10CEF000590BF0905A0B80915B0B90915C0BA091B9
:10CF00005D0BB0915E0B8C159D05AE05BF0510F451
:10CF1000D701C601C090530BD090540BE090550B35
:10CF2000F090560BBC01CD016C157D058E059F055B
:10CF300010F4C701B6010F94CDB12B013C0161E0A3
:10CF400081E00E94F46E209113102E831D828E8149
:10CF500081110BC08091121081112CC080910D1095
:10CF600010920D10811120C025C02E81213061F456
:10CF700080911210813009F08DC080910D101092B7
:10CF80000D10811129C086C08E81823009F0ABC09E
:10CF900080911210823009F01FC180910D10109203
:10CFA0000D108111BFC018C10E94EE6F80912E102C
:10CFB00081118BC280918802882309F487C081E0A7
:10CFC00090911210911180E003E023E040EE50E1D7
:10CFD0006D810E940E767AC00F94AA892AE037EDFF
:10CFE00043E25DE3C301B2010F942EB220E030E0D2
:10CFF000A9010F94CCB84B015C0120E030E040E087
:10D000005FE40F94C8B187FD05C0812C912CA12C41
:10D010005FE4B52E2AE037ED43E25DE36091870BD4
:10D020007091880B8091890B90918A0B0F942EB28E
:10D0300020E030E0A9010F94CCB820E030E040E8D7
:10D040005FE30F94CBB80F943FBA69837A838B83E5
:10D050009C83C501B4010F9438BA7B018C0121E097
:10D06000E21AF10801091109812C912C49EBA42E37
:10D0700044ECB42EC980DA8021E030E040E050E09A
:10D0800067E87BE086E792E10F949E8880912E10FE
:10D0900081111BC2809188028823C1F011E0809128
:10D0A0001210813009F010E06091870B7091880BAD
:10D0B0008091890B90918A0B0E94556D00E09C0134
:10D0C00046E752E16D81812F0E9487758D818F5FC8
:10D0D0008D832E812F5F2E83843009F038CF88E036
:10D0E00080930E10F2C18E81833061F48091121012
:10D0F000833009F0F9C080910D1010920D1081114C
:10D1000095C0F2C02E81243009F080C080911210A9
:10D11000843009F024C180910D1010920D108111FE
:10D120000CC11DC10F94AA8960915F0B7091600BB7
:10D130008091610B9091620B0F94CDB120E030E0B3
:10D14000A9010F94CCB84B015C0120E030E040E035
:10D150005FE40F94C8B187FD05C0812C912CA12CF0
:10D160003FE4B32E20E030E0A90160918B0B709179
:10D170008C0B80918D0B90918E0B0F94CCB820E08E
:10D1800030E048EC52E40F94CBB80F943FBA698377
:10D190007A838B839C83C501B4010F9438BA7B01D9
:10D1A0008C0124E6E21AF10801091109812C912C65
:10D1B00023EBA22E24ECB22EC980DA8024E630E0E4
:10D1C00040E050E06BE87BE08CE692E10F949E88B3
:10D1D00080912E10811179C180918802882309F4F1
:10D1E00075CF11E080911210823009F010E060914B
:10D1F0008B0B70918C0B80918D0B90918E0B0E94FC
:10D20000556D00E09C014CE652E15CCF8E8185308B
:10D2100009F084C080911210853009F0DEC0809141
:10D220000D1010920D108111C6C0D7C00F94AA899D
:10D230002AE037ED43E25DE3C301B2010F942EB261
:10D2400020E030E0A9010F94CCB84B015C0120E054
:10D2500030E040E05FE40F94C8B187FD05C0812C49
:10D26000912CA12C9FE4B92E2AE037ED43E25DE337
:10D2700060918F0B7091900B8091910B9091920B1C
:10D280000F942EB220E030E0A9010F94CCB820E03A
:10D2900030E040E85FE30F94CBB80F943FBA698366
:10D2A0007A838B839C83C501B4010F9438BA7B01C8
:10D2B0008C0121E0E21AF10801091109812C912C5D
:10D2C00089EBA82E84ECB82EC980DA8021E030E00A
:10D2D00040E050E06FE87BE083E692E10F949E88A7
:10D2E00080912E108111F1C080918802882309F469
:10D2F000EDCE11E080911210833009F010E06091C2
:10D300008F0B7091900B8091910B9091920B0E94DA
:10D31000556D00E09C0143E652E1D4CE2E812630CB
:10D32000D1F580911210863009F085C080910D10E2
:10D3300010920D1081116DC07EC00F94AA890BE66A
:10D3400013E624E630E040E050E063E57BE08CE566
:10D3500092E10F9443A880912E108111B6C0809164
:10D360008802882309F4B2CE11E080911210843033
:10D3700009F010E06091530B7091540B8091550BA4
:10D380009091560B0F94CDB10E94DE6A00E09C0193
:10D390004CE552E197CE8E81873009F097CE80918F
:10D3A0001210873009F075C080910D1010920D1089
:10D3B00081115DC06EC00F94AA8901E713E624E6CF
:10D3C00030E040E050E067E57BE085E592E10F94D6
:10D3D00043A880912E10811178C080918802882303
:10D3E00009F474CE11E080911210853009F010E03C
:10D3F0006091570B7091580B8091590B90915A0B7B
:10D400000F94CDB10E94DE6A00E09C0145E552E137
:10D4100059CE0F94AA890FE613E62AE030E040E0E7
:10D4200050E06BE57BE08EE492E10F9443A880919D
:10D430002E1081114AC080918802882309F446CEBB
:10D4400011E080911210863009F010E060915B0BC2
:10D4500070915C0B80915D0B90915E0B0F94CDB140
:10D460000E94DE6A00E09C014EE452E12BCE0F9454
:10D47000AA890DE613E624E630E040E050E06FE5CF
:10D480007BE087E492E10F9443A880912E108111F4
:10D490001CC080918802882309F418CE11E0809185
:10D4A0001210873009F010E060915F0B7091600BF3
:10D4B0008091610B9091620B0F94CDB10E94DE6A56
:10D4C00000E09C0147E452E1FDCD26960FB6F894AA
:10D4D000DEBF0FBECDBFDF91CF911F910F91FF90A7
:10D4E000EF90DF90CF90BF90AF909F908F907F9004
:10D4F0006F905F904F9008952CEA35EC47E25EE321
:10D5000060914D0370914E0380914F0390915003B1
:10D510000F94C6B960931A1170931B1180931C115C
:10D5200090931D1108952CEA35EC47E25EE360917B
:10D5300051037091520380915303909154030F94BF
:10D540002EB2609316117093171180931811909357
:10D55000191108952CEA35EC47E25EE360914D0322
:10D5600070914E0380914F03909150030F94C6B970
:10D5700060931A1170931B1180931C1190931D11CD
:10D5800008952CEA35EC47E25EE360915103709117
:10D59000520380915303909154030F942EB26093E1
:10D5A0001611709317118093181190931911089503
:10D5B000FC0184910895FC0180810895CF93DF934D
:10D5C00000D01F92CDB7DEB70F943FBA0F94CDB104
:10D5D00069837A838B839C83CE0101960F94244BBD
:10D5E0000F900F900F900F90DF91CF9108958F9231
:10D5F0009F92AF92BF92CF92DF92EF92FF92CF9322
:10D600006B017C0120E030E0A9010F94C8B187FDD7
:10D6100005C06DEB77E386E095E304C06DEB77E33F
:10D6200086E095EBA70196010F94CCB86B017C01C5
:10D6300020E030E040E251E40F942EB220E030E0F0
:10D6400048EC52E40F942EB24B015C0120E030E034
:10D65000A901C701B6010F94C8B187FD05C020E03C
:10D6600030E040EA50E404C020E030E040EA50EC12
:10D67000C501B4010F94CCB820E030E040E251E4A1
:10D680000F94C6B90F9438BA6B017C0197FF0AC09A
:10D69000F094E094D094C094C11CD11CE11CF11C06
:10D6A0008DE201C08BE280932F10C701B60120E10B
:10D6B00037E240E050E00F9440B88AE0882E912C89
:10D6C000A12CB12CCA01B901A50194010F9440B855
:10D6D000605D60933010C701B60128EE33E040E092
:10D6E00050E00F9440B8CA01B901A50194010F940C
:10D6F00040B8605D60933110C701B60124E630E0A8
:10D7000040E050E00F9440B8CA01B901A50194016E
:10D710000F9440B8605D609332108EE280933310B6
:10D72000C701B601A50194010F9440B8C62FCA01E4
:10D73000B901A50194010F9440B8605D6093341065
:10D74000C05DC09335108FE290E1CF91FF90EF90D4
:10D75000DF90CF90BF90AF909F908F900895CF9221
:10D76000DF92EF92FF92CF93DF9300D01F92CDB75D
:10D77000DEB76B017C0120E030E0A9010F94C8B155
:10D7800087FD05C06DEB77E386E095E304C06DEBA4
:10D7900077E386E095EBA70196010F94CCB86983F7
:10D7A0007A838B839C83CE0101960F94D04B0F908C
:10D7B0000F900F900F90DF91CF91FF90EF90DF903F
:10D7C000CF9008958F929F92AF92BF92CF92DF92A7
:10D7D000EF92FF926B017C0120E030E0A9010F94F1
:10D7E000C8B187FD05C06DEB77E386E095E304C023
:10D7F0006DEB77E386E095EBA70196010F94CCB82B
:10D800006B017C0120E030E040E251E40F942EB245
:10D8100020E030E040E251E40F942EB24B015C0175
:10D8200020E030E0A901C701B6010F94C8B187FD1F
:10D8300005C020E030E040EA50E404C020E030E0E1
:10D8400040EA50ECC501B4010F94CCB820E030E0C0
:10D8500040E251E40F94C6B90F9438BA9B0177FFA8
:10D8600006C022273327261B370B8DE201C08BE22F
:10D8700080933110C90164E670E00F94AFB8CB011A
:10D88000EAE0F0E0BF010F94AFB8805D8093321002
:10D89000C901BF010F94AFB8282FCB01BF010F946E
:10D8A000AFB8805D809333108EE280933410205D9A
:10D8B0002093351081E390E1FF90EF90DF90CF90BF
:10D8C000BF90AF909F908F9008958F929F92AF924C
:10D8D000BF92CF92DF92EF92FF92CF936B017C01C8
:10D8E00020E030E0A9010F94C8B187FD05C06DEBC1
:10D8F00077E386E095E304C06DEB77E386E095EB94
:10D90000A70196010F94CCB86B017C0120E030E0B8
:10D91000A9010F94C8B187FF1BC0C701B601905879
:10D9200020E030E040E251E40F942EB220E030E0FD
:10D9300040E251E40F942EB24B015C0120E030E054
:10D94000A901C701B6010F9480BB1816FCF019C0DD
:10D9500020E030E040E251E4C701B6010F942EB25E
:10D9600020E030E040E251E40F942EB24B015C0124
:10D9700020E030E0A901C701B6010F94C8B187FDCE
:10D9800005C060E070E080EA90E404C060E070E010
:10D9900080EA90ECA50194010F94CCB820E030E02F
:10D9A00040E251E40F94C6B90F9438BA6B017C0180
:10D9B00080E280932F1080E1C81687E2D806E10448
:10D9C000F10494F0C701B60120E137E240E050E0F5
:10D9D0000F9440B8CA01B9012AE030E040E050E0BD
:10D9E0000F9440B8605D01C060E26093301088EE33
:10D9F000C81683E0D806E104F10494F0C701B6012B
:10DA000028EE33E040E050E00F9440B8CA01B9017D
:10DA10002AE030E040E050E00F9440B8605D01C083
:10DA200060E26093311084E6C816D104E104F10489
:10DA300094F0C701B60124E630E040E050E00F94D6
:10DA400040B8CA01B9012AE030E040E050E00F944C
:10DA500040B8605D01C060E2609332108AE0882EB9
:10DA6000912CA12CB12CC701B601A50194010F94F2
:10DA700040B8C62FCA01B901A50194010F9440B85E
:10DA8000605D609333108EE280933410C05DC0936C
:10DA900035108FE290E1CF91FF90EF90DF90CF9023
:10DAA000BF90AF909F908F900895CF92DF92EF92AA
:10DAB000FF92CF93DF9300D01F92CDB7DEB76B01FB
:10DAC0007C0120E030E0A9010F94C8B187FD05C0BA
:10DAD0006DEB77E386E095E304C06DEB77E386E0DA
:10DAE00095EBA70196010F94CCB869837A838B8359
:10DAF0009C83CE0101960F94244B0F900F900F90B2
:10DB00000F90DF91CF91FF90EF90DF90CF9008952D
:10DB1000CF92DF92EF92FF92CF93DF9300D01F92CC
:10DB2000CDB7DEB76B017C0120E030E0A9010F9496
:10DB3000C8B187FD05C06DEB77E386E095E304C0CF
:10DB40006DEB77E386E095EBA70196010F94CCB8D7
:10DB500069837A838B839C83CE0101960F9403881B
:10DB60000F900F900F900F90DF91CF91FF90EF905B
:10DB7000DF90CF9008958F929F92AF92BF92CF92F5
:10DB8000DF92EF92FF921F93CF93DF9300D01F920B
:10DB9000CDB7DEB76B017C0120E030E0A9010F9426
:10DBA000C8B187FD05C06DEB77E386E095E304C05F
:10DBB0006DEB77E386E095EBA70196010F94CCB867
:10DBC0006B017C0169837A838B839C8320E030E046
:10DBD00040E251EC0F94C8B1181654F420E030E044
:10DBE00048EC52E4C701B6010F9480BB87FD05C025
:10DBF000CE0101960F944E4C92C020E030E040E2FE
:10DC000051E4C701B6010F942EB220E030E048EC99
:10DC100052E40F942EB24B015C0120E030E0A901E8
:10DC2000C701B6010F94C8B187FD05C020E030E000
:10DC300040EA50E404C020E030E040EA50ECC50186
:10DC4000B4010F94CCB820E030E040E251E40F94EE
:10DC5000C6B90F9438BA4B015C0120E030E0A9014D
:10DC6000C701B6010F9480BB87FD0AC020E030E0F9
:10DC700040E251E4C701B6010F94C8B187FD1EC050
:10DC8000B7FC12C0C501B40128EE33E040E050E01B
:10DC90000F9440B8CA01B9012AE030E040E050E0FA
:10DCA0000F9440B8605D0BC0B094A09490948094A1
:10DCB000811C911CA11CB11C6DE201C060E260934B
:10DCC0003110C501B40124E630E040E050E00F948B
:10DCD00040B88AE0C82ED12CE12CF12CCA01B90140
:10DCE000A70196010F9440B8605D609332108EE2F8
:10DCF00080933310C501B401A70196010F9440B879
:10DD0000162FCA01B901A70196010F9440B8605DB2
:10DD100060933410105D1093351081E390E10F9003
:10DD20000F900F900F90DF91CF911F91FF90EF9088
:10DD3000DF90CF90BF90AF909F908F900895CF923B
:10DD4000DF92EF92FF926B017C0120E030E0A901AD
:10DD50000F94C8B187FD05C06DEB77E386E095E3CE
:10DD600004C06DEB77E386E095EBA70196010F9475
:10DD7000CCB86B017C0120E030E0A9010F94C8B160
:10DD800087FD05C020E030E040E05FE304C020E014
:10DD900030E040E05FEBC701B6010F94CCB80F94C0
:10DDA00038BACB01FF90EF90DF90CF900D949E4D4D
:10DDB0004FE350E0BC0186E59CE00D94E6BD63E9CD
:10DDC00072E084E690E00F9432836AEB72E084E6BE
:10DDD00090E00D94328381110C94DF6E68EB71E05A
:10DDE00084E190E00D943283382F81E080938502A6
:10DDF00010921A1080911E1090911F10A091201067
:10DE0000B0912110B7FF08C010921E1010921F1081
:10DE1000109220101092211020911E1020931210A9
:10DE200010922E1080910E101816ECF4082E000C93
:10DE3000990B831B9109022E000C330B281739070D
:10DE400094F097FF02C080E090E080931210092EBA
:10DE5000000CAA0BBB0B80931E1090931F10A09375
:10DE60002010B0932110809112106623A9F0909198
:10DE70001310891714F48093131020911310022E9D
:10DE8000000C330B2D5F3F4F482F082E000C550B15
:10DE9000241735071CF483508093131008950F93B3
:10DEA0001F93522F2091FE133091FF13281739072B
:10DEB000D1F19093FF138093FE138B0120E030E0AB
:10DEC00000931E1010931F102093201030932110E8
:10DED0004093131050930E108954994731F41092C7
:10DEE000D00F1092BC041092850380E094E10F944F
:10DEF00031278091BC0481110BC081E02091FE1379
:10DF00003091FF132954394709F080E00E94EDA6B3
:10DF100082E08093880281E080932E108FEF8093BF
:10DF20008502109290031F910F91089520E040E028
:10DF300060E070E089E499E70C944F6F0F931F93B2
:10DF4000CF93DF93CDB7DEB76E970FB6F894DEBFF1
:10DF50000FBECDBF97FD08C0FC01EE0FFF1FE45FB1
:10DF6000FD4F2081318104C020910A0230910B02C3
:10DF70003F932F939F938F9386ED92E19F938F937F
:10DF80008E010F5F1F4F1F930F930F9460B1C80155
:10DF90000E94D86E0E94966F0FB6F894DEBF0FBE37
:10DFA000CDBF6E960FB6F894DEBF0FBECDBFDF912A
:10DFB000CF911F910F91089580911110082E000CA0
:10DFC000990B0C949E6F8091B4139091B513891B9B
:10DFD0008F7011F40C94488381E00895E0918503DB
:10DFE000EE2389F0E150E093850388E0E89FF0019B
:10DFF0001124EB5AFC4F6281738127814681808115
:10E0000091810C944F6F0C94966FE0918503E630EC
:10E0100010F581E08E0F8093850340911E10509182
:10E020001F10609120107091211090911310809119
:10E030000E1028E0E29FF0011124EB5AFC4F2091D2
:10E04000FE133091FF133183208342835383648313
:10E0500075839683878308952091880321110BC0CF
:10E06000009711F486EA92E19093870380938603E8
:10E0700081E0809388030E94057020E040E060E02A
:10E0800070E080EF97E70E944F6F81E08093D00FA0
:10E090000E94848E1092D00F0C94EE6FAF92BF92BC
:10E0A000CF92DF92EF92FF920F931F93CF93DF9364
:10E0B000EC015B018A01FB01199587FD05C090E029
:10E0C000A0E0B0E0219628C1982F907E903CC9F442
:10E0D0008F7190E0A0E0B0E06C017D0126E0CC0CF7
:10E0E000DD1CEE1CFF1C2A95D1F7CE010196F5012F
:10E0F00019958F73A7019601282BDA01C901229681
:10E100000BC1982F907F903E29F58F70C82ED12C8F
:10E11000E12CF12C86E0CC0CDD1CEE1CFF1C8A955A
:10E12000D1F7CE010196F50119958F73C82A96E0B3
:10E13000CC0CDD1CEE1CFF1C9A95D1F7CE0102968B
:10E14000F50119958F73A7019601282BDA01C901F2
:10E150002396E2C0982F987F903F91F58770C82E44
:10E16000D12CE12CF12CF6E0CC0CDD1CEE1CFF1CBC
:10E17000FA95D1F7CE010196F50119958F73C82A4A
:10E18000A6E0CC0CDD1CEE1CFF1CAA95D1F7CE013D
:10E190000296F50119958F73C82AB6E0CC0CDD1CE8
:10E1A000EE1CFF1CBA95D1F7CE010396F501199527
:10E1B0008F73A7019601282BDA01C9012496ACC000
:10E1C000982F9C7F983F09F03FC08370C82ED12CB8
:10E1D000E12CF12C56E0CC0CDD1CEE1CFF1C5A95FA
:10E1E000D1F7CE010196F50119958F73C82A66E023
:10E1F000CC0CDD1CEE1CFF1C6A95D1F7CE010296FB
:10E20000F50119958F73C82A76E0CC0CDD1CEE1C45
:10E21000FF1C7A95D1F7CE010396F50119958F73FE
:10E22000C82AE6E0CC0CDD1CEE1CFF1CEA95D1F7F9
:10E23000CE010496F50119958F73A7019601282B3D
:10E24000DA01C901259668C0982F9E7F9C3F09F08E
:10E250004CC08170C82ED12CE12CF12C86E0CC0C66
:10E26000DD1CEE1CFF1C8A95D1F7CE010196F5014D
:10E2700019958F73C82A96E0CC0CDD1CEE1CFF1C90
:10E280009A95D1F7CE010296F50119958F73C82A98
:10E2900026E0CC0CDD1CEE1CFF1C2A95D1F7CE012C
:10E2A0000396F50119958F73C82A36E0CC0CDD1C56
:10E2B000EE1CFF1C3A95D1F7CE010496F501199595
:10E2C0008F73C82A46E0CC0CDD1CEE1CFF1C4A955F
:10E2D000D1F7CE010596F50119958F73A701960127
:10E2E000282BDA01C901269617C0982F907C903808
:10E2F00041F4807C803869F42196CE01F5011995AE
:10E30000F8CF8E7F8D3F28F02196CE01F50119952B
:10E31000F8CF80E090E0DC010115110529F0F8014B
:10E3200080839183A283B383CE01DF91CF911F912C
:10E330000F91FF90EF90DF90CF90BF90AF90089536
:10E34000AF92BF92CF92DF92EF92FF920F931F9303
:10E35000CF93DF9300D01F92CDB7DEB7062F5A01BF
:10E36000122F6E3F29F43CE9C32E32E1D32E04C0B4
:10E370002AE4C22E25E2D22EF82EE92E11160CF038
:10E3800090C0AE014F5F5F4F68ED7AE68F2D9E2DF6
:10E390000E944E70F82EE92E69817A818B819C81D2
:10E3A000611571058105910509F47BC06D33710517
:10E3B0008105910509F45AC06E37710581059105F3
:10E3C00009F454C06A32710581059105B9F06432CF
:10E3D00071058105910571F4A114B10459F0412F23
:10E3E000012E000C550B68ED7AE6C5010E9454A77A
:10E3F000181BC4CF0E9450A71150C0CF07FD38C0D2
:10E4000065E470E080E090E00E9450A7115009F4AC
:10E4100047C061E089819A81AB81BC81CD97A1051C
:10E42000B10509F460E0862F800F8A3094F06AE02D
:10E430000F948DB8092F682F880F770B605D7F4F81
:10E44000072E000C880B990B0E9450A7115041F128
:10E45000802F682F880F770B605D7F4F072E000C91
:10E46000880B990B0E9450A711500CC007FFD1CF09
:10E47000412F012E000C550B68ED7AE6C6010E9473
:10E4800054A7181B112361F0412F012E000C550BCE
:10E4900068ED7AE68F2D9E2D0E9454A7181B01C0AF
:10E4A00010E0812F0F900F900F900F90DF91CF9180
:10E4B0001F910F91FF90EF90DF90CF90BF90AF90A2
:10E4C00008951F93CF93DF9300D01F92CDB7DEB78F
:10E4D00010E0AE014F5F5F4F68ED7AE60E944E702C
:10E4E00049815A816B817C81452B462B472B11F04A
:10E4F0001F5FEFCF812F0F900F900F900F90DF9144
:10E50000CF911F9108952F923F924F925F926F92F9
:10E510007F928F929F92AF92BF92CF92DF92EF92B3
:10E52000FF920F931F93CF93DF9300D0CDB7DEB749
:10E530004C013B015A012B83232E280181E080935B
:10E54000850240911E1050911F1060912010709113
:10E550002110411551056105710571F0141615065C
:10E560000CF080E08093900310921E1010921F1008
:10E5700010922010109221101091900330900D10E5
:10E5800010920D10311005C080918802882309F483
:10E59000AFC0C2010E946172082FC114D10409F4F6
:10E5A000A5C0C6010E9461721A821982E114F104A9
:10E5B000B1F4402F50E0282F30E0CA01820F931FA2
:10E5C00045976CF484E190E0841B950B821B930BC0
:10E5D00097FD0196959587958A8381E0898301E06F
:10E5E00028ED3AE6A201BE016F5F7F4FCE01029691
:10E5F0000E94F37DE114F10491F08A81882321F0D7
:10E600001A8289818F5F898300E02BED3AE6A701AA
:10E61000BE016F5F7F4FCE0102960E94F37DC11451
:10E62000D10459F000E028ED3AE6A601BE016F5F83
:10E630007F4FCE0102960E94F37D63E080E00E944E
:10E64000FBA7111105C06BE570E080E090E004C00D
:10E6500060E270E080E090E00E9450A7C3010E9459
:10E66000F5A7111105C06DE570E080E090E004C0F1
:10E6700060E270E080E090E00E9450A7C4010E9438
:10E68000617263E092E1981B892F0E94FBA7111130
:10E6900005C060E270E080E090E004C06BE570E0EF
:10E6A00080E090E00E9450A7C4010E94F5A71111DC
:10E6B00005C060E270E080E090E004C06DE570E0CD
:10E6C00080E090E00E9450A7332061F0111102C059
:10E6D000AB80B22CA114B10419F0F501199502C058
:10E6E0000E94EE6F81E08093D00F02C080E05CCF8B
:10E6F0000F900F900F90DF91CF911F910F91FF908E
:10E70000EF90DF90CF90BF90AF909F908F907F90D1
:10E710006F905F904F903F902F9008951F93CF93ED
:10E72000DF9300D01F92CDB7DEB710E0AE014F5F90
:10E730005F4F6BED7AE60E944E7049815A816B8182
:10E740007C81452B462B472B11F01F5FEFCF812F8C
:10E750000F900F900F900F90DF91CF911F91089520
:10E760006F927F928F929F92AF92CF92EF920F9380
:10E770001F93CF93DF93DC013B01F901EB0119817A
:10E78000EA01898190E0811B910901962881EB01C2
:10E790003881622F70E0631B71096F5F7F4F111129
:10E7A00033C0102F137081F161307105B9F42081ED
:10E7B000321719F02FEF2C9327C0128188248394ED
:10E7C000912C153008F59401012E01C0220F0A94F6
:10E7D000EAF73C91232B2C931F5FF3CF00FDEACF88
:10E7E00030812313E7CF128188248394912C153034
:10E7F00058F49401012E01C0220F0A94EAF73C91CB
:10E80000232B2C931F5FF3CF202F2570C1F0E30142
:10E810002881211114C039812181321302C09380D3
:10E8200002C028E0922E8A2E9D01122F1819191568
:10E8300030F4E9011881106119939E01F6CF8130FF
:10E840009105F9F4E3019981818198133FC061300A
:10E85000710531F498818081981306C0848105C0C8
:10E8600001FF02C0EA01F6CF81E0803278F59381A2
:10E870009D01290F311DE9019881982B9883880FFC
:10E88000F4CF029719F5802F8C7001F1EA0199817C
:10E89000818198131BC06130710539F4E3019881BF
:10E8A0008081981306C0848105C003FF02C0EA017D
:10E8B000F6CF81E0803250F493819D01290F311D04
:10E8C000E9019881982B9883880FF4CFEA01888119
:10E8D000908189131AC0E3019881891711F00A7099
:10E8E000A1F0E30199818181981302C0938101C055
:10E8F00098E03A2FCA2FDB2F8C2F831B891728F41F
:10E9000028818481822B8993F7CFBD018E2D0F94AE
:10E91000F2952E2DEE0C330B440B550B6A2D8C2DDE
:10E92000DF91CF911F910F91EF90CF90AF909F907B
:10E930008F907F906F900C9416A8CF92DF92FF92E9
:10E940000F931F93CF93DF938C01EB018FEF809395
:10E950008502C0900F10D0901010F090111061E05F
:10E9600080E00E94FBA723E1A6016F2DC8010E9451
:10E97000A071182F209719F16AE370E080E090E011
:10E980000E9450A7CE010E948E738F5F11501817FE
:10E9900010F061E001C062E020E230E040E050E0D1
:10E9A00094E1981B892F0E9416A8CE01DF91CF9188
:10E9B0001F910F91FF90DF90CF900C9497A7DF915C
:10E9C000CF911F910F91FF90DF90CF9008950F93FB
:10E9D0001F93CF93DF93FC01EB0180911E10909168
:10E9E0001F10A0912010B0912110B7FF08C0109205
:10E9F0001E1010921F101092201010922110809162
:10EA0000221090912310A0912410B09125104091D4
:10EA10001E1050911F1060912010709121108417CA
:10EA20009507A607B70744F480931E1090931F1014
:10EA3000A0932010B093211080918802882301F1C7
:10EA400040911E1050911F10609120107091211064
:10EA50008091261090912710A0912810B091291034
:10EA60008A019B01080F191F2A1F3B1FC901B8010A
:10EA70001995BC0180912C1090912D100E949D74CD
:10EA800080910D10811108C080911B108823D1F155
:10EA9000809188028823B1F180912A1090912B10E7
:10EAA0000097B1F000911E1010911F1020912010BE
:10EAB000309121104091261050912710609128101C
:10EAC00070912910400F511F621F731FFE0119958D
:10EAD000E0911C10F0911D10309741F080911B10B7
:10EAE000811103C080910D108111199580910D1035
:10EAF00010920D10882331F0DF91CF911F910F916B
:10EB00000C94EE6FDF91CF911F910F910895CF92EA
:10EB1000DF92EF92FF920F931F93CF93DF93C82E54
:10EB2000162F7A01E901209709F44EC0C90100238C
:10EB300019F00E94617202C00E948E73D82EC1101B
:10EB400005C020E230E040E050E004C02EE330E0B9
:10EB500040E050E0612F80E00E9416A822E12D19CC
:10EB600040910F105091101060911110C7010E9438
:10EB7000A071182FDD2009F448C06AE370E080E03E
:10EB800090E00E9450A7112341F060E270E080E025
:10EB900090E00E9450A71150F6CFCE01002351F013
:10EBA000DF91CF911F910F91FF90EF90DF90CF9069
:10EBB0000C94F5A7DF91CF911F910F91FF90EF90EB
:10EBC000DF90CF900C9497A7882329F02EE330E0B4
:10EBD00040E050E004C020E230E040E050E0612F2F
:10EBE00080E00E9416A840910F105091101022E171
:10EBF00060911110C701DF91CF911F910F91FF908C
:10EC0000EF90DF90CF900C94A071DF91CF911F9186
:10EC10000F91FF90EF90DF90CF9008950F93CF93D7
:10EC2000DF93EA01882331F0022E000C330B440BF2
:10EC3000550B04C020E230E040E050E080E00E944C
:10EC400016A840910F105091101022E16091111000
:10EC5000CE010E94A071C82FCC2341F060E270E089
:10EC600080E090E00E9450A7C150F6CF602F000FC7
:10EC7000770B880B990BDF91CF910F910C9450A7D4
:10EC8000AF92BF92CF92DF92EF92FF920F931F93BA
:10EC9000CF93DF9361E081E00E94F46EC091131086
:10ECA000B12C43E0A42EC1110BC080911210811130
:10ECB0001BC080910D1010920D1081110FC014C057
:10ECC000C13011F580911210813009F0C0C08091DF
:10ECD0000D1010920D108111ADC0B9C00E94EE6FE1
:10ECE00080912E10811104C180918802882361F0E7
:10ECF00081E090911210911180E003E023E040EE5A
:10ED000050E16B2D0E940E768091F610882371F0F1
:10ED1000C23071F480911210823009F0CBC0809122
:10ED20000D1010920D108111ADC0C4C0D2E001C011
:10ED3000D3E0DC1339C0809112108D131AC080917A
:10ED40000D1010920D108823A1F00F94AA89E12CC8
:10ED500010E8F12E0BE314E420E030E0A9016CE9A7
:10ED600070E188EB92E10F940E8980912E10811151
:10ED7000BFC0809188028823B9F011E08091121001
:10ED80008C1310E060919C1070919D1080919E10EA
:10ED900090919F100E949F6E00E09C0148EB52E111
:10EDA0006B2D812F0E94877581E08D0F8C1339C0E8
:10EDB000809112108C131AC080910D1010920D10BA
:10EDC0008823A1F00F94AA89E12C10E8F12E0BE31F
:10EDD00014E420E030E0A90160EA70E180EB92E108
:10EDE0000F940E8980912E10811182C0809188022B
:10EDF0008823B9F011E0809112108C1310E060911B
:10EE0000A0107091A1108091A2109091A3100E9467
:10EE10009F6E00E09C0140EB52E16B2D812F0E9420
:10EE20008775B394CF5F84E0B8123DCFDE5FD09397
:10EE30000E105EC08091F6108C278093F610A09281
:10EE400088020E94828D80912E10811151C0809184
:10EE50008802882309F458CF81E0909112109130F4
:10EE600009F080E09091F610911103C02DE83EE387
:10EE700002C021E93EE301E04CEC52E16B2D0E941F
:10EE8000877542CF0F94AA8922E8C22E2DE8D22E90
:10EE9000E12CF12C00E510E420E030E040EC5FE3F1
:10EEA00062EF70E182EC92E10F940BAA80912E1038
:10EEB00081111EC0809188028823C1F0D1E0809129
:10EEC0001210823009F0D0E06091F2107091F310CE
:10EED0008091F4109091F5100E94886D00E09C01E3
:10EEE00042EC52E16B2D8D2F0E948775D3E05CCFF1
:10EEF000DF91CF911F910F91FF90EF90DF90CF9016
:10EF0000BF90AF900895CF92DF92EF92FF920F9350
:10EF10001F93CF93DF937B01C42F8901682F80E07B
:10EF20000E94FBA7E114F10429F0C7010E9461725D
:10EF3000C82E01C0C12C0115110529F0C8010E947D
:10EF40008E73D82E01C0D12CC0FF1DC084E190E08B
:10EF50008C199109C7FC93958D199109D7FC93954C
:10EF600097FD019695958795C4E1DBEED80F8D2F1F
:10EF70008C0F87FD09C060E270E080E090E00E94A5
:10EF800050A7C150F4CFC4E1CC2059F040910F10EC
:10EF9000509110102C2F60911110C7010E94A07188
:10EFA000C82FDD2051F04C2F0C2E000C550B6BEDB3
:10EFB0007AE6C8010E9454A7C81B1C1644F460E2FC
:10EFC00070E080E090E00E9450A7C150F6CFDF9142
:10EFD000CF911F910F91FF90EF90DF90CF90089508
:10EFE00080918802882351F0609186037091870395
:10EFF00020E030E041E081E00C9483770895809137
:10F00000B4139091B513891B8F70B9F48091A90442
:10F010008770873051F01092A9041092A80486E0FE
:10F0200093E19093550C8093540C20E040E060E015
:10F0300070E089E49FE90C944F6F0895FC01A08172
:10F04000B1811C92A281B3818C918F5F8C930280DD
:10F05000F381E02D608180E00C94FBA70E949483F3
:10F06000882321F180912C1590912D15A0912E15BA
:10F07000B0912F150097A105B105C1F0BC01CD01DC
:10F080006D597F4F8F4F9F4F24E630E040E050E0B6
:10F090000F941EB860913015709131158091321522
:10F0A000909133150F941EB8822F089580E0089533
:10F0B000AF92BF92CF92DF92EF92FF920F93CF93D6
:10F0C000DF9361E081E00E94F46ED0911310C0E004
:10F0D0008DE1E82E83E1F82E94E3C92E93E1D92E39
:10F0E0002BE4A22E23E1B22ED1110BC0809112107D
:10F0F000811129C080910D1010920D1081111DC039
:10F1000022C0D13059F490911210913091F5809134
:10F110000D1010920D10811124C02BC0D23009F0B7
:10F120003FC090911210923009F04FC080910D10A5
:10F1300010920D10811141C048C00E94EE6F809165
:10F140002E10811164C080918802882309F181E02A
:10F1500090911210911180E003E023E049E653E41E
:10F1600014C0B092550CA092540C80912E108111B5
:10F170004EC080918802882359F081E0913009F0D7
:10F1800080E000E22EE34BE353E16C2F0E940E7609
:10F19000CF5FDF5FC43009F0A7CFC0930E1037C038
:10F1A000D330B1F790911210933021F580910D106A
:10F1B00010920D10811116C01DC0D092550CC09236
:10F1C000540C80912E10811122C0809188028823D6
:10F1D000F9F281E0923009F080E000E22EE345E2AE
:10F1E00053E1D3CFF092550CE092540C80912E1045
:10F1F00081110DC080918802882351F281E0933003
:10F2000009F080E000E22EE34AE053E1BECFDF9157
:10F21000CF910F91FF90EF90DF90CF90BF90AF9084
:10F220000895CF92DF92EF92FF920F931F930F9466
:10F230002F8D0091920310919303209194033091AC
:10F2400095036B017C01C01AD10AE20AF30AF7FCAC
:10F2500013C020919103209520939103DC01CB01F1
:10F260008A549C4FAF4FBF4F809392039093930368
:10F27000A0939403B093950381E090919103911131
:10F2800001C080E01F910F91FF90EF90DF90CF9031
:10F2900008954F925F926F927F928F929F92AF925A
:10F2A000BF92CF92DF92EF92FF920F931F93CF9373
:10F2B000DF93CDB7DEB72E970FB6F894DEBF0FBE43
:10F2C000CDBF10921A100F942F8D00917A0F1091CC
:10F2D0007B0F20917C0F30917D0F6B017C01C01A58
:10F2E000D10AE20AF30A970186010858134121095D
:10F2F000310937FD08C060937A0F70937B0F8093BC
:10F300007C0F90937D0F80910D1010920D1088232B
:10F3100059F020E040E060E070E08AEC90E50E9467
:10F320004F6F0E943AA73BC420912D0230912E02CC
:10F3300040911E1050911F10C901840F951F243653
:10F34000310559F44730510514F0069722C04A3F61
:10F350005F4F0CF06CC006961CC0243631052CF4AF
:10F36000853691050CF063C004C08436910524F401
:10F370005EC08A3091053CF0883EE3E09E072CF0A9
:10F3800087EE93E002C08AE090E02817390731F455
:10F3900011C08A30910584F78AE090E090932E02A4
:10F3A00080932D0210921E1010921F1010922010A8
:10F3B000109221100E941179182F60E080E00E94C5
:10F3C000FBA780900B1190900C11A0900D11B090A4
:10F3D0000E1160910F1170911011072E000C880B07
:10F3E000990B0F94CFB16B017C0162E070E080E07B
:10F3F00090E00E9450A720E030E040E05FE3C501CC
:10F40000B4010F94CCB80F9438BACB010F949E4D31
:10F410000E9497A76FE270E080E090E00E9450A702
:10F42000111108C08091FB10811173C003C084E6E4
:10F4300090E0A2CF20E030E040E05FE3C701B601FA
:10F440000F94CCB80F9438BACB010F94734D0E942F
:10F4500097A761E070E080E090E00E9450A760E232
:10F4600070E080E090E00E9450A720E030E040E2B1
:10F4700051E4C701B6010F94C8B187FF06C060E22E
:10F4800070E080E090E00E9450A760E08AE00E9477
:10F49000FBA7112331F08091F110882311F00FE5C3
:10F4A00001C000E08090000F9090010FA090020F2B
:10F4B000B090030F6091040F7091050F072E000CA0
:10F4C000880B990B0F94CFB16B017C01602F000F5B
:10F4D000770B880B990B0E9450A720E030E040E0AA
:10F4E0005FE3C501B4010F94CCB80F9438BACB01D7
:10F4F0000F949E4D0E9497A76FE270E080E090E02D
:10F500000E9450A711112CC080910011811119C3C4
:10F5100027C060E270E080E090E00E9450A720E009
:10F5200030E040E251E4C701B6010F9480BB87FD93
:10F5300006C060E270E080E090E00E9450A720E00A
:10F5400030E048EC52E4C701B6010F9480BB87FD60
:10F5500080CF60E270E080E090E00E9450A779CF19
:10F5600020E030E040E05FE3C701B6010F94CCB883
:10F570000F9438BACB010F94734D0E9497A761E0A6
:10F5800070E080E090E00E9450A760E270E080E0D0
:10F5900090E00E9450A720E030E040E251E4C70133
:10F5A000B6010F94C8B187FF06C060E270E080E04A
:10F5B00090E00E9450A761E080E00E94FBA72091AC
:10F5C0005A0530915B0540915C0550915D05609155
:10F5D00053027091540280915502909156020F94FB
:10F5E000CCB86B017C0120915E0530915F054091A4
:10F5F00060055091610560915702709158028091A9
:10F60000590290915A020F94CCB84B015C0120E052
:10F6100030E0A901C701B6010F94C8B187FD05C04C
:10F6200020E030E040E05FE304C020E030E040E074
:10F630005FEBC701B6010F94CCB80F9438BACB0179
:10F640000F94F24CD82E092F68E570E080E090E02E
:10F650000E9450A711111AC08091A80480FD16C005
:10F66000ED2CF02EF70161917F01662399F06F3246
:10F6700034F4062E000C770B880B990B04C06FE353
:10F6800070E080E090E00E9450A7ECCF8D2D902F8D
:10F690000E9497A760E270E080E090E00E9450A78F
:10F6A00020E030E0A901C501B4010F94C8B187FD85
:10F6B00005C020E030E040E05FE304C020E030E03F
:10F6C00040E05FEBC501B4010F94CCB80F9438BA99
:10F6D000CB010F94F24CD82E092F69E570E080E041
:10F6E00090E00E9450A711111BC08091A80486953C
:10F6F00080FD16C0ED2CF02EF70161917F0166238D
:10F7000099F06F3234F4062E000C770B880B990BAE
:10F7100004C06FE370E080E090E00E9450A7ECCF5F
:10F720008D2D902F0E9497A761E08CE00E94FBA78F
:10F730002091620530916305409164055091650503
:10F7400060915B0270915C0280915D0290915E021B
:10F750000F94CCB86B017C0120E030E040E251E432
:10F760000F942EB220E030E048EC52E40F942EB219
:10F770004B015C0120E030E0A901C701B6010F9404
:10F78000C8B187FD05C020E030E040EA50E404C085
:10F7900020E030E040EA50ECC501B4010F94CCB851
:10F7A00020E030E040E251E40F94C6B90F9438BA3B
:10F7B0006B017C0197FF0AC0F094E094D094C09450
:10F7C000C11CD11CE11CF11C8DE201C080E28093C0
:10F7D0002F10F0E1CF16F7E2DF06E104F10494F018
:10F7E000C701B60120E137E240E050E00F9440B895
:10F7F000CA01B9012AE030E040E050E00F9440B87F
:10F80000605D01C060E26093301028EEC21623E014
:10F81000D206E104F10494F0C701B60128EE33E00A
:10F8200040E050E00F9440B8CA01B9012AE030E04E
:10F8300040E050E00F9440B8605D01C060E260932A
:10F840003110C701B60124E630E040E050E00F94EB
:10F8500040B86AE0862E912CA12CB12CCA01B901C6
:10F86000A50194010F9440B8605D60933210C70108
:10F87000B601A50194010F9440B8062F662381F0CC
:10F880008EE280933310CA01B901A50194010F944F
:10F8900040B8605D60933410005D0093351017C070
:10F8A000CA01B901A50194010F9440B8662339F04B
:10F8B0008EE280933310605D6093341005C080E267
:10F8C000809334108093331080E2809335106AE582
:10F8D00070E080E090E00E9450A7112329F08FE2B1
:10F8E00090E10E9497A71EC08091A80486958695F6
:10F8F00080FDF5CF9FE2E92E90E1F92EF7016191AD
:10F900007F01662379F06F3234F4062E000C770BFA
:10F91000880B990B04C06FE370E080E090E00E94D8
:10F9200050A7ECCF26E030E040E050E062E080E01D
:10F930000E9416A880912D0290912E020F949E4D48
:10F940000E9497A765E270E080E090E00E9450A7D7
:10F950000F94874A2B013C0120E13EE040E050E05B
:10F960000F941EB869017A018CE3882E912CA12C8A
:10F97000B12CC301B201A50194010F941EB8CA01B4
:10F98000B901A50194010F941EB89E012F5F3F4F4E
:10F99000590134E6C316D10498F47F936F93DF9234
:10F9A000CF9282E994E19F938F93BF92AF920F948D
:10F9B00060B10FB6F894DEBF0FBECDBF05E012C038
:10F9C0007F936F93DF92CF9288E894E19F938F9318
:10F9D000BF92AF920F9460B10FB6F894DEBF0FBE26
:10F9E000CDBF06E027E030E040E050E062E083E198
:10F9F000801B0E9416A8C5010E9497A762E08CE0B8
:10FA0000801B0E94FBA70E942E78082F8EE994E1AC
:10FA10000E94F5A7002331F0802F0F94464E0E94DC
:10FA200097A704C08AE19CE10E94F5A765E270E017
:10FA300080E090E00E9450A763E080E00E94FBA776
:10FA40000F942F8DC0907A0FD0907B0FE0907C0F99
:10FA5000F0907D0FDC01CB018C199D09AE09BF0927
:10FA6000885B9B40A109B109B7FF92C080917E0FCE
:10FA7000882309F48DC08EE79FE00E948E73082FC3
:10FA8000853178F48EE79FE00E9497A7043109F44E
:10FA900086C060E270E080E090E00E9450A70F5FB7
:10FAA000F5CFE090790F8E2D90E09C012258304FD9
:10FAB0007901C9010E948E73082F44E150E06BED7B
:10FAC0007AE6C7010E9454A70431C0F46EE270E0E8
:10FAD00080E090E00E9450A7033181F06EE270E078
:10FAE00080E090E00E9450A742E1401B39F050E0D6
:10FAF0006BED7AE68EE79FE00E9454A78091960313
:10FB0000181709F44CC0109396038EE79FE00E94EB
:10FB10008E739091790F981788F481E0890F21E016
:10FB2000280FE82FF0E0E258F04F9081907C903859
:10FB300011F4822FF4CF8093790F31C01092790F96
:10FB40002EC060E270E080E090E00E9450A720E0CC
:10FB500030E040E251E4C701B6010F9480BB87FD5D
:10FB600006C060E270E080E090E00E9450A720E0D4
:10FB700030E048EC52E4C701B6010F9480BB87FD2A
:10FB8000FECC60E270E080E090E00E9450A7F7CCED
:10FB90000E942E78833008F46ECF0E949DA72E9687
:10FBA0000FB6F894DEBF0FBECDBFDF91CF911F918E
:10FBB0000F91FF90EF90DF90CF90BF90AF909F900C
:10FBC0008F907F906F905F904F9008950E943AA71A
:10FBD0003E98469A3C98449A3A98429A0F946B847D
:10FBE0001092770F08954F925F926F927F929F923B
:10FBF000AF92BF92CF92DF92EF92FF920F931F933B
:10FC0000CF93DF93CDB7DEB728970FB6F894DEBF5A
:10FC10000FBECDBF7C013B016A015901FB01608130
:10FC2000FC0180810E94FBA7C114D10409F49AC091
:10FC3000FA82E9827C826B82011103C01C2D0D2D9A
:10FC400076C09D2C0C2D192DD12CAE014B5F5F4F32
:10FC5000B5018C2D992D0E944E70C82E992E4D8085
:10FC60005E806F8078844114510461047104C9F08E
:10FC7000F0E24F1651046104710481F0D301C20116
:10FC80008D97A109B1090297A105B10550F08BE24A
:10FC90004816510461047104B1F503C0DD2009F474
:10FCA0005AC0F70120818D2D90E0820F911D45975C
:10FCB00034F0253020F0CE0101960E941E7881E0BC
:10FCC000411451046104710409F480E0D80EF70175
:10FCD00080818D0D8083DD2081F0DA94AE014B5F51
:10FCE0005F4FB501C8010E944E708C016D817E810D
:10FCF0008F8198850E9450A7EECF45284628472837
:10FD000009F0A0CF2FC0D3940115110509F09DCFA4
:10FD10000C2D192D9ACF0E9450A7F70180818F5F7B
:10FD20008083843120F0CE0101960E941E78AE01BE
:10FD30004B5F5F4FB501812F902F0E944E70182F9F
:10FD4000092F6D817E818F819885611571058105EF
:10FD5000910509F707C00115110509F473CF0F5F6D
:10FD60001F4FD2CF28960FB6F894DEBF0FBECDBF7F
:10FD7000DF91CF911F910F91FF90EF90DF90CF9087
:10FD8000BF90AF909F907F906F905F904F9008953D
:10FD90000E945D3E882339F062E370E080E090E0ED
:10FDA0000E941883F5CF62E370E080E090E00C944D
:10FDB0001883CF93DF93EC010E94057020E040E0B0
:10FDC00060E070E0CE01DF91CF910C944F6F6F92A5
:10FDD0007F928F929F92AF92BF92CF92DF92EF92DB
:10FDE000FF920F93CF93DF9361E081E00E94F46E66
:10FDF000D0911310C0E088E1A82E84E1B82E9FEFC7
:10FE0000E92E97E7F92E25E4C22E24E1D22E3DE615
:10FE1000832E34E1932E42E8642E44E1742ED111F6
:10FE200020C08091121081110CC080910D10109291
:10FE30000D10882331F00E94EE6F80912E108111F9
:10FE40004DC180918802882361F081E09091121069
:10FE5000911180E003E023E04FEF52E16C2F0E940C
:10FE60000E768091F110882369F0D130C9F4909119
:10FE700012109130D1F580910D1010920D1081115A
:10FE80002CC033C0D13061F490911210913009F040
:10FE900041C080910D1010920D10811133C03AC0F5
:10FEA000D23061F480911210823009F053C08091F9
:10FEB0000D1010920D10811145C04CC0D33009F0C7
:10FEC00077C080911210833009F059C080910D10D5
:10FED00010920D1081114DC052C07092550C60925D
:10FEE000540C80912E108111F9C0809188028823D2
:10FEF00001F181E0913009F080E000E22EE343E778
:10FF000054E114C09092550C8092540C80912E10A4
:10FF10008111E4C080918802882359F081E09130FA
:10FF200009F080E000E22EE340E654E16C2F0E94ED
:10FF30000E76CF5FDF5FC43009F071CF88E0809329
:10FF40000E10CCC08CE790E80E94D97E80912E10D4
:10FF50008111C4C080918802882359F381E0909177
:10FF60001210923009F080E00EE32EE34FE454E1EA
:10FF7000DDCF0E94FF7780912E108111AFC080915C
:10FF800088028823B1F2FF92EF92DF92CF92CF9353
:10FF900081E090911210933009F080E08F930E94DD
:10FFA00021C60F900F900F900F900F900F90C1CF20
:10FFB000D43059F480911210843059F580910D108D
:10FFC00010920D1081111DC024C0D53061F48091B4
:10FFD0001210853009F044C080910D1010920D1060
:10FFE000811136C03DC0D63021F580911210863087
:10FFF00009F04EC080910D1010920D10811140C07B
:020000021000EC
:1000000047C08FEA9DE90E94D97E80912E10811110
:1000100065C080918802882309F48BCF81E090919C
:100020001210943009F080E00EE32EE348E354E12F
:100030007DCFD73009F07DCF90911210973009F025
:100040003FC080910D1010920D10811131C038C049
:1000500088E598E70E94D97E80912E1081113EC0DC
:1000600080918802882309F464CF81E09091121076
:10007000953009F080E00EE32EE348E254E156CFDC
:1000800080EF91E80E94D97E80912E10811126C0C8
:1000900080918802882309F44CCF81E0909112105E
:1000A000963009F080E00EE32EE34EE154E13ECFBE
:1000B000B092550CA092540C80912E1081110EC05C
:1000C00080918802882309F434CF81E0973009F0C9
:1000D00080E000E22EE348E054E128CFDF91CF91A9
:1000E0000F91FF90EF90DF90CF90BF90AF909F90D7
:1000F0008F907F906F9008954F925F926F927F9252
:100100008F929F92AF92BF92CF92DF92EF92FF9227
:100110000F931F93CF9361E081E00E94F46EC09132
:10012000131010E08AEA682E8DE9782E95E8492EA2
:1001300093E1592E26EEE22E22E1F22E36EEC32E68
:1001400032E1D32E4BEEA42E43E1B42E54EF852E94
:1001500052E1952EC1110BC080911210811128C05F
:1001600080910D1010920D1081111CC021C0C13062
:1001700059F490911210913091F580910D101092D8
:100180000D10811124C02BC0C230C9F590911210FE
:10019000923009F086C080910D1010920D108111DF
:1001A00078C07FC00E94EE6F80912E10811108C12F
:1001B00080918802882309F44BC081E0909112104D
:1001C000911180E003E023E049E653E414C09092EB
:1001D000550C8092540C80912E108111F1C08091A9
:1001E00088028823A9F181E0913009F080E000E2E3
:1001F0002EE345EF53E1612F0E940E7629C0C330F4
:1002000081F1C430D1F1C53009F458C0C63009F4C9
:1002100079C0C730E9F480911210873009F494C096
:10022000809188028823A1F07F926F925F924F9213
:100230001F9381E090911210973009F080E08F9326
:100240000E9421C60F900F900F900F900F900F906B
:100250001F5FCF5F143009F07DCF88E080930E10D0
:10026000AFC080911210833009F03CC080910D1016
:1002700010920D1081112EC035C090911210943043
:1002800009F054C080910D1010920D10811146C0DC
:100290004DC0B092550CA092540C80912E1081113B
:1002A0008FC080918802882399F281E0923009F012
:1002B00080E000E22EE34AED53E19DCF80911210E1
:1002C000853009F050C080910D1010920D108111F1
:1002D00042C049C081EE96EB0E94D97E80912E10DB
:1002E00081116EC080918802882309F4B1CF81E02A
:1002F00090911210933009F080E00EE32EE349EC68
:1003000053E179CF90911210963009F044C080915A
:100310000D1010920D10811136C03DC0D092550CB9
:10032000C092540C80912E1081114AC08091880295
:10033000882309F48DCF81E0943009F080E000E259
:100340002EE348EB53E157CF80910D1010920D1022
:1003500081112FC065CF81EE96EB0E94D97E8091EE
:100360002E1081112DC080918802882309F470CF4E
:1003700081E090911210953009F080E00EE32EE3B9
:1003800047EA53E138CFF092550CE092540C80913B
:100390002E10811115C080918802882309F458CF4E
:1003A00081E0963009F080E000E22EE346E953E177
:1003B00022CF0E94AA9D80912E10882309F430CF6D
:1003C000CF911F910F91FF90EF90DF90CF90BF9052
:1003D000AF909F908F907F906F905F904F90089517
:1003E000EF92FF920F93CF93DF9361E081E00E9441
:1003F000F46ED0911310C0E080E7E82E83E1F82E70
:10040000D1110BC080911210811129C080910D1063
:1004100010920D1081111DC022C0D13059F480916D
:100420001210813091F580910D1010920D108111F4
:1004300024C02BC0D23009F042C0909112109230EB
:1004400009F061C080910D1010920D10811153C000
:100450005AC00E94EE6F80912E108111B7C080911A
:100460008802882319F181E090911210911180E0A7
:1004700003E023E049E653E416C084E693EA0E94D1
:10048000D97E80912E108111A1C08091880288238D
:1004900069F081E090911210913009F080E00EE354
:1004A0002EE345E653E16C2F0E940E76CF5FDF5FAF
:1004B000C43009F0A5CF86E080930E1087C0D330FA
:1004C00061F480911210833009F040C080910D10CA
:1004D00010920D10811132C039C0D43009F58091CD
:1004E0001210843009F04AC080910D1010920D1046
:1004F00081113CC043C0F092550CE092540C8091A5
:100500002E10811163C080918802882379F281E0E6
:10051000923009F080E000E22EE34CE553E1C3CFD6
:10052000D53021F680911210853009F03FC08091BE
:100530000D1010920D10811131C038C081EE96EB74
:100540000E94D97E80912E10811140C08091880236
:10055000882309F4ABCF81E090911210933009F019
:1005600080E00EE32EE34CEC53E19DCF8AE89DEB57
:100570000E94D97E80912E10811128C0809188021E
:10058000882309F493CF81E090911210943009F000
:1005900080E00EE32EE342E553E185CF81E495EA66
:1005A0000E94D97E80912E10811110C08091880206
:1005B000882309F47BCF81E090911210953009F0E7
:1005C00080E00EE32EE347E85AE16DCFDF91CF9153
:1005D0000F91FF90EF900895EF92FF921F93CF93AA
:1005E000DF9388E3E82E80E1F82E15E0C0E0D0E04C
:1005F000F701EC0FFD1F60817181828193819B0166
:10060000AC010F946DBC81110CC02496C431D1058E
:1006100079F7115084E1E80EF11C1111E7CF81E068
:1006200001C080E0DF91CF911F91FF90EF9008957E
:10063000CF92DF92EF92FF926B017C0183E3C816A9
:10064000D104E104F10470F082E3C81AD108E10892
:10065000F10862E370E080E090E00F94F58C0F9475
:10066000297AECCFC701B6010F94F58CFF90EF907B
:10067000DF90CF900D94297ACF93C091440321E06D
:10068000209344030E941883C0934403CF9108959C
:1006900080911D0E81110AC08091A10E813041F020
:1006A0008091341582FB882780F9089580E00895B1
:1006B00081E00895129A08955F9A80E00E941C9547
:1006C0008A9A81E00E941C95809108018095817032
:1006D0008093060182E00E941C950C945A83CF936C
:1006E0000E947D91C82F8091B5138093B41380939D
:1006F000B3138093B21384E68093B1130E94909158
:1007000080ED93E09093510B8093500BC1110E94A8
:100710008A9181E08093150F0E94848E8EEF0F9452
:10072000AB41CF910D945F419091341593FB882795
:1007300080F993FF06C081E090912C13911101C0C4
:1007400080E0089580911D0E811110C08091A10E4E
:10075000823061F00E949483882349F0809134159F
:1007600082FB882780F991E08927089581E0089528
:1007700010928E0508958F929F92AF92BF92CF9262
:10078000DF92EF92FF920F93CF93DF931F92CDB73B
:10079000DEB75C016B017A014901F501808191812D
:1007A0000F94F8B78983002311F0F6018083BE010E
:1007B0006F5F7F4FC4010F94DA95F50180819181BD
:1007C000019691838083FFEFCF1ADF0A81E0E81A58
:1007D000F10819F780E00F90DF91CF910F91FF9012
:1007E000EF90DF90CF90BF90AF909F908F90089543
:1007F0009091C00095FFFCCF8093C6000895CF93E1
:10080000C82FCC2329F080E20E94F883C150F9CF91
:10081000CF910895CF93DF93FC018491EF0121964E
:10082000882321F00E94F883FE01F7CFDF91CF915A
:1008300008950F931F93CF93DF938B010E940A8437
:10084000E8018991882319F00E94F883FACFDF919B
:10085000CF911F910F91089580E397E10C940A8442
:100860008AE297E10C940A84FF920F931F93CF932F
:10087000DF93EC018B01F42E0F94D6760E942C842A
:100880008AE097E10E940A840115110511F40DEA2E
:100890001DE0209711F4C1E0D7E10E94E67D1F938F
:1008A0000F93DF93CF938AEF96E19F938F9381E02D
:1008B0008F930F94DA830E94966F60E080E00E942D
:1008C000FBA78EE79FE00E9497A74BEE56E162E000
:1008D00080E00E9426A84EED56E163E080E00E9491
:1008E00026A8EDB7FEB737960FB6F894FEBF0FBE39
:1008F000EDBF89EE93E030E6019729F0232F2A958A
:100900000000E9F7F9CFF89489EE93E038EE01970B
:1009100029F0232F2A950000E9F7F9CF0F94D67616
:10092000FF2019F00E945C8302C00E945A839099B4
:1009300002C0A895FCCF909B02C0A895FCCFE0E038
:10094000F0E0DF91CF911F910F91FF9019947F926A
:100950008F929F92AF92BF92CF92DF92EF92FF92CF
:100960000F931F93CF93DF931F92CDB7DEB77C0118
:1009700059018B016B01C40ED51E0C151D0559F1D3
:10098000F70180809180F80171908F017982C40114
:100990000F94F8B7781691F0672DC4010F9400B842
:1009A000C4010F94F8B79981891741F00E943084EF
:1009B0008DE595E10E940A8481E00EC0BE016F5F63
:1009C0007F4FC5010F94DA95F701808191810196DF
:1009D00091838083D2CF80E00F90DF91CF911F91E0
:1009E0000F91FF90EF90DF90CF90BF90AF909F90CE
:1009F0008F907F9008958F929F92AF92BF92EF92C7
:100A0000FF920F931F93CF93DF93CDB7DEB7A097DD
:100A10000FB6F894DEBF0FBECDBF6115710581051D
:100A2000910591F100E0842E912CA12CB12C102F76
:100A3000EE24E394F12CEC0EFD1EE00EF11C07FDFC
:100A4000FA94A50194010F941EB8F7016083B901CF
:100A5000CA010F5F611571058105910541F71F3FBF
:100A600031F1E1E0F0E0EC0FFD1FE10FF11D17FDAA
:100A7000FA9580818A3010F097E301C090E3890FE6
:100A80000E94F8831150EBCF80E3A0960FB6F89444
:100A9000DEBF0FBECDBFDF91CF911F910F91FF90B1
:100AA000EF90BF90AF909F908F900C94F883A0969A
:100AB0000FB6F894DEBF0FBECDBFDF91CF911F916F
:100AC0000F91FF90EF90BF90AF909F908F900895FF
:100AD000CF92DF92EF92FF926A017B010E940A841B
:100AE0004AE0C701B601FF90EF90DF90CF900C94E1
:100AF000FB84CF93DF93EB010E940A84BE0180E068
:100B000090E04AE0DF91CF910C94FB84CF92DF928A
:100B1000EF92FF926B017C0197FF0BC08DE20E9468
:100B2000F883F094E094D094C094C11CD11CE11CD3
:100B3000F11C4AE0C701B601FF90EF90DF90CF9023
:100B40000C94FB84AB01672B11F40C94F883BC016B
:100B5000990F880B990B4A30510511F40C94868536
:100B60000C94FB84CF93DF93EB010E940A84BE01B7
:100B7000DD0F880B990BDF91CF910C9486858F92B6
:100B80009F92AF92BF92CF92DF92EF92FF92CF935C
:100B90006B017C01B42E20E030E0A9010F94C8B1B4
:100BA00087FF07C08DE20E94F883F7FAF094F7F808
:100BB000F094C0E060E070E080E09FE3CB1541F08E
:100BC0002DEC3CEC4CEC5DE30F942EB2CF5FF6CFF6
:100BD0009B01AC01C701B6010F94CCB86B017C013D
:100BE0000F943FBA4B015C014AE00E94FB84CC2386
:100BF00089F1C501B4010F94CDB19B01AC01C701CE
:100C0000B6010F94CBB86B017C018EE20E94F88391
:100C100020E030E040E251E4C701B6010F942EB26B
:100C20004B015C010F9438BA6B01770FEE08FF0897
:100C3000C701B6010E948685C701B6010F94CFB1E6
:100C40009B01AC01C501B4010F94CBB86B017C01D1
:100C5000C150F1F6CF91FF90EF90DF90CF90BF9011
:100C6000AF909F908F9008950C94BF85CF92DF92A4
:100C7000EF92FF926A017B010E940A8442E0C70161
:100C8000B601FF90EF90DF90CF900C94BF858DE080
:100C90000E94F8838AE00C94F883CF93DF93EC01F1
:100CA0008991882319F00E94F883FACFDF91CF91C0
:100CB0000C944786ECEAF3E080818183089580916B
:100CC000AC039091AD03981759F0E92FF0E0E4558B
:100CD000FC4F82819F5F9F779093AD0390E00895D2
:100CE0008FEF9FEF08952F923F924F925F926F92F6
:100CF0007F928F929F92AF92BF92CF92DF92EF92AC
:100D0000FF920F931F93CF93DF93CDB7DEB72A9750
:100D10000FB6F894DEBF0FBECDBFF82E8091170E30
:100D2000843008F0DAC18091170E843008F001C1D8
:100D30008091AC039091AD03891B8F7709F4F9C0C2
:100D40000E945F8697FDEFCF8A3019F08D3009F051
:100D5000E7C010922E048091E4049091E504FC0118
:100D6000E15DFB4F1082892B39F01092E50410925F
:100D7000E4040FE214E003C00F94297AD4CFF80101
:100D80008191803211F48F01FACF8E3409F06AC05C
:100D90000115110509F466C06CE076E1C8010F94F5
:100DA00009B16C01892B41F06EE470E0C801049632
:100DB0000F94C6BD009709F4C8014AE050E060E016
:100DC00070E001960F9471AE4B015C018091E604D6
:100DD0009091E704A091E804B091E9040196A11D67
:100DE000B11D88169906AA06BB0631F0CD2821F45C
:100DF00060E089ED95E149C06AE270E0C8010F94B6
:100E0000F5BD9C01009709F1982F901BE12C9923C7
:100E100039F09150F801E90FF11D8081E826F7CFF4
:100E20004AE050E060E070E0C90101960F9471AEB5
:100E30004E2C512C612C712C641575058605970577
:100E400041F060E08AEB95E120C060E080E995E147
:100E50001CC08092E6049092E704A092E804B0924D
:100E6000E90416C08091341580FF12C06EE779E363
:100E7000C8010F9409B1009729F0FC0183818053C8
:100E80008A3030F460E080E995E10E9475AE51C08F
:100E90008091190E8130E1F067E470E0C8010F9491
:100EA000C6BD0097A9F04AE050E060E070E001960E
:100EB0000F9471AE643071058105910548F486EE9A
:100EC00094E10E940A8460E086E895E10F946983CA
:100ED00061E875E1C8010F94C9B0892B21F4109223
:100EE0007202109255056CE775E1C8010F94C9B004
:100EF000892B39F441E060E070E08AE598E00E94D7
:100F0000348467E775E1C8010F94C9B0892B11F4E7
:100F10000E946F8361E08FE294E00E94B9AE03CF3C
:100F200024EE34E04FE254E06EE274E00E9410AE32
:100F3000FACE8091341582FFD0C01A82198211E056
:100F400040913015509131156091321570913315E3
:100F500080912C1590912D15A0912E15B0912F15E3
:100F6000481759076A077B0708F410E000E680E19C
:100F7000E82E99E6D92E8091170E843008F0ADC086
:100F80001111ABC08091311390913213A0913313A2
:100F9000B09134138093301590933115A09332158E
:100FA000B093331541E050E0BE016D5F7F4F89E2A1
:100FB00093E10F946B6E019719F48B8190E002C05E
:100FC0008FEF9FEF409030155090311560903215A3
:100FD0007090331580902C1590902D15A0902E15A3
:100FE000B0902F1511E0481459046A047B0408F4EA
:100FF00010E08F3FFFEF9F0761F4481459046A0423
:101000007B0438F40E942C8481E196E10E940A84DA
:10101000B2CF4091530C8A3079F08D3069F048148A
:1010200059046A047B0408F47CC389819A8100977F
:1010300019F001969A83898310928F0489819A818D
:10104000FC01049FE00DF11D1124EA56F34F1082BC
:10105000892B31F01A82198280E00E94A4AE02C06E
:101060000F94297A481459046A047B0408F483CF46
:101070000E94848E89E293E10F94736B80912B150B
:10108000882331F1815080932B15D89EC001112403
:1010900062E08E5D914F0F94BB2DE0912B1524E003
:1010A000E29FF0011124E25EF14F408151816281A3
:1010B00073814093301550933115609332157093BE
:1010C000331589E293E10F94152C0F94DE2753CF4B
:1010D0000F94CD27E092190E4ECF0F942F8D4B0118
:1010E0005C01F1102BC380911D0E811127C310E00C
:1010F00040913F035091400360914103709142033E
:101100004115510561057105A1F08091F80E90918E
:10111000F90EA091FA0EB091FB0E840F951FA61F39
:10112000B71FA5019401281B390B4A0B5B0B57FF16
:101130000FC38091010290910202A0910302B0912D
:101140000402892B8A2B8B2B09F451C09091B41384
:101150008091B513981749F08092F80E9092F90E8D
:10116000A092FA0EB092FB0E42C0111106C30F946A
:101170002F8DC090F80ED090F90EE090FA0EF090FE
:10118000FB0E0091010210910202209103023091A6
:1011900004020C0D1D1D2E1D3F1DDC01CB01801B0B
:1011A000910BA20BB30BB7FDE8C28091A304811190
:1011B0001EC081E08093A3045F9A80E00E941C958A
:1011C0008A9A81E00E941C95809108018095817027
:1011D0008093060182E00E941C950E945A838091B0
:1011E000BC04882321F01092BC041092D00F80918F
:1011F000A1049091A204909902C0019604C018160F
:1012000019062CF401979093A2048093A104809175
:10121000A1049091A2048E3E92406CF00E942C8416
:1012200080E296E10E940A8440E060E070E080E0A5
:1012300090E00E9434840F942F8D6B017C0180918B
:10124000950490919604A0919704B0919804970109
:101250008601081B190B2A0B3B0B37FD57C0D70122
:10126000C6018C53964FAF4FBF4F80939504909318
:101270009604A0939704B09398048091060180FF90
:1012800006C04F9B04C07A9B02C0029979C2C092EB
:101290009104D0929204E0929304F092940480918D
:1012A000B20B882311F14090910450909204609009
:1012B0009304709094044114510461047104A9F0E2
:1012C0002091B00B3091B10BA8EEB3E00F9472B83F
:1012D000460E571E681E791EC418D508E608F70882
:1012E000F7FE03C09091AE0B02C09091AF0B9093AC
:1012F000900480910201911180958071809300018A
:101300006091900470E087E00F942D8C80919D0493
:1013100090919E04A0919F04B091A004A501940116
:10132000281B390B4A0B5B0B57FD23C19091B4135B
:101330008091B513981751F0E091B5133BE5E39F09
:10134000F0011124EA50FA4F608102C060918E05CD
:10135000662311F070E002C060E070E089E00F9455
:101360002D8C8091F70E882309F4F6C0E0903D02A1
:10137000F0903E0200913F021091400260910F11E7
:10138000709110116E5F7F4F072E000C880B990B28
:101390000F94CFB19701A8010F94C8B187FDDCC0AD
:1013A0003090B513212C1C821D821E828091B413B3
:1013B000831509F467C0832D90E04BE5489FF00149
:1013C000499FF00D1124E056FA4F458956896789E7
:1013D000708D452B462B472B89F4418D528D638DA3
:1013E000748D452B462B472B49F4458D568D678DC3
:1013F00070A1452B462B472B09F43FC05BE5589F56
:101400009001599F300D1124C90180569A4F6C01EB
:10141000FC0161817281838194810F941EBC2B0138
:101420003C01F60161A172A183A194A10F94CDB1F9
:101430006F83788789879A87F60165A176A187A14E
:1014400090A50F94CDB19B01AC016F817885898502
:101450009A850F94C6B9A30192010F942EB23B0155
:101460006C01222D3C814D815E810F9480BB18164A
:1014700024F4262C7C82CD82DE8281E0830D8F7065
:10148000382E94CF209135023091360240913702A8
:1014900050913802622D7C818D819E810F942EB2F5
:1014A0009701A8010F94CCB83B016C012090390240
:1014B00030903A0240903B0250903C029B01AC01BC
:1014C000B701C8010F9480BB18166CF09101A201FE
:1014D000B301C6010F9480BB18161CF47101820180
:1014E00002C0730186014090990450909A04609064
:1014F0009B0470909C049701A801C301B2010F9452
:1015000080BB1816C4F420E037ED43EA5CE3B70172
:10151000C8010F942EB26B017C0128E431EE4AE73A
:101520005FE3C301B2010F942EB2A70196010F949D
:10153000CCB87B018C01C701D801809399049093AA
:101540009A04A0939B04B0939C04B701C8010F9424
:1015500038BACB010F947C72F4E68F0E911CA11C5B
:10156000B11C80929D0490929E04A0929F04B09220
:10157000A0040F94297A8091190E882309F417C1C9
:1015800080910901817011E0182700910E02011766
:1015900009F440C0909134159062909334151093E3
:1015A0000E0281110DC064EF71E080E090E00E94B6
:1015B00018830F948C288091341583FD09C0E5C0F1
:1015C0000F94CD2780913415877F806280933415E6
:1015D000112309F4DDC0023028F460E08FEC96E1BD
:1015E0000F9469830E943AA783E0809388020F9446
:1015F0002F8DDC01CB018C599F4FAF4FBF4F809394
:10160000700F9093710FA093720FB093730F11111D
:101610000F94D9260F942F8D6B017C018091440388
:1016200081112FC080910002882359F180915605C5
:10163000882339F14091A4045091A5046091A60437
:101640007091A70497018601041B150B260B370B1D
:1016500037FD2AC0833079F03CF4813094F00E9449
:1016600030848FEA96E10BC0843059F40E943084B4
:1016700080E896E104C00E94308488E996E10E94E7
:101680000A842091000230E0A8EEB3E00F9472B813
:10169000C60ED71EE81EF91EC092A404D092A5045F
:1016A000E092A604F092A7040F94797F0F944285EC
:1016B0008091440381117BC080913E03882309F40B
:1016C00076C00F942F8D00913A0310913B03209127
:1016D0003C0330913D03DC01CB01801B910BA20B3D
:1016E000B30BB7FD64C00F942F8D6B017C0120916B
:1016F0003E0330E0A8EEB3E00F9472B8C60ED71EDA
:10170000E81EF91EC0923A03D0923B03E0923C03DC
:10171000F0923D0380E00F942C768AE00E94F883DB
:1017200046C0049FA00111244A56534F9E012F5FCB
:101730003F4F6FE874E00E9410AE1DCC8092F80E0F
:101740009092F90EA092FA0EB092FB0E11E0D0CC5E
:101750000E942C84609158057091590583E496E1AC
:101760000E9419848AE00E94F88340E060E070E003
:1017700080E090E00E943484DCCC1092A30437CD4A
:101780008091060F811183CD8ACD002309F442CFC9
:10179000023058F460E081EC96E10F946983809107
:1017A000D00F811102C00E94966F10E01BCF2A96C5
:1017B0000FB6F894DEBF0FBECDBFDF91CF911F9162
:1017C0000F91FF90EF90DF90CF90BF90AF909F90E0
:1017D0008F907F906F905F904F903F902F900895E3
:1017E000CF92DF92EF92FF92CF93DF936B017C0158
:1017F000D42FC091560583E08093560581E08093F5
:101800005505C114D104E104F10431F00F942F8D7A
:10181000C60ED71EE81EF91E80915505882399F043
:10182000C114D104E104F10421F48D2F0E947386C8
:10183000F3CF0F942F8DDC01CB018C199D09AE09DC
:10184000BF09B7FDF2CF10925505C0935605DF9141
:10185000CF91FF90EF90DF90CF9008951F920F925D
:101860000FB60F9211240F900FBE0F901F90189576
:101870001F920F920FB60F9211240BB60F922F9357
:101880008F939F93EF93FF939091C6002091AD03A8
:10189000E091AC0381E08E0F8F77281729F0F0E0FC
:1018A000E455FC4F9283E82FE093AC03FF91EF9156
:1018B0009F918F912F910F900BBE0F900FBE0F90A5
:1018C0001F9018958EBD0DB407FEFDCF08958FEFC4
:1018D0008EBD0DB407FEFDCF8EB5089590916400C6
:1018E0009B7F90936400982F906A96959CBD80FD95
:1018F00003C091E0863009F490E09DBD08959F9269
:10190000AF92BF92CF92DF92EF92FF920F931F930D
:10191000CF93DF9300D01F921F92CDB7DEB7E5E3E0
:10192000F9E10027BB27462F572FA82FAA2341F400
:10193000A52F542FB85FAA2319F4A52F5527B85FF8
:10194000A03138F45295A295452F4F70507FA42BAB
:10195000BC5FA03428F4550FAA1F550FAA1FBE5F05
:10196000A03818F4550FAA1FB395550FAA1FEA0FF8
:10197000F01F449151E0AA27B85081F1C8F0B0FFA0
:1019800002C0440F551FB1FF04C0440F551F440F40
:10199000551FB2FF06C052954295142F1F70407F0D
:1019A000512BB3FF1BC0A52F542F44270C94EE8C52
:1019B000B195B0FF02C055954795B1FF04C055954C
:1019C000479555954795B2FF05C05295407F429582
:1019D000452B5F70B3FF02C0452F5527DD24CC2473
:1019E000BB24B2E0649FD018C108B00AB00B749F4A
:1019F000C018B108B00B849FB018B109659FC0181A
:101A0000B108B00B759FB018B109859FB0196A9FD6
:101A1000B018B1097A9FB0194D9DA12C992499272E
:101A2000332722275D9DA00C911C901F301F201F83
:101A3000AD9D900C911D301F201F4C9DA00C911C42
:101A4000901F301F201F5C9D900C911D301F201F88
:101A5000AC9D900D311D201F4B9D900C911D301F92
:101A6000201F5B9D900D311D201FAB9D300D211D52
:101A70004B9F900D311D201F5B9F300D211DAB9F93
:101A8000200DB1E0BB24CC24DD24699FD018C1080F
:101A9000B00AB00B799FC018B108B00B899FB0187D
:101AA000B109639FC018B108B00B739FB018B1099A
:101AB000839FB019629FB018B109729FB019D61AEE
:101AC000C70AB80A20F0B1E09B0F301F201F112475
:101AD000692F70E0732BCB01A0E0B0E0BC01CD0119
:101AE000822B0F900F900F900F900F90DF91CF915E
:101AF0001F910F91FF90EF90DF90CF90BF90AF902C
:101B00009F900895CF92DF92EF92FF928091F6100E
:101B1000882371F1C090F210D090F310E090F4108F
:101B2000F090F51020E030E0A901C701B6010F9454
:101B3000C8B18823E9F020E030E040E05FE3C7016E
:101B4000B6010F942EB29B01AC010F942EB22BED77
:101B50003FE049E450E40F942EB29B01AC0160E0F9
:101B600070E080E89FE30F94C6B96B017C0106C06A
:101B7000C12CD12C80E8E82E8FE3F82EC092AA0465
:101B8000D092AB04E092AC04F092AD0460913302C9
:101B900070913402072E000C880B990B0F94CFB173
:101BA0002AE037ED43E25CE30F942EB2A7019601E1
:101BB0000F942EB260934D0270934E0280934F02A9
:101BC00090935002FF90EF90DF90CF900895CF92C6
:101BD000DF92EF92FF92CF93DF93C82FD0E0FE0108
:101BE000E15BF84E6491611107C00E94308485E387
:101BF0009AE10E940A846AE0FE01EE0FFF1FEE0FD9
:101C0000FF1FEE5AF84EC590D590E590F49070E025
